:020000040000FA
:1000000000400020C96B0100056C0100076C010075
:1000100000000000000000000000000000000000E0
:10002000000000000000000000000000096C01005A
:1000300000000000000000000B6C01000D6C0100CE
:100040000F6C0100195701002D7001000F6C0100A9
:100050000F6C010000000000310701000F6C01006F
:10006000991600000F6C0100F50601000F6C0100ED
:100070000F6C01000F6C01000F6C01000F6C010090
:100080000F6C0100857501000F6C01000F6C010001
:100090000F6C010031A401000DA40100D517000070
:1000A000E51700000F6C01000000000000000000D8
:1000B0000000000000000000000000000000000040
:1000C00010B5064C2378002B07D1054B002B02D02E
:1000D000044800E000BF0123237010BD9C020020F3
:1000E0000000000064C20300084B10B5002B03D0D1
:1000F0000749084800E000BF07480368002B00D10B
:1001000010BD064B002BFBD09847F9E7000000001C
:10011000A002002064C203009C0200200000000036
:10012000164B002B00D1144B9D46402292029A1A86
:10013000924600218B460F461348144A121A2BF0A0
:10014000F5FB0F4B002B00D098470E4B002B00D037
:1001500098470020002104000D000D48002802D01F
:100160000C4800E000BF21F06FFB2000290029F0BF
:1001700033FA21F041F8C04600000800004000209A
:1001800000000000000000009C020020300B002056
:100190000000000000000000014B58687047C04696
:1001A000C4090020014B18687047C046C4090020EC
:1001B000F0B5194E87B03368050000200C0001939C
:1001C00023F09DFB30600090206827F035F9019BFB
:1001D00007003360114E022D03D0A06813F0BEF863
:1001E0000600210063680831A81E039305F0AEFDE8
:1001F000009B04900593002203AB032130000FF015
:1002000085F8074B04009F4203D00100380025F019
:1002100021FF200007B0F0BDC40900208CE40200DB
:10022000D8F50200F8B50326050007003540022D79
:1002300016D10E4B0340062B12D0FF23DB05C4184A
:10024000B443201C00211AF08DFB002806D0802327
:100250001B06E418B443064B2C43E7183800F8BDDE
:1002600038000AF0C7FC0700F8E7C046070080FF27
:100270000000808010B50FF043F9040020000FF05B
:100280008BF9002801D1044810BD13F08DFA002825
:10029000F4D10248F8E7C04610D6020008D60200A2
:1002A00010B50FF02DF9040020000FF075F90028AB
:1002B00001D1044810BD13F077FA0028F4D00248A9
:1002C000F8E7C04608D6020010D6020007B5044B76
:1002D0000190002269460220009309F0A9FD0EBD9D
:1002E0000604000010B513F0BDF8034B002800D140
:1002F000024B180010BDC04610D6020008D60200FE
:1003000037B513F013F901AB7F2806D80121187017
:100310000122180008F088FB3EBD1F49820988426F
:100320000BD8402149420A431A703F2202408020E4
:100330004042104358704231EAE7184C010BA0428A
:100340000ED8202464422143197080215F34494231
:10035000224020400A43014399705A700321D7E795
:100360000F4CA04212D81024850C64422C431C7000
:100370003F258024294064422A40284021432243CB
:10038000204359709A70D8700421C1E70549064886
:1003900025F044FE16F00BFAFF070000FFFF0000F7
:1003A000FFFF100008340300ACFD020010B502008E
:1003B00002490A200FF030F910BDC046BE0400000B
:1003C00010B5020002490A200FF026F910BDC04600
:1003D0003E050000F0B585B0019202900D000022AC
:1003E00031490198039314F0F9FB0090002801D0E3
:1003F00043680093029B012B10D000263400019625
:10040000029B9E421FD0009B002B3DD12F68002CE9
:1004100040D12C68019701360435F1E700242868A3
:100420000FF06EF82700029002980FF0B5F8051E45
:100430000CD1002C07D122001C49019814F0CEFBEE
:1004400000281BD04468200005B0F0BD009B2E00A2
:10045000002B04D02900180026F0F5FF0600002C20
:1004600009D03A00310003980FF0D6F8104B9842AB
:1004700001D025003E002C003700D5E70D490E487D
:1004800025F0CCFD16F093F92968009826F0DBFFE3
:100490000700BCE7019A390003980FF0BDF8044B40
:1004A0009842B8D1B5E7C046D60600001E05000048
:1004B00010D6020029340300ACFD020037B501A9B3
:1004C000050008F05FFF1E4B04002B40062B05D0F3
:1004D000AB072AD11B4B2A689A4226D101992000EA
:1004E00028F085FD0190012822D1207843B2002B0D
:1004F00004DB012023785B0018433EBD7F230134D9
:1005000018403F3B034208D13F2223781900914312
:10051000802905D025F03DFBEFE798435B10F1E71C
:100520008001134001341843EFE7019B012BE0D019
:10053000019A054905480BF0C3FE16F038F9C0468C
:10054000070080FF081803004234030034FD020056
:10055000F0B5140087B002900391002223492000D7
:1005600014F03CFB002205002149200014F036FB6A
:1005700001230400049305931E4F002D07D06868E3
:100580001D4B984203D004A908F0FCFE07001B4E47
:10059000002C07D06068184B984203D005A908F0DA
:1005A000F1FE06000024029B154D9C420AD1002357
:1005B000059A019300933100280015F037FB0E488F
:1005C00007B0F0BD002C07D00023049A01930093DC
:1005D0003900280015F02AFB0399A3000022C9580E
:1005E000280012F0D3FE0134DDE7C046EE0500001E
:1005F000F6050000A2800300D8F50200B3660300F0
:100600008C2203007FB50D4D0400A84213D00C4E80
:1006100001220100300012F0B9FE0A49300028F032
:10062000C9FD04230293084B0394DB6902AA03214A
:10063000064801939847280004B070BDD8F5020021
:100640008C220300B366030028F20200C4C5020036
:1006500010B5040086B06A4602A8102110F018F9FF
:1006600001222100684612F091FE02A9024808F01A
:10067000A5F906B010BDC0460818030070B50C6897
:10068000E30726D4A30703D1254B22689A4220D042
:10069000012820D9486812F049FF0600200012F016
:1006A000A9FF051C30001BF023F9011C1D481DF09B
:1006B000C3FD011C041C281C1AF026FE1DF068FA5C
:1006C000211C1AF031FC032302249843164B0443E7
:1006D000E418200070BD200012F08CFF051C1DF0F6
:1006E00057FA061C1BF0E4F8311C0400281C1AF011
:1006F0002BFFFC218905051C1AF02EF9002803D0D8
:10070000013401239C4306E0BF21281C09061AF08E
:1007100023F90028F5D1200025F03BFA0400D8E7A2
:1007200044010300000020410000808013B5040054
:10073000080008F09BF96A46010020000EF064FEF4
:10074000009B0248002B00D1014816BD10D60200C4
:1007500008D6020037B50024022800D98C68486802
:100760000D6808F083F90A4B0100002C00D0094BFA
:1007700028006A4698470098002806D0019904008E
:10078000002902D000F00CFF040020003EBDC0464E
:1007900069F4000009F4000070B5040008001500B9
:1007A00008F064F92A00010020000EF085FE0148DF
:1007B00070BDC046D8F5020010B50EF0C7FE002887
:1007C00004D1034825F01DFC15F0F1FF10BDC04613
:1007D00074FC020030B50B0085B01400012805D967
:1007E0000A490B4825F01AFC15F0E1FF09480121E0
:1007F000C2680192019D0022A8472200039003A92C
:10080000012003F0BBF8039805B030BD7C34030031
:1008100034FD020004D40200F8B50E0000280FD108
:100820000400294B1D680021080024F047FA002726
:100830000600002D34D10025002C40D13000F8BD39
:100840000868830715D10268204B9A420DD125F024
:10085000F1F90500306812F081FD1D4BC2680024DB
:100860009A42E0D134680434DDE71A4903008A4231
:1008700002D012F073FD03009D6B002DEAD0164BE1
:100880002A689A42E6D00025E4E7EA68FB00995816
:10089000002904D0042902D0300003F00DF80137FC
:1008A000AB689F42F1D3C6E7A268EB0099580029D4
:1008B00004D0042902D0300002F0FEFF0135636845
:1008C0009D42F1D3BAE7C046C409002028F20200D5
:1008D000697C00008CE40200CCCB020010B504005F
:1008E000080022F0BAFC0300002C03D0012C06D033
:1008F000002003E00348002B00DC034810BD40004B
:100900002043FBE710D6020008D6020070B5456808
:10091000C6688468102025F01EF8034B4560C66049
:100920000360846070BDC046DCC8020070B50D0075
:100930004A688B680849040028F007FDEA68012A24
:1009400004D10649200028F035FC70BD0449200080
:1009500028F0FBFCF9E7C046A73403002FA70300EB
:10096000B434030030B5040087B00D000020042A21
:1009700020D1200022F071FCAB071DD1154B2A6855
:100980009A4219D103AA290010F0CCFE102024F0BD
:10099000E2FF114B039A0360E36861685A435218FF
:1009A0004260049A616801925A4352188260059A23
:1009B0005343C36007B030BD002301002A00206804
:1009C00012F08CFEE36858436368C31801205B0093
:1009D0001843EFE7B81E0300A0C80200F0B50500F9
:1009E00089B002AFB96016003B6001F0D3F9AB6883
:1009F0007B611423F81822F01AFD14237860F8188C
:100A000022F015FD032358437B68C0188300FB6068
:100A10002C2B29D86B46F8682A30C008C0001B1A56
:100A20009D46002302ACFB60AA687B6929009B1AE3
:100A300063607B682000A3613B680093BA68330061
:100A400000F00CF91A4E00217368200063616B6896
:100A500073600DF0B1FC6369B860736000280AD060
:100A6000022819D0134D08E0F8681C3024F080FFEC
:100A7000041ED9D1CEE7E3681D68FB68002B07D0C0
:100A80000023BB60200024F08DFFBB68002B0BD13E
:100A90002800BD4607B0F0BD7B6805339B00E31816
:100AA0005D68FB68002BEDD1280015F080FEC04684
:100AB000C4090020D8F502000122030030B513401C
:100AC00085B004004510002B14D128491D00884230
:100AD00010D0274988420DD0264B1500984209D0E6
:100AE0000323034009D1244A0168914205D125F02E
:100AF0008DF80500280005B030BD204A25002240B1
:100B0000062A05D0002B08D11D4B22689A4204D139
:100B100001A9200008F036FCEBE7200012F01EFCD3
:100B2000184B984207D1FF23DB05E01803239843B5
:100B30001AF0BEFEDDE7144B984206D101AA6946C1
:100B4000200024F03AFB019DD4E7104B984205D1D8
:100B500001AA6946200024F0C8F8F4E7022201A99E
:100B6000200028F02FF80028C4D0ECE7D8F50200C8
:100B700008D6020010D6020044010300070080FFDF
:100B800008180300141903009CDC020004D40200BE
:100B9000F7B506000F0000920193041E00D04468D0
:100BA0003800431E984120180430800024F0D3FE02
:100BB0000C4B050003600C4B5B684360009B83603B
:100BC000019BC360002E05D03100A2000831103017
:100BD0002AF091FE002F02D00434A40067512800AF
:100BE000FEBDC04654C90200C409002070B506000D
:100BF00010200D00140024F0AEFE034B466085600B
:100C00000360C46070BDC04618C902007FB50B0008
:100C1000012803D10021186812F0D2FB102102A88C
:100C200026F0CCFC0A4902A822F0B6FE039B0193F1
:100C3000002B06D1042804D1064825F0E2F915F06E
:100C4000B6FD02A9044807F0B9FE07B000BDC046D2
:100C5000C6650300CCF8020008180300F0B51600C2
:100C600042688FB0944606938369CA6805938B687F
:100C7000826063445A1C42601A78040001929A1CF4
:100C800042605A7804910092DA1C42609A780021FE
:100C900003921A1D4260DB789C4A029303001833CA
:100CA000C360059B1C309A1893000793C3182361F7
:100CB000079BB5000C331A0008932AF037FE149BEB
:100CC000009A5B190B93059B9B1A039A09939D1A33
:100CD000AB1D009A9B00E7180123B24268D2019A2B
:100CE0001A4207D13300009A89498A480BF0E8FA82
:100CF00015F05DFD009B05359900149BAD0059185A
:100D0000009B6519F01A05F021F8009E043F686009
:100D10000022964200D075E0069B002B03D1019B78
:100D20001B0700D4D9E002230026019A1A400A9238
:100D3000B24204D0069822F0E2FD06003860002797
:100D4000A3680B9D0893069B9F4264D1099D029A5C
:100D500007350499AD000332631992008A1819000F
:100D6000029E002E00D085E0029A92009B18079AFE
:100D70002832A218934200D285E00827009B089AE7
:100D80009B001C3DD31865190693039B9E4200D21D
:100D900083E065680DA825600D9522F048FB2D18AD
:100DA0006E1C2D78FF2D00D0A5E066600FB0F0BD61
:100DB000019A1A4205D00535AD00574B6519043F1D
:100DC0006B60069B002BA3D1019B1B07A0D4009B4B
:100DD000029A9A1A964213D3009A029B991A3200E9
:100DE0008900009B9A4200D392E79300049D581813
:100DF0002818089D0069EB1AE31898610132F0E7A2
:100E0000330071E7149908989300C958C31AE3187E
:100E1000996101327DE7009B039800221B189C46D4
:100E20002968624507D30A9B002B1ED13B493948EC
:100E300025F0F4F85CE7089B90001858814212D125
:100E4000059B013B9B1A9B00E318DA69002A05D039
:100E5000CA0833492F480BF033FA49E76A68DA6168
:100E6000013708356FE70132DBE76A68300022F0AE
:100E70007EFDF5E70868002801D110680860013E92
:100E80000431043A6DE7191D1B68002B03D1521A77
:100E900092102449DEE70B006CE7AA69002A11D101
:100EA000019B3B4211D002990498043189000858F3
:100EB0000699B3000430C95813F090FE002804D0FE
:100EC0004368AB610136043D5FE7009B1649F618A5
:100ED000089BB600F258D208BCE7039B002B01D058
:100EE0001249A4E7019B9B0700D452E7039822F024
:100EF00006FD38604DE7ED43059BED18AD00651923
:100F0000E8690BF09DFAE861350049E7FDFFFF3F16
:100F1000BA34030034FD020094DC020022350300E1
:100F2000F33403004B3503007D350300AD3503007A
:100F300070B5137804000A3BD8B20F2809D90A000B
:100F4000104811490BF0BCF90025A368186028006F
:100F500070BD002552781B021A43E3689D420AD1F6
:100F600023880025042BF2D1084906480BF0A8F984
:100F7000A3681860EBE72069A90009589142E6D000
:100F80000135EBE7B0FC0200573703006C37030074
:100F9000F0B585B004000D00100003A91E0023F079
:100FA000F4FC002809D12A000B490C480BF088F901
:100FB000A3681860002005B0F0BD039812F0E2FAB3
:100FC0000300B343F7D0030000962A000449034806
:100FD0000BF076F9ECE7C04613370300B0FC0200D3
:100FE0002B370300F7B51E0013780D000A3BD9B26A
:100FF00004001B480F2904D850781B02184326F020
:101000001AF903780193174B5A1C0023177801999A
:101010008F421BD141785778B94217D181789778A0
:101020008F4213D1002F0ED10E4A9B00D05CB042EC
:1010300008D933002A000C490C480BF041F9A36889
:1010400018600020FEBDC778002FEDD001330432B8
:10105000152BDBD12A00064904480BF031F9EEE7E5
:10106000C6650300CF37030083370300B0FC0200DE
:101070009C370300F0B5137887B005000E0001938C
:10108000992B47D103A9100023F0A3FC039B98429E
:1010900040D003781A000A3A0F2A0AD802000F2318
:1010A00031002800FFF79EFF01248440200007B094
:1010B000F0BDAE2B2ED123F087FC040023F07FFC83
:1010C00004900378B22B25D10127A33B22003100E5
:1010D0002800FFF787FF3C0005A98440049823F00F
:1010E00078FC059B04909842E0D0019904A823F075
:1010F0007FFC049A059B9A42D8D00F233100280028
:10110000FFF770FF3B00834004981C4323F057FC1B
:101110000490EEE73200044904480BF0D1F8AB68C4
:1011200000241860C2E7C046B4370300B0FC0200D8
:10113000F0B50E0087B0040004A930001F00019232
:1011400026F07EF8019B0500002B0CD1322E05D134
:10115000BF210902606922F090FA16E0482E00D003
:1011600078E0B549F6E7019B012B00D089E0412EDC
:101170000DD101003A682000FFF7DAFE0100606936
:1011800022F0D1FA002800D1C7E107B0F0BD422E0D
:1011900009D101003A682000FFF7CAFE010060692A
:1011A00022F019FBEEE7432E0AD101000F233A6823
:1011B0002000FFF717FF8E21C000C9010143C9E7D6
:1011C0000378622B32D1049B032B07D0052B2DD142
:1011D000C3785F2B2AD103796E2B27D101260023F8
:1011E00068787642954AD1184A78824205D1AA7821
:1011F00089788A4201D1914A9E5C03332A2BF1D12E
:10120000731C27D03A6829002000FFF791FE04994B
:10121000020000236069052904D12B79773B5D42E8
:101220005D41EBB2310022F09AFAABE7462E01D1D4
:1012300083498FE7472E01D182498BE7442E12D193
:1012400029003A682000FFF715FFFF231B02B42195
:10125000184214D0019B2A007B497C480BF030F8DF
:10126000A368186091E7452EF4D13A682900200060
:10127000FFF700FFFF231B021842EBD1BC2109023C
:101280009CE7019B022B00D0E8E07B681B780A3BBF
:101290000F2B48D8332E12D13A6801000F232000BB
:1012A000FFF7A0FE7A68060029000F232000FFF751
:1012B00099FE31000200606922F01EFA65E7002302
:1012C0000293342E1AD18026F6013A6829000723AA
:1012D0002000FFF787FE7A6801902900072320008D
:1012E000FFF780FE019A03003100606922F0FDF9EA
:1012F0004BE7029B013302930F2BABD0029B0322DF
:101300009E00534B711C591828002AF07CFC0028C1
:10131000EFD1EB78002BECD14D4BF65C80233601FE
:10132000DB011E43D1E7332E19D1802607233A680B
:1013300029002000FFF756FEFF23019029007A685C
:101340002000FFF725FE019BB60119020643314339
:1013500000E7A026EAE7C026E8E7E026E6E7352E24
:10136000F7D0362EF7D0372EF7D00023394A990020
:101370005018408886425BD18B5A200002933A680D
:1013800007232900FFF72EFE7E6803903378982B01
:1013900031D1300023F058FB00282CD1300023F04D
:1013A00013FB03789A2B26D105A923F012FB05998C
:1013B000060023F0F8FA02281DD1300023F0FFFACE
:1013C00007233200070029002000FFF70BFE029BD5
:1013D0000600DB0417D51F233A0029002000FFF781
:1013E000D7FDF100039B029E80011E433143F82686
:1013F000F6003040E2E62A00174914480AF060FF80
:10140000A368186026E76B4608229B5E002B07DA6C
:101410003E233A0029002000FFF7BAFD4008E0E72C
:101420007C233A0029002000FFF7B2FD8008D8E7AE
:101430000133062B9BD10DE730BF0000D4350300EC
:1014400072B6000062B600008E360300B0FC0200E7
:10145000D7360300102F030063360300019B032BD4
:1014600000D0F7E6382E21D100263A68072329005C
:101470002000FFF7B7FD7A680190072329002000BC
:10148000FFF7B0FD1F230290BA6829002000FFF784
:101490007FFD019F029B374381013943DE0056E700
:1014A00080263601E1E780267601DEE7392EF7D087
:1014B0003A2EF8D0362E2BD1C02607233A682900C1
:1014C0002000FFF78FFD072301907A682900200094
:1014D000FFF788FDBA687601137802900A3B0F2B5C
:1014E0000DD8072329002000FFF77CFD029BD900BF
:1014F000019B194331430F00810139432AE68023C0
:10150000DB001E43290007232000FFF741FDEDE724
:10151000372E00D09EE6D026CFE703490348A468C3
:1015200024F07CFD206030E6C3360300B0FC0200EE
:10153000F7B506000D0000240192019B9D420AD0E0
:10154000631C0093052B08D1B4681249124824F09B
:1015500065FD206000242000FEBD28780A38C3B253
:101560000F2B02D9B4680D49F0E76B7800021843DD
:1015700025F061FE023507002AF03EFB0228F1D17A
:101580003B78722BEED17B783034A342EAD1009CB9
:10159000D3E7C046FE350300B0FC0200313603003D
:1015A00070B505000C200C0024F0D5F9024B456005
:1015B0000360846070BDC046F4C902008022044B01
:1015C00052001A600123034A1360034A13607047F4
:1015D00000E100E00C8C0040008000408022054BC0
:1015E0005200DA67044BFF3A5A600022034B1A603C
:1015F0007047C04604E100E0008000400C8C0040D1
:1016000070B501251D4B1E4C18601E4BE550C046A1
:10161000FFF7E4FF1C4A1D4BE560E2500023032165
:101620001B4AFF20A3500432A15049190832A1508F
:101630008021C12209039200A150053AFF3AA3502C
:10164000C224144BA4001959C13A8143FF3A0A43FA
:1016500080211A510C341A5909061202120A0A433F
:101660001A51C0220434195981430A431A51802265
:1016700012041A60802252041A6070BDC802002051
:1016800000800040FC0F0000701700004C050000B7
:101690000405000000E100E070B51F4C1F4D636CB5
:1016A000002B0AD0002363641D4B1B689847A823B6
:1016B000DB00EA5800018018E850A36C002B09D029
:1016C0000023A364164B5B689847164B0001EA5849
:1016D0008018E850E36C002B0AD00023E364104B21
:1016E0009B689847A923DB00EA5800018018E8505E
:1016F000236D002B0ED000230B4A2365AB580B49FA
:101700005B18AB500A4A1368063313608022094BFA
:1017100012045A6070BDC046FC800040008000404A
:1017200004000020440500004C0500007017000074
:10173000C8080020FCE100E0F7B50191032823D898
:10174000134B8000C758C223124D9B00EF5001235A
:1017500044192364A8230F210F4EDB009C46E35855
:10176000AE59921BD218D3170B409A1801990B4B04
:101770001211C150C1239B00EF506346002001327B
:1017800012019619E650FEBD01204042FBE7C0461B
:1017900030CA0200008000404C0500000400002018
:1017A00003280BD8074B8000C158C223064A9B0070
:1017B000D150064A064BC2500020704701204042DB
:1017C000FBE7C04630CA020000800040BB35020083
:1017D0000400002010B5024B1B68984710BDC0469E
:1017E000C802002010B50024054AA358002B02D0DF
:1017F0000021A15098470434102CF5D110BDC046EB
:10180000B8020020074A89008B58002B06D1885067
:1018100080211800044A4904516070470120404269
:10182000FBE7C046B8020020FCE100E070B505000F
:1018300000291CDB032905D80800002418F0AEFE9F
:10184000181806060123023999430C00FE26B5211B
:1018500009023143280021F010FF002C04D0054973
:101860002800214321F009FFEE612C6270BD0024A5
:10187000F226ECE780B0000010B504000C2024F044
:101880006AF8034B446003600223037210BDC04634
:1018900084CB020010B50400102024F05CF8044B47
:1018A0000360237A0371636883600023C36010BD03
:1018B00048CB020010B50400102024F04CF8044B73
:1018C00084600360034B43600023C36010BDC046C7
:1018D00040DE02009738020010B5043027F0A0FA6D
:1018E000004810BDD8F50200002803D0012808D018
:1018F000002005E007224B680448934300D10448C8
:1019000070474B68DB085B001843F9E710D602000C
:1019100008D6020010B50349034824F07FFB14F0F9
:1019200046FFC0464838030040FA020070B5150073
:101930001A001C0013F052F9002802D04368002B53
:101940000BD12B1E04D1074B022C01D1FFF7E2FF74
:10195000012C00D14360180070BD022CFBD1002285
:101960004260F8E7D8F50200F8B504000D000B7AE4
:10197000124A9B00995827F01DFC1149200027F0BE
:1019800019FC2800FFF786FF01260700380021F028
:101990008CFF051E04D10B49200027F00BFCF8BD7D
:1019A000002E03D10849200027F004FC0122290061
:1019B000200011F0EBFC0026E8E7C046C0CB020097
:1019C00080380300863803008338030030B50025D3
:1019D00085B001A90400019521F048FFA84205D176
:1019E0000A490B4824F01AFB14F0E1FE636802A9CF
:1019F000083B63600368029343680393042328C091
:101A0000022004F0A3F905B030BDC046233803001E
:101A100040FA0200F0B513681400012287B00F6885
:101A20000D000092D9080223060008F05DFE022E88
:101A300012D10323686803401DD101682B4AC9688D
:101A4000914218D12A68904206D0059305A968688A
:101A500021F00CFF061E06D1002563689D4233D39A
:101A6000234807B0F0BD381D0122316813F0B6F8E5
:101A700073684360EAE70DF043FD039003980DF0AF
:101A80008BFD0028E8D00DF03BFD05000DF084FD36
:101A9000029028000DF080FD060028000DF07CFD6E
:101AA000029B002B03D0002E01D0002805D0114945
:101AB000114824F0B3FA14F07AFE381D012202997D
:101AC00013F08CF84660D9E7A368EE009959002915
:101AD00009D0042907D0381D012213F07FF8A3682C
:101AE0009E19736843600135B7E7C046DD1C0000EE
:101AF000D8F5020050380300ACFD020073B50C00AD
:101B000015001B280DD000231F2808D1081D002216
:101B1000290013F063F81A4B002800D1194B180064
:101B200076BD0323194208D1174922688A4204D19D
:101B30002B4002D129689142F1D0AB07EED1134B73
:101B40002A689A42EAD16A6863685340072293433D
:101B5000E4D1019301A9200021F088FE061E01D1E5
:101B6000074BDCE7281D0022316813F037F8002806
:101B7000D4D04168706811F087FC0028EAD1CDE725
:101B800010D6020008D6020008CC0200CCCB02001E
:101B9000F7B50B681C4A04000D00934203D05A6845
:101BA0001A4927F0D2FB1A49200027F003FB002333
:101BB0000127019301A9280021F058FE061E0CD12F
:101BC0001449200027F0F6FA2B680F4A934203D0FD
:101BD0001149200027F0EEFAF7BD002F03D10F497D
:101BE000200027F0E7FA01223168200011F0CEFB37
:101BF0000B49200027F0DEFA01227168200011F065
:101C0000C5FB0027D6E7C046CCCB02004238030014
:101C100046380300CD3703002FA7030083380300A5
:101C20004269030010B504000C2023F094FE034B1E
:101C3000446003600023037210BDC04684CB0200E1
:101C400010B504000C2023F086FE034B44600360B3
:101C50000123037210BDC04684CB020010B50430CE
:101C6000002212F0BBFF002805D10449044824F0EB
:101C7000D5F914F09CFD406810BDC04648380300FB
:101C800040FA020010B5024B08C027F0AAF810BDB8
:101C9000CCCB0200F8B5070048680E000DF030FC10
:101CA000040011F05DFD0C4D022F00D9B56800282D
:101CB00009D121F024FE060020000DF06DFC011E6C
:101CC00003D13000F8BD4010F3E7331D01221800A6
:101CD00012F084FF4560EFE7D8F50200F0B5070089
:101CE00089B000201E000D00019221F008FE0E4B6D
:101CF000040007609F4203D1042302791343037158
:101D0000019B2B430DD03368AA00B218019905A896
:101D10000394049327F077F8681C05AA03A9FFF73A
:101D200079FE200009B0F0BD08CC020010B5002AF1
:101D300003D121F026FE08480AE0042A09D1043024
:101D4000002212F04BFF002801D1FFF7E3FD4068AD
:101D500010BD21F00CFEEEE7D8F50200034B82B077
:101D600001AAA0331A6002B07047C046C40900201F
:101D7000014BA43318607047C409002010B5034913
:101D8000034824F044F914F012FDC046FE08000098
:101D90002CFC0200064B07B51A00A033A4321B68C6
:101DA000126801A95B1A9A4201D8FFF7E7FF07BD45
:101DB000C4090020F0B50E4C421E27681100002017
:101DC000BE09FB0F73407B403E097D087340BF088E
:101DD0007B406B40DB072B4301251F0040002B405D
:101DE0001843E940ECD18242E8D32760F0BDC046F9
:101DF000CC02002070B50123A12400250B4A0C4819
:101E00001360E4000421002345604668002EFCD0E6
:101E100016591B02013933430029F5D1002BF1D0AB
:101E200004490B600123536070BDC04600D00040E0
:101E3000FCD00040CC020020014B18607047C04627
:101E4000CC020020F8B5224E3568686801281DD9FB
:101E5000AA68431ED15C0A2918D1002B03DD591E44
:101E6000545C0A2C13D11C00844202D2115D20293B
:101E70000FD0002B0FDC1218023AE31A14789B08DB
:101E80003A3C614261415C18002C11D1F8BD0B0055
:101E9000E3E70134E8E7611C8842ECD1591E0029D0
:101EA000E9D00139575C0A2FF0D0202FF7D0E2E7B4
:101EB000084F04223900280025F05FFB0421380078
:101EC00005F07CFC3369013C04333361DCE7C04638
:101ED000D00200209F80030010B52022002102487C
:101EE00029F024FD10BDC0460C0A0020084B10B597
:101EF000426818600020986018750138D8600800A2
:101F00005A601A61996123F027FAFFF79BFF10BD11
:101F1000D0020020F8B503780400002B1DD00F4E2E
:101F2000B06C002804D0210029F05CFE002814D0F9
:101F3000200029F061FE471C380023F019FD051E22
:101F40000BD03A00210029F0D6FC054B054A196850
:101F5000043B99609A42FAD1B564F8BDC4090020E7
:101F6000240A0020080A0020F0B5B64C06002068BC
:101F7000A568436885B00193002D00D010E1731E61
:101F8000042B0AD825F062FB6368984200D1A3E0D5
:101F9000012E00D140E1022E10D0032E00D19BE093
:101FA000042E13D1206821694368994200D32AE1A5
:101FB000012225F0E3FB0025012726E12369626861
:101FC000934200D94EE10126764285E0052E00D1EC
:101FD0000EE1062E0FD123685D682369AB42AD4147
:101FE0006D42002DEFDD2368290098682369C01831
:101FF00005F0E4FB20E00B2E22D1019B2269206832
:10200000991A25F0AFFB2368019A5B689A4204D9BC
:1020100013002269981A05F009FC226823695168A7
:102020009068C91AC01805F0C9FB2368586823696D
:10203000C01A401B05F0E8FB23695D192561C2E762
:102040000E2E13D1E368002BBDDB2068013BE3605B
:1020500062684368991A25F085FBE368002B17DB5B
:102060001233794A9B00995820680FE0102E16D140
:10207000E368062BA7DC5A1C734913339B0059589D
:102080000029A0D020686368E260436025F02AFB45
:1020900063682269D61A22685568ED1A0BE0152E7E
:1020A0000DD12369626861689A1A206825F066FB81
:1020B000236962689E1A0127002E30DCA3E70D2EEB
:1020C0000DD1624823F048F9206825F0F1FA6368E1
:1020D0000026C018FFF71EFF300005B0F0BD012339
:1020E0001B2E66D0082E01D07F2E21D12169626877
:1020F000914200D867E7002320688668B618F75C2D
:10210000202F13D101339F188F42F8D30126032BC0
:1021100000DD0336891B320025F030FB012730003B
:1021200005F072FB23699E1B26617FE00126F1E723
:10213000092E29D163682269D11A22689068444A1D
:10214000C01803AB13F05EFC061E00D13BE700276E
:10215000431C0BD1A06923F0FFF863682269D11AF0
:1021600022689068C01805F029FB4CE723692068B5
:10217000F918039B01375A1C03921A7825F0E0FAEC
:10218000BE42F3D135003EE73300203B5E2B00D941
:1021900019E732002169206825F0DBFA012532E7D2
:1021A000012D08D104234F2E03D002235B2E00D033
:1021B0000023A36007E7022D21D13300303B092B18
:1021C00003D803232675A360FDE60023A360412EF8
:1021D00000D14DE7422E00D134E7432E00D1FAE67C
:1021E000442E00D1EAE6482E16D0462E00D0EAE66C
:1021F000002723683E005D682369ED1A11E0032D76
:1022000028D17E2E03D000252F002E0009E0237D4B
:10221000312B01D0372B0DD100252F0023696268A7
:102220009E1A0023A3609E4200DD78E7002F00D1B4
:10223000D7E6E8E61A00FB21343A0A42D8D0332B1D
:10224000E1D1AFE6D0020020C4090020B26603004D
:102250008C2203000023042DABD1462EC8D0482E7B
:10226000DAD0A6E7002501262F0058E7F0B50F00C9
:10227000496887B005001600002901D0002A05D161
:102280003900280021F0B0FC07B0F0BD0F3213096F
:10229000C918019321F01AFC0F22A868B9687C685C
:1022A000324000D11032019B1E19254BF3185B0000
:1022B000C3180393224B1020E3185B00CB189C46F5
:1022C000039B210002930023801A0590002922D14C
:1022D00003986400041B1020821AD34018482380FE
:1022E0008446019B5B00E41A019B023463445A005C
:1022F000200029F01BFB002E04D07300023BE35AA0
:10230000002B1BD001216E603A782B780A408B435A
:1023100013432B70B8E76046008801390343180067
:102320000493059BD840029B18800298049B0238B6
:102330000290022040421B048444C7E7013EDAE7D2
:10234000FFFFFF7FF0B54B681500526889B00600AB
:102350000C00934201D22C000D0001272278616805
:102360003A4000D12A783A405118300021F0AEFBB3
:10237000B3683800019363682978029323781A00C0
:1023800098430300A8684A400490A0683A4003902C
:1023900001988F43BC460590029F68680299C01B54
:1023A00001390690481C17D1029B5900019B59180E
:1023B000002A02D001230B800231019821F072FB28
:1023C000012170602B7822785A4033780A408B4381
:1023D0001343337009B0F0BD0398078812483F18C3
:1023E000FF18069B5B1899421CD3049B1B881B1883
:1023F00004980230049038006344584000936B46C0
:10240000D883D88B009B84460598624402800230B2
:10241000059003981B0C02309C46120C3B0C039059
:102420000139BFE7004BE6E7FFFF0000F0B591B0D0
:1024300007935B6804000E000692002B03D14360F3
:102440004B6011B0F0BD069B5B68591C019321F0F5
:102450003DFB069B00215B68A0685A1C520001935B
:1024600029F064FA00236360069B30005B68591C06
:10247000019321F02BFB0699300021F0B5FBB368E6
:1024800075680293079B9B680393079B5B680593A2
:10249000A3680893059BAB421AD81BD3039A290063
:1024A000029821F058FB002810D10123089A70608F
:1024B00013806360069B1A78079B1B785A400123A0
:1024C0001A42BED0227813432370BAE7002801DAFB
:1024D0000023EEE78A4A059B9B185B009C4600227E
:1024E000039B634404931B8801921AB2002A6CDA9E
:1024F000634610200027991C039B019A5B180993DF
:10250000821A039B0A92099A934264D300201027EF
:10251000029A6B00D0526A1C029D099272609A1C4A
:10252000AA180A922A00019D791B0B910A998A42E6
:102530005CD3049A12880D92029AD518059B099AC9
:10254000D11A6F4B6160C918089B49005B180A9348
:10255000022362465B429B1A0F9373680B930B9A9C
:10256000059B93424DD310220020019BD21A039B5E
:1025700004998B4200D8A8E0614A102194460025B6
:102580000B9B029A63445B00D318019A891A029A42
:102590009A4200D8A7E06368002B07D0584A0899F0
:1025A0009A185200525A002A00D1A6E07368002BF4
:1025B00000D17FE7524A02999A185200525A002AD3
:1025C00000D077E7013B7360F0E7019A5B000132CE
:1025D0009BB292B288E71A880198110081400F439C
:1025E0000A991F800A41023397B28CE71588019936
:1025F0002F008F400B9938430D411080A8B2023252
:1026000094E7AB1E28880E931B88000418430D998D
:1026100017F0E2FF002284460F9BEB180C93039BFC
:102620000C9909938D4212D82B889A422BD3D31A36
:102630005A42190C9BB22A805A1E9341CB18099317
:10264000099B002B21D0039F0C99002030E06046AD
:10265000099B0F881B884343BB4202D2F81A904261
:102660000DD8DB1B9B189FB2781E87415A420A8007
:102670001A0CD219099B023102330993D2E7821A4C
:102680000A800022F6E79A1A2A8062460A9B0E9D6B
:102690001A80023B0A930B9B013B73605DE70B883A
:1026A0001A003B880237D31818180880000C023132
:1026B0008D42F4D82B881818099B2880000C1B1A0F
:1026C000099301235B429C44BAE7049B019D1B884C
:1026D00019002941934001430498018098B2049B5A
:1026E000023B049343E71A88019F100038418A4057
:1026F0002843188095B2023B49E7013B63604AE7F3
:10270000FFFFFF7F436870B55A00002384680A4DBD
:10271000A218944206D30278D20700D55B4201206A
:102720000B6070BD023AAB4203D816881B043343DA
:10273000EFE70020F5E7C046FF7F0000F8B51F0077
:102740008B1E160000241E2B14D80B4B4068595CBE
:10275000000117F041FF0500A74204D0013003211A
:1027600017F03AFF0400301E01D029F045FA033576
:102770002C1924182000F8BDAA380300004870471F
:10278000ECCC020070B506000D00002814DD002915
:1027900007DD154817F0AAFF0124864209DC002452
:1027A00007E00100C020000617F0A0FF01248542C9
:1027B000F5DAE4B2200070BD002907DDC020000674
:1027C00017F094FF01248642F3DBE8E70024A042DF
:1027D000F0D00100044817F089FF0123854200DB97
:1027E000231CDCB2E6E7C046FFFFFF3FF7B5002839
:1027F00006D13A4A3A493B4826F0A7FD3A48FEBD81
:102800000D68280010F0AAFD43680600EF2B04D1E4
:102810006D68280010F0A2FD06000023334AD9009D
:102820008858A84205D1521851682E4826F0C2FC9B
:10283000E4E70133612BF2D12D4B2A4C9D4201D0AC
:102840009E4202D12B492000F0E72B49200026F0C0
:102850007CFD0021280010F0B3FD7268274920009C
:1028600026F073FD264B9E4228D1280023F0E2F982
:1028700021F090F80025061EC0D073689D42BDD29D
:10288000B268EB00D3181F68002F15D05B681D4994
:102890002000019326F059FD0021380010F090FD32
:1028A0001949200026F051FD0021019810F088FD03
:1028B0001649200026F049FD0135DEE7144B9E4203
:1028C00000D12E00B06B002898D0830796D1114B11
:1028D00002689A4200D091E7CAE7C0463E39030039
:1028E000F2BC03008C220300D8F5020048CD0200A0
:1028F000FCD90200B53D0300D13D0300D93D0300E2
:1029000028F20200A1800300E93D0300B366030042
:102910008CE40200CCCB0200002313B5044A046A05
:1029200009050093890C8A58A16B21F04DFF13BD56
:102930005CD00200F0B587B000931B7804000F0054
:1029400002927C2B05D18268525C002A01D09A2A1F
:1029500014D11A006B3A022A2DD8A568E819037819
:10296000032B5ED104A9666821F0FAFFAB199842E7
:1029700006D167600499200021F056FF07B0F0BD32
:102980000378032B4DD105A921F0EAFF009B1B78AA
:102990006B2B04D1049B059A13430493E6E76C2B3D
:1029A00003D1049B059A5340F7E76D2BDED1059BBD
:1029B000049A1340F1E76E2B04D0022219009143D0
:1029C000702966D1A368D81901930378032B28D105
:1029D000636804A9039321F0C3FF0600019B039AD7
:1029E0009B189E42C5D0B378B01C7578032B18D1C4
:1029F00005A921F0B5FF0600372D15D1059A1F2A2C
:102A00000FDC4149049B114199420ADBC0210906B0
:102A100011418B4205DB93400493049A53005340C9
:102A2000DCD5029D00224FE0392D08D1059B1F2BDC
:102A300001DD1F230593049B059A1341ECE72F2D1D
:102A400003D1049B059A9B18E6E7302D03D1049B24
:102A5000059A9B1AE0E7312D09D105990498FFF7F3
:102A600091FE0028DDD1059B049A5343D4E7332D12
:102A7000D7D00599352D06D10029D2D0049821F060
:102A800006FE0490C9E70029CBD0049821F00FFE80
:102A9000F7E7752BC5D1A368D8198378032BC0D16C
:102AA0004578023021F06BFF2F2D01D1049060E7B3
:102AB000302D06D1404243000490584000D458E7DE
:102AC000AFE7C043F2E73200561CED09FBD1636863
:102AD000DB1B01930135DB09FCD1023252193900AD
:102AE000200024F00BFE0400009B029A1B783100AA
:102AF0001A330370013021F0E9FD701C2018019A8F
:102B0000290021F0E3FD39E7FFFFFF3FF0B597B063
:102B10000890C020002540230AAC80000F0016005A
:102B200025706360A56022F023FF2561E060656188
:102B3000A561E5612762E562A84218D1C349C4488E
:102B400023F06CFA0023060013930D9822F02AFF5D
:102B5000002E00D1E0E10023BA6B3968300009F0A3
:102B60001FFC380024F0A9FB300013F020FE321EB9
:102B700003D00422022E00D0033A0026B549009665
:102B8000920052582000B96B330021F01DFE102036
:102B900022F0E1FE1021040024F010FD0AADAB6824
:102BA000002B00D194E12A78002A00D090E1013B6B
:102BB0000C32AB605343EA68A649D318DA785D68F3
:102BC0009200525802921A689B681202120A0393EA
:102BD000029B05925B7806930F23069A1340049399
:102BE000002D01D1636803933023069A1340102B04
:102BF00027D0202B66D0002E00D042E10123069A78
:102C00001A400992099A02992A405300CB18802150
:102C10005B88490107931B0B1B038B4200D048E1E3
:102C20003B00079940331B780905090D8B4200D002
:102C300026E1002A00D11EE1380024F0AEFB013568
:102C4000E0E7002D0BD180213800029B6A009A1822
:102C500049014030049BAB4205D801269EE7002E77
:102C6000F1D100269AE753881E0B36038E4214D109
:102C700006781B0502321B0D9E4221D121000AA8B5
:102C800021F0E1FD0028ECD13B0040331B78062BFE
:102C900000D035E17049714852E7049A6B1C9A42A2
:102CA00006D9039A059900920AA8029A21F08CFD90
:102CB000029B6D005D1969880AA8FFF72DFED0E719
:102CC0000135C7E7002E0BD0029A6B009B5A1B0BF5
:102CD000032B48D10121200024F0D8FC00230370ED
:102CE000029B6E009E19049BAB4240D800238020BB
:102CF0001E004001049A934269D3A368039A98186E
:102D000000230693A2686368D31898426DD3029B90
:102D10001B781F2B01D02E2B00D10126029B597846
:102D200040230B4018004342434149B25B421E40DE
:102D3000002900DA01260025039B0495D018079589
:102D4000069B9D4258D1002E02D1079B012B63D0D8
:102D50000499200024F006FD029B059A03992000A7
:102D6000FFF7E8FD7DE7012D00D876E78CE78021AD
:102D7000738849011A0B12038A4226D13A00403265
:102D80001278DBB29A421CD1082A07D1B96CF86CD0
:102D90000AF01AFD0100200021F00CFD002D0AD1DF
:102DA000029B5B787F2B06D90E9B2000591C069353
:102DB0000E9121F039FD380024F0EFFA013502368A
:102DC00091E7002D00D148E75EE76B1C69E70299A7
:102DD0005A008A185288110B0903814203D1D2B2DA
:102DE000072A00D90126013384E7069B012101331C
:102DF000069321F08EFC85E7049A03780132049251
:102E0000002B04D0079B0133079300230493012177
:102E100021F07FFC013593E7A268039B944663444D
:102E20001D00069B9E4200D11BE72B78002B07D18B
:102E3000A3680122E91A200024F0A0FC0136F0E783
:102E40002800012121F065FC0500F7E7915F0300F0
:102E500000FB02005CD00200B95F0300C8F9020069
:102E6000012D00D1F9E601232A001A402ED0049A40
:102E7000032A0DD008E721000AA821F0E4FCDEE6D1
:102E80000135049B022BEBD10023012D00D1E4E698
:102E9000069A691ED20705D5029A9288120B012A5A
:102EA00000D16908012900D056E7002B00D1D8E6EF
:102EB00052E7039A059900920AA86B1C029A21F026
:102EC00083FC07990AA8FFF727FD67E61300DFE7F1
:102ED0002B78002B00D031E63B0040331E78002ECB
:102EE00000D0D1E66368002B00D1CDE62B6920002D
:102EF000591C21F099FCA3686B62EB69AB6224E674
:102F0000022B01D10949C6E60B3B09480949012BAF
:102F100000D815E6084913E6380024F0CEF9089ADF
:102F200013AB13CB13C2089817B0F0BDCB5F0300EF
:102F3000B0FC0200FF5F0300266003000022104B7C
:102F400010491A6003001233FF3341185A701A7087
:102F500004338B42FAD10100030000220931083307
:102F6000FF311A709A705A70DA7004339942F8D1AE
:102F7000C3237F229B00C254034A044B1A6070474C
:102F8000EC020020110300003E600300100000204E
:102F9000F0B500267E24330031009A008218FF32FB
:102FA000577C7F2F44D0927CB618F6B25A1CEF2E75
:102FB0002BD9C1267D25B60086193700AC46D2B282
:102FC000944516DA92008218FF3251749174D174CC
:102FD00011757D220233DBB29A4211DA00269A0083
:102FE0008218FF3254749174D17411750133DBB2BD
:102FF000D3E73D68043FBD6001256D42AC44DFE787
:103000003568013A7560043EE6E77D2FEED8094D3C
:10301000EF5D01252F42E9D0D3B2C1227D26920077
:1030200082189E42DADB1568013E5560043AF8E7E3
:10303000F0BDC0462161030070B5012240240F4954
:10304000531EDBB29B00C318FF335D7C7F2D13D072
:103050004D5D25420DD05D7D7F2D0AD04D5D7F2DCC
:1030600007D9DD7D002D04D06EB2002E01DB0135C5
:10307000DD740132D2B2E3E770BDC046D060030018
:103080000300F7B500214B4A1333FF338218197040
:1030900004339342FBD1FC2300249C462200844449
:1030A00053B2002B04DA444A444B00201A6008E073
:1030B00063461F69BC4205D37F23443292001354F8
:1030C0000120FEBD6346DE68355D602D01D9203DDF
:1030D000EDB2611CC9B28F424FD0735C602B01D935
:1030E000203BDBB2232D4BD1303B092B01D9344A95
:1030F000DAE70234E1B28F4204D8FF2BF7D84370ED
:103100000C00CDE7745C2500303D092DF5D80A256B
:103110006B430131303BE318C9B2ECE70136512E65
:103120002FD10023274C1F5DDEB22A2F0CD1264F52
:10313000FF5CAF4208D19300C318FF335E7444783C
:1031400001321C75D2B2DBE70133512BEBD11F4C9E
:10315000493B08342678AE4207D0013C002B01D110
:103160001B4AA1E7013BDBB2F4E7002BF8D01400C7
:103170004334A4000419A370C2E7232DB7D0002361
:103180000026F7B20197104FF75DAF42C6D10D4F41
:10319000F75D2A2FC2D09F42C0D1694693000979BA
:1031A000C318FF3359744178013202341975D2B211
:1031B000E1B2A5E712030000416003001000002007
:1031C00053600300606203000F620300B1620300FA
:1031D0006160030010B51130084A0949FF300378D7
:1031E0007F2B00D110BD02240457002C03DCCB5CE4
:1031F00043700430F3E7D35CFAE7C046BF610300D5
:103200006F61030084460023F0B585B09F006744DA
:103210003800FF30417C7F2901D105B0F0BD022488
:10322000544A525C224202D10133DBB2EEE7012460
:10323000224246D11A190C19E4B200944E4C7D2555
:1032400064186478D2B20194C47C007D0294039027
:10325000C120800060440400954228DA6C46920048
:1032600024786244FF3254746C4624798D1C947423
:103270006C46247AEDB2D4746C46247B14753E4CB3
:103280009A1C61183C00FF348E78217DE77C009108
:103290007D21D2B291420FDA92006244FF3255741E
:1032A0009674D7746946097803331175BDE72668AB
:1032B000013D6660043CCFE704680139446004388E
:1032C000E8E71A000132D2B21000644644308000B0
:1032D000005D0028F6D05A1C7F2809D00825254C0F
:1032E000245C2C4201D0D3B290E724380128FAD9CB
:1032F0003C00481CC0B200901F48FF344018407882
:103300007D260190E07CD2B20290207D0390C12006
:10331000800060440500964222DA6D4692002D78C6
:103320006244FF3255746D462D79134E95746D4687
:103330002D7AD5746D462D7B15758D1C71188F787F
:10334000217D9A1C00917D21E67CD2B2EDB29142A2
:103350000BDA92006244FF3255749774D674A1E779
:103360002F68013E6F60043DD5E704680139446071
:103370000438ECE7D06003006F610300F7B500216B
:103380008B00C3181A00FF32547C9C46002C02D1DB
:103390000131CBB24AE07F2C00D129E11026954BB8
:1033A0001D5D4B1C35422BD0AD06ED0F2C00D67C9D
:1033B000177DC1227D25143492000194DBB282185E
:1033C0009D4218DA6A469B001279C318FF335A747B
:1033D0000022DE749A741F756246FF32547C4B1CC7
:1033E000352C00D0C6E0517B834C615C490700D48A
:1033F00092E0102187E01468013D5460043ADFE751
:103400004E2C1ED118210D25D47C5574167DC12259
:103410009200DBB2821870359D420DDA9A00821854
:10342000FF3251740021D474917416751900A7E706
:103430001B21E8E71C21E6E71768013D5760043AC5
:10344000EAE74F2CF4D0502CF4D06DB2002D2CDADA
:10345000D57C002D29D0DBB21D004435AD002D5C9C
:10346000002D22D18E1CF5B20195AD004519FF3516
:103470006F7C7F2F19D05F4EF75D7F2F15D9EF7CC2
:10348000002F12D0C1227D2192008218019C8C4213
:1034900006DD1F226A740022AA74EA742A75C5E741
:1034A000146801395460043AF0E74B1C172C2CD1F6
:1034B000557B4C1EE4B2452D1CD12A2353732300A7
:1034C00043339B001B5C4B4AD55C4B1C7F2D23D99F
:1034D0000134E4B2A4000419FF34617C00297FD0D8
:1034E000525C7F2A18D9E27C002A15D162461E213F
:1034F000FF3208E0392D01D12C23DFE73D49495D3A
:103500007F2909D91221517406E0182C08D1517B6A
:10351000384C615C7F2901D8DBB287E71321F2E7E1
:10352000202C04D1517B3C29F6D12621EBE7482CF5
:1035300015D1547D7F2C02D14B24547403E02D4DC2
:103540002C5DA406F8D5547C2A4D2D5DED0700D4E2
:1035500042E7557B202D3CD10C3C5474DCE73C2CDD
:10356000F1D1517D7F29D7D0224C615C8906D3D41B
:103570003F21C8E72A2C17D1D17C147DC1227D259B
:103580009200DBB282189D4209DA2B259A0082183C
:10359000FF3255740025D1749574147546E716688A
:1035A000013D5660043AEEE72C2C12D1D17C147DFB
:1035B000C1227D259200DBB282189D4204DA9A0076
:1035C0008218FF322D25E4E71668013D5660043A63
:1035D000F3E7452C02D0392C00D0D9E60C006EE779
:1035E000617D7F2998D0525C7F2A00D97EE793E7DE
:1035F000F7BDC046D060030021610300F7B50500A8
:103600000022130044339B005B5D7F2B41D05E4C56
:10361000E35CDB075FD51300511EC9B2443189005A
:103620005A4F6918013BDBB2002B34D102279900B5
:103630006918FF314A7C7F2A00D1A4E053488446B0
:10364000805C44B2002C5BDA41265A1CD2B2900056
:103650002818FF30447C019000967F2C02D06646EB
:10366000365D009666464020365D064236D1123CF5
:10367000012C0CD860460233DBB244339B005B5D07
:10368000C35C4020034202D08B7C013B8B7413004F
:10369000CDE70023CAE708787F2803D0385C0439D7
:1036A0007F28BFD999006918FF31487C7F280ED048
:1036B0002027265C3E4204D0344E305C0426304243
:1036C00005D0887C4608B4460130604488740133D4
:1036D000DBB29342E6D10132D2B292E7009B5B07A4
:1036E00006D4009BDB07D2D58B7CD8081B1ACDE70C
:1036F000019B9B7B591C9B08CB1801998B73C6E7D8
:10370000214CA25C0824224210D00133DAB293008B
:10371000EB18FF33597C7F29B9D06046415C3942B0
:10372000B5D00621997405219973B0E738421DD0B0
:1037300018000130C0B2020044329200525D002AEB
:10374000F7D001337F2A01D1DAB2A0E70F4CA25C97
:103750003A42F9D080002818FF30827C52080132AA
:1037600082748A7C520801328A74EDE7102002428A
:1037700007D060464A7B825C3A4202D08A7C023A99
:103780008A740133E0E7F7BD21610300D0600300D4
:1037900070B50400FFF7D2FB2000FFF771FC230097
:1037A0000022FC330100DA601A61904226D0250025
:1037B000224E11353368FF35934203D0290020484B
:1037C00002F03CFD2000FFF7D9FD2000FFF734FC9C
:1037D0002000FFF7FFFC2000FFF710FF2000FFF79D
:1037E00011FDC4222B009200A1181A78502A07D983
:1037F0007F2A08D00021134A134B1A60080070BDBD
:1038000004338B42F1D13368002B02D00F481EF0F5
:1038100061FD2000FFF7BCFB3368002B03D02900BB
:103820000B4802F00BFD200021F062F9064B09491C
:10383000186828F0D7F941424141DFE7F002002043
:10384000786003008760030010000020AD60030073
:10385000BD6003003E600300002803D0012807D0AC
:10386000002004E08B680448002B00D10348704717
:103870008B685B001843FAE710D6020008D60200F6
:1038800000228168F0B5CB0F094C5B185B100E1954
:103890009A4201DB0748F0BDC568B11A940089005F
:1038A0002C196D5827682560C46801326750EFE70E
:1038B000FFFFFF3FD8F5020070B583680D00416837
:1038C00004008B4212D3C900C06822F05AF8636822
:1038D0000A495A00A3686260D21A013352189B0049
:1038E000E0609200C018002128F020F8A368E26888
:1038F000591C9B00A16002489D5070BDFFFFFF3F17
:10390000D8F50200F8B5070016004C10836803D5FF
:10391000E418E243D2171440A34200D21C000B4922
:103920003800FFF7C9FFBB68094A591E9B189B0066
:10393000181FFA688C4203DBA40016510348F8BD37
:1039400015580139D5500300F2E7C046D8F50200FA
:10395000FFFFFF3F70B50025040085601021C0689F
:1039600022F00FF804232900E0606360102227F0A2
:10397000DDFF014870BDC046D8F5020030B50C002F
:1039800085B0104B02AD043100930138022301953C
:1039900006F0DCFE23680C4C996801290FD9D86821
:1039A0000A4B029AC91889004118A24200D100228C
:1039B0002D79074B002D00D1064B21F0D5F82000C2
:1039C00005B030BD00D30200D8F50200FFFFFF3F75
:1039D00008D6020010D6020070B50C680B00A16872
:1039E0000200002905D11A491A4822F017FB12F0EB
:1039F000DEFE2068012A27D05A6800230FF06EFEF1
:103A0000E168A26886008B19013A1D680436A2603D
:103A1000121A92008919180027F076FF0021A36876
:103A2000E0689A001150616804290BD95B00994243
:103A300008D949088900E06821F0A3FF6368E060C5
:103A40005B086360280070BD01225242D5E7C04682
:103A5000BA62030004FA020007B500900191022047
:103A6000694621F0E7F8694601900220FFF7B4FFAC
:103A700000480EBDD8F5020070B50E000D490500D6
:103A8000002425F097FBB3689C4204D328000A4920
:103A900025F090FB70BD002C03D00849280025F0CC
:103AA00089FBF168A3000122595828000FF06EFC31
:103AB0000134E8E7026303004FC1030083380300C9
:103AC00070B5032604000D000E4029D1174B0A687B
:103AD0009A4225D183688A6899184368994210D917
:103AE00004318900C06821F04CFFAA68A368E06037
:103AF0009B181A1D9B006260C0181022310027F02D
:103B000015FFA368E9689800E3681818AB689A0085
:103B100027F0F1FEAB68A268D318A360044870BD1B
:103B20002900200021F08FF8F8E7C04604D40200F5
:103B3000D8F5020010B50400102021F00CFF044B52
:103B400084600360034B43600023C36010BDC04624
:103B500040DE02004D4B02000B4B70B505000360C8
:103B60000C000800042900D204206860AC608000CA
:103B700021F0F1FE6A68E860121BA40092000019AF
:103B8000002127F0D3FE70BD04D402007FB50C00E5
:103B9000150012283CD005D8052819D007283CD09C
:103BA000002432E00300193B042BF9D893070DD110
:103BB000284B12689A4209D1AB6800938A68EB6877
:103BC000C9680DF0E9FD244C00281ED1234C1CE0EF
:103BD00003231340E4D11F4A2968914238D1A368D6
:103BE000AA68981821F047F80600A368E1689A00CF
:103BF000C06827F080FEA068F36880001818AB68E2
:103C0000E9689A0027F077FE3400200004B070BD08
:103C100011002000FFF754FFF7E703A910000FF091
:103C2000C3FC0028BCD0039B002B01DA00230393C4
:103C3000A3680398584321F01EF80500C3680421C7
:103C40000093A268E068039B23F091FE2C00DCE760
:103C50001C00DAE704D4020010D6020008D60200E5
:103C6000F0B5040087B017000326002A29D10E40C2
:103C70001FD1544B0A689A421BD103AA80680DF0E9
:103C800051FD0499039BA268E0685D1A521A8900ED
:103C9000920041189B00181827F036FEA368AA006E
:103CA000E818E368800052421818310027F03EFE01
:103CB0006BE00491022003A90394FFF78DFE4248B4
:103CC00012E0042A2DD1314221D13E4B0A689A429A
:103CD0001DD103AA80680DF025FD002806D103AA96
:103CE000E168A06823F056FE07B0F0BD039B04987E
:103CF000C01A20F0C0FF05008368E1689A00039BAA
:103D0000C0689B00C91827F0F6FD2800ECE70023E7
:103D10000A002068A1680FF0E1FCE3688000C05849
:103D2000E2E70E4048D1274B0A689A4244D103AAE1
:103D300080680DF0F7FC049B0398BA68C51AAD18AB
:103D40000193002D25DDA368E9186368994207D91E
:103D50008900E06821F015FEA368E0605B196360EC
:103D6000039BA268E068D21A9900EB189B004118E7
:103D70009200C01827F0C8FD039BF9689800E3681B
:103D80001818BB689A0027F0B6FDA3685D19A560F6
:103D900095E7E3688000F9681818920027F0ABFDFA
:103DA0000499B868A268039FE368521A381889001A
:103DB0009200591880006EE73A00200020F09CFF26
:103DC0007DE7C046B81E0300D8F502007822054BF7
:103DD000054890331B681A80743A5A801A715A71D8
:103DE0007047C046C4090020D8F50200084A10B543
:103DF000130090331B689979002908D0116B0029B2
:103E0000F9D0002199711B69587901F0FFF910BDB3
:103E1000C409002013B5084C90342368188821F099
:103E2000B8FE23680090588821F0B3FE69460190DF
:103E3000022001F08BFF16BDC409002010B50D4C07
:103E4000002803D0086803F0B7FB040020000A49EB
:103E500012F008FA6079002101F0D8F9200012F080
:103E6000EBF90022054B064890331B681A619A71E2
:103E700010BDC04630E10200C4220300C409002086
:103E8000D8F502001FB50C4B02AC0093019402233D
:103E900006F05CFC029A002A03D0084B90331B68A2
:103EA0005A806268002A03D0044B90331B681A8042
:103EB000034804B010BDC0469CD50200C4090020D0
:103EC000D8F50200F0B5264B89B004AC00930194FC
:103ED000042306F03BFC234F04223B0090331B6875
:103EE00004981A715A71204B0340062B06D08307A1
:103EF00030D102681D4B92699A422BD10123039461
:103F00000293002590373B68186912F095F93B68D9
:103F100060681D6103F050FB1549060012F0A2F91C
:103F2000144A3B6812689D719A60227B0299DA718B
:103F30009981DD81039A012900D112685A61012219
:103F40001E619A71237A002B01D0FFF74FFF0A48B8
:103F500009B0F0BD03AA02A90FF08AFBD1E7C04661
:103F60003CD50200C4090020070080FF3D990000F5
:103F7000C4220300C8080020D8F50200F0B5294B80
:103F800089B004AD01950093042306F0DFFB6B6854
:103F9000A868049E039303F00FFB234F040090379F
:103FA0003B68186912F048F900223B681F4920005D
:103FB0001A6112F057F9607980212D7B01F026F902
:103FC000002E1DD1607901F0A9F9039B002B14DBB1
:103FD0000022154B164990331B68096803989A71A3
:103FE0000918DA719A81DA815A61023299601C618A
:103FF0009A71002D01D0FFF7F9FE0E4809B0F0BD0F
:1040000031000D4816F0E8FA01F0CCF80028DCD0B9
:10401000607901F083F90949094821F0FFFF12F0A6
:10402000C6FBC0466CD50200C4090020C4220300B0
:10403000C8080020D8F5020040420F00CE620300FD
:10404000ACFD020010B5182021F085FC074B903321
:10405000186078230380743B43800371437100230D
:10406000837103614361024810BDC046C40900204A
:10407000D8F50200F0B56D4C87B026009036336855
:10408000002B40D09A79002A3DD0694D9A68296862
:104090008A4238D89A79022A0BD11B6900215879B3
:1040A00001F0B4F82B6832680A33936001239371EE
:1040B00029E09A79012A26D19A89D989914204DB8B
:1040C000DD79002D19D00021D9815869012A02D04B
:1040D000DA8992008058574A904216D11B69002114
:1040E0005879903401F092F824685348218816F0EA
:1040F000FDFA0123A060A37105E09D71186912F01B
:104100009BF833681D6107B0F0BD05A905F03AF9C9
:104110009034236801901B69802158790293059E91
:1041200001F074F8019B24681F781F2321884248FE
:104130001F4016F0DBFA618816F0D8FA7D1EEDB24A
:104140000390012E5AD9019B5B78232B4DD0622B13
:1041500050D1002D4BD0023FFDB26A1E5142514159
:104160004A42022E4ED0012102230198C05C3A2817
:1041700003D00F27384020710133207984469E42B6
:104180000ED90198C05C3A280AD1581C864207D93A
:10419000019F0233385C0F2738409E4235D860714A
:1041A000092D3DDC6346043B9A1852B26F00234B45
:1041B000002900D1224BD85B002A2EDB104100F0F1
:1041C000F1FF1A4B039990331A68537959430B0046
:1041D0000A3B0A2B00DA0A2315490968CB189360B9
:1041E000D3890133D381022361E70022B9E72A0092
:1041F0000625B6E7002101230A00B6E700210123C6
:104200000A00BAE733000121B7E70A267043019E8E
:104210006071F65C3E408019C1E752429040CEE7A3
:10422000029B0021587900F0F1FFCAE7C409002081
:10423000C8080020D8F5020060EA0000E833030057
:10424000DA33030010B50B790349002B00D1034981
:1042500024F0B0FF10BDC04659860300518603000C
:1042600037B50C00110000221D0000920123200030
:1042700006F03AFA054B002C06D028680FF094FAA5
:10428000034B002800D1014B18003EBD08D60200A8
:1042900010D60200F0B5214B8DB005AC013800936B
:1042A00004310194072306F051FAA0681C4D002642
:1042B000A84202D00FF03AF9C6B260691827A842A6
:1042C00002D021F02BF80700A0691922A84202D0E1
:1042D00021F024F802002069A8420DD003AA02218F
:1042E0000FF0E8F9039B186821F018F8039B07000A
:1042F000586821F013F80200390003A812F020FEDC
:10430000059903A812F078FE03A8E36832006168FB
:1043100012F082FE28000DB0F0BDC046F8D60200B3
:10432000D8F5020010B503F025FA034B002800D1A0
:10433000024B180010BDC04610D6020008D602007D
:10434000002803D0012807D0002004E08B6804482F
:10435000002B00D1034870478B685B001843FAE7D5
:1043600010D6020008D602007FB504000122080022
:1043700001A90FF095FA00222179402010F0DAFD12
:1043800001000500029816F027F9636806001A0A72
:10439000904217D9A368C1186943E06821F0F1FA87
:1043A0002379E0602A00A06863606843E368724391
:1043B0001818019927F09FFAA36805489E19A6606E
:1043C00004B070BD121A1202DBB21343EAE7C04612
:1043D000D8F50200F7B5FF27456804000191BD43F9
:1043E0001DD101792A00402010F0A4FD6368060069
:1043F0003B408027A1683F011F430831414367606C
:10440000E06821F0BEFA6368E0601A0AA368013A26
:10441000013372435E432900801927F087FA20791F
:10442000019BA268E16810F0D9FEA368034801333C
:10443000A3606368013BFF3B6360FEBDD8F50200EB
:1044400010B50400102021F098FA024B446003607C
:1044500010BDC0467CD7020070B50A7904000D007B
:10446000002A0DD1194924F0A5FE0123AA68E968A4
:10447000200004F03FFA1649200024F09BFE70BD96
:10448000144924F062FFAB68002BF4D012492000DD
:1044900024F090FE0026AB689E4204D30F49200012
:1044A00024F088FEE7E7002E03D00D49200024F019
:1044B00081FE3200E968287910F05EFD01220100DA
:1044C00020000EF063FF0136E5E7C046E962030015
:1044D0002FA70300F5620300006303004FC1030030
:1044E00083380300F8B5002207000D0001004020CA
:1044F00010F020FD061E05D10C490D4821F08EFD5F
:1045000012F055F9102021F026FA0A4B0400002F72
:1045100000D0094B28002360FBB2A56070436360A4
:1045200021F019FAE0602000F8BDC046DC6203000B
:10453000ACFD020014D80200D8D7020070B5060006
:104540008AB00C00150012285CD003D8052826D0AC
:10455000002454E01B2800D16CE01F28F8D1012270
:1045600007A9280024F02EFB032300284FD01C426B
:1045700013D13B4B22689A420FD1012204A920009B
:1045800020F009FC0123079A00930599089B0498E1
:1045900021F07DF8334C002831D1334C2FE001223B
:1045A00004A9200020F0F7FB2800012207A90FF042
:1045B00077F9069B002203936B464020197B10F08D
:1045C000B9FC01000600089816F006F8069BA168E1
:1045D00003936B4641180500187BFFF783FF059B8B
:1045E00004001A000499C068039327F084F92A0094
:1045F0000598E36872431818079927F07CF92000A2
:104600000AB070BD11002000FFF7AEFEF7E7EA0721
:104610000DD41D4203D1154B2A689A4207D00323BB
:104620002B40022BB9D1124B1D40062DB5D011489D
:104630000BF012FD012204A9200020F0ACFB0122A6
:1046400007A9280024F0BEFA0028A6D0089B059AE6
:1046500000930499079B300023F0BDF99AE7C04608
:1046600014D8020010D6020008D60200440103004C
:10467000070080FFC6650300F0B5050087B00E0097
:10468000002808D08B0726D10B68254A934202D018
:10469000244A93421FD1012203A9300024F092FA48
:1046A000002818D000222900402010F043FC01000F
:1046B0000700049815F090FF060001002800FFF79E
:1046C00011FF320004007A430399C06827F013F900
:1046D000200007B0F0BD30000FF042F8071E00D0F8
:1046E000471039002800FFF7FDFE040030000AF0F3
:1046F00007FF0026009000980AF04EFF031EE7D047
:10470000002F04D119002000FFF764FEF3E7721CAC
:104710000192E1683200280010F060FD019EEAE796
:1047200040EE020014D8020070B5050086B0161ED7
:1047300044D003240C402DD1214B0A689A4229D140
:1047400003AA80680CF0EEFF002802D11D480BF090
:1047500083FC2000042E1BD122002979402010F078
:10476000E9FB049B06000093039B28790193019ABF
:10477000009B991AFFF7B6FE04000399049AC068DB
:10478000521A71437243EE68711827F0B4F8200092
:1047900006B070BD0A000023A96828680EF09EFFCD
:1047A00002002879042E03D1E96810F0E5FBEFE759
:1047B0003300E96810F012FD0348E9E71000E7E76D
:1047C000B81E030004630300D8F5020037B50C00DF
:1047D000110000221D0000920123200005F084FF3B
:1047E000002C04D121002000FFF77CFE3EBD29688B
:1047F000CB0705D48B0713D10B4B0A689A420FD114
:1048000008000EF093FE010005000020FFF76AFE8D
:1048100004002A000021C06827F088F82000E5E79E
:104820000020FFF729FFE1E744010300F0B54568E8
:1048300087B00393AB6805A81700029105931EF09B
:10484000F6FD060005A81EF0F2FD03000320584304
:1048500033000933C018800021F07DF804000A4BB2
:10486000AA6803606B6829004360059B06629B1A77
:10487000C360039B08300093029A3B00FCF7EEF9FB
:10488000200007B0F0BDC0469CD8020070B50500FE
:1048900088680C001EF0C2FD2300020002492800B7
:1048A00024F053FD70BDC0463563030010B50248C7
:1048B00021F0A7FB11F07BFF74FC020010B504008F
:1048C000082021F048F8024B4460036010BDC04648
:1048D000D8D80200F8B50400C0681D00002801D136
:1048E0001860F8BD200063692030834208D1154B61
:1048F000994206D01449154821F090FB11F057FF5A
:1049000019602000124E63681100083077687360E8
:1049100009F052FD7760012807D00023E3600228E8
:104920000AD063691B682B60DBE763691B682B6037
:10493000002BD6D1E360D4E7236A07339B00E41849
:104940006368F0E7D8F502007363030034FD0200EA
:10495000C409002013B501AB1400FFF7BBFF012809
:104960000ED0184C02281CD0019BA34228D0002B4B
:1049700026D001AA0121144821F03DFB11F017FFB8
:10498000002C0CD020000EF0E9FC104903F034FBA1
:10499000002804D00E490F4821F040FBEEE70198B3
:1049A00016BD01980EF0DAFC074903F025FB00283C
:1049B00001D10198E2E7019807F062FCA042F8D12A
:1049C0000020EDE7D8F5020074FC020050F9020067
:1049D000536303002CFC020010B50C0002280BD11D
:1049E00048680BF051FA064902002068FFF7B2FF51
:1049F000002803D1FFF75AFF8868F2E710BDC046D0
:104A0000D8F5020010B500220149FFF7A3FF10BD41
:104A1000D8F5020013B5124C01AB124A2100FFF782
:104A200059FF012803D0022807D0200016BD0E49E7
:104A30000E4821F0F3FA11F0BAFE01980EF08EFC48
:104A40000B4903F0D9FA0028EFD101980EF086FC4B
:104A5000084903F0D1FA0028E7D10198EBE7C046F6
:104A6000D8F50200A4F70200536303002CFC0200F7
:104A700050F9020074FC020073B50090000C431E54
:104A800001910A2B1AD80126330083400C4A118861
:104A90000B439BB213800B4B1A780F2A0EDC1A784B
:104AA00019783240F14092009040074C655C2843F1
:104AB000C0B260541A789219D2B21A7073BDC0464F
:104AC000100900202809002020090020094A70B59B
:104AD0001378002B0CD1084D2C78E4B2002C07D1B0
:104AE0000068013313702B7003685B6898472C7063
:104AF00070BDC0461E0900201F09002010B504002B
:104B00000430FFF7E3FF606826F036F9034B8000BE
:104B1000C3580620DB00184310BDC04614D902005C
:104B200010B503F0A3FF0023074A99008958884273
:104B300008D001330C2BF8D10449054821F06EFA56
:104B400011F035FED8B210BD14D90200A9630300DC
:104B5000ACFD020070B504000800FFF7E1FF05009E
:104B6000201DFFF7B3FF606826F006F9024B85426F
:104B700000D0024B180070BD10D6020008D602000B
:104B800070B504000800FFF7CBFF0500201DFFF7FC
:104B90009DFF0123AB40064A064811880B4200D115
:104BA00005481188994311800022044B1A7070BD8A
:104BB0001009002010D6020008D6020028090020A3
:104BC000F8B50430FFF782FF124C13482378002B0E
:104BD0001FD020780021C0B201F0B8F801260022D1
:104BE0000E4F2378934212D915005308FB5C3540D1
:104BF000AD002B410F252B40094D9B005B5906252D
:104C00009100DB0041182B438B600132E9E7002360
:104C10002370F8BD2809002094DC02002009002040
:104C200014D90200C02307B5002200931B21024BB8
:104C3000024813F065FD07BD794A0000CC0500204D
:104C4000F0B505008BB008680C0004F085FB0490FB
:104C500004A820F044F900270126049B0390069342
:104C6000069B197800291ED1380001F06FF8012247
:104C7000009007A960680EF013FE079B089A059341
:104C80009B1801920293022D22D9A0680EF04EFCCF
:104C900000281ADA089BC01817D52D492D4821F095
:104CA000BDF911F084FD080010F004F9002806D0C9
:104CB00006A820F026F9069B1B78732B00D1300044
:104CC000069B3F1801330693CAE7059B1818059009
:104CD0000024BC4202D300980BB0F0BD049B1878AE
:104CE0000028F8D010F0E6F80125002803D004A829
:104CF00020F007F905000598029A43199A42CCD38F
:104D0000049B1B78732B09D0009BA6009E1901956C
:104D1000019B0436002B10D164190AE0290003F02E
:104D20009BFE059B009A5D19A31C9B000595013411
:104D30009850049B01330493CBE7049B05AA197890
:104D4000039810F07BF9019B7060013B0193DFE752
:104D5000B9630300ACFD0200F0B589B00391019284
:104D60001E0004F0F9FA049004A820F0B8F800241A
:104D70000290B44201D309B0F0BD049B187800281A
:104D8000F9D010F097F80125002803D004A820F0EE
:104D9000B8F80500039B019A5B199A4205D21D4998
:104DA0001D4821F03BF911F002FD049B1B78732B89
:104DB00010D064190E9BA700DF19002D25D0049B8D
:104DC000AA0052421978BA5803AB029810F096F92B
:104DD000013DF2E70E9B671CA400E058012205A9E3
:104DE0000EF05EFD069CAC4200D92C002200059915
:104DF000039826F080FD039B2A1B18193C00002114
:104E000026F094FD039B5D190395049B01330493E5
:104E1000AFE7C046B9630300ACFD0200F0B50E0079
:104E200089B0039001CE0F0020F081F844102100DA
:104E300004A822F0DAFB069D22000021280026F0BB
:104E400075FD039B0096013B2A1929003868FFF77E
:104E500083FF04A9024803F0B1FD09B0F0BDC046CC
:104E600040EE020030B50C0089B0050002226068F7
:104E700005A90EF015FDA0680EF058FB002809DA10
:104E8000069B0393C01805D509490A4821F0C6F8C6
:104E900011F08DFC0599069AEB1E8A18091820005E
:104EA0000C3000902068FFF757FF034809B030BD71
:104EB000B9630300ACFD0200D8F50200F7B50D00A0
:104EC0000EF034FB684C207028000EF02FFB674B6F
:104ED000C0B218702378012B14D0022B1CD0102BD9
:104EE0001CD00F2B1CD0052B1CD00E2B1CD00D2B37
:104EF0001CD05F490B2B06D05E495F4821F08EF82D
:104F000011F055FC5D49012812D0022855D05C4CA7
:104F100010280ED05B49F0E75B49F4E75849F2E707
:104F20005A49F0E75A49EEE75A49ECE75A49EAE7A5
:104F3000524CA02604224B79F605C133FF339B0067
:104F40009A516079013A0300C133FF339B009A51B3
:104F5000023A130083401800A123DB00F0500A201E
:104F60000138C046C046C046C046C046C046C046DE
:104F7000C046C046C046C046C046F1D11000637965
:104F800000249840454BF050A920454BC0001B68B9
:104F90009A641D584348056010004979019688407D
:104FA000414900900868A227019EFF00F759009E22
:104FB0003E4204D0002C0ED00CE0334CB9E7012067
:104FC0009864A920C0001858384F441BA446140008
:104FD000BC45E8D9086001229A64A9220026D200C3
:104FE0009858334C334A10602268A027A225FF0549
:104FF000ED007F59009D3D4202D1002E0CD00AE009
:1050000001229A64A922D2009A58284F161AB4464F
:105010000126BC45E9D9226001229A64A922D20066
:105020009B58254D181A0B60244B421E2860244CB7
:105030009A420DD923481DF04DF9296822481DF0E8
:1050400099F800232360012023685B001843FEBD0C
:1050500016F09EFC1D4916F057F91D4915F064FF26
:1050600016F026FC2060EEE7290900202A0900201E
:1050700040E10200CA63030034FD020078E102004F
:1050800068E102000964030088E1020060E10200B7
:10509000A0E1020058E1020050E102000C0500000E
:1050A00018000020B8030020B8090020C8AF000095
:1050B000BC090020B4090020C0090020C6AF0000D0
:1050C000F402002028640300316403000000084259
:1050D0000000FA44F7B5244900250B000833DA6FC5
:1050E000224B94461B785488981C80001618805ACE
:1050F000883144430968A4120195F078002823D030
:10510000B07801268640A1273000A026FF00F605D2
:105110000133F051DBB2981C80001618805A07004A
:10512000508878438012001BE7D0104A1370019B0F
:10513000002B02D00C4B88331960002D03D062463F
:10514000094B0833DA67FEBDA024094B5668E40515
:10515000E650002902D10B000C00DCE701258C464B
:105160000A0001950100F6E7C40900202B09002080
:105170000C050000044B05491A000832D1670022D3
:1051800088331A607047C046C4090020ECDA020078
:1051900010B5782202490220FCF7CEFA10BDC046B5
:1051A000D5500000421E104BFF3A70B59A4218D8F5
:1051B000061172B60D4C00212300220088331D68B1
:1051C0000832196062B68D4200D1D56F2978280067
:1051D0001FF042FF6B6888344360468020600020E7
:1051E00070BD01204042FBE740410F00C409002090
:1051F000054B1A0088331B680832002B00D1D36F8F
:10520000588800017047C046C4090020F7B5414ADC
:1052100007000B00914200D913008022D200D21A5D
:10522000019272B63C4A002011008832146808319D
:10523000106062B6844200D1CC6F0126BE40626825
:10524000324207D13A00A0210320C132FF3292003E
:10525000C9055050002521788D421CDB002B19D048
:10526000013120001FF0F8FE6A46636892881E43F1
:10527000466023789B00C3181A8101229F72DA725C
:1052800001216388021D4380037899421CDB224B75
:1052900088331860F7BDAA00A218927A97422CD0E2
:1052A0000135D9E7013920001FF0D6FE6368B3430A
:1052B000436023785A1EAA42E2DD01339B00023587
:1052C0001B59AD002B50DBE71700D37A1489967A6F
:1052D00001934B1EBD88A54204D97D68043FFD6043
:1052E000013BF7D203339B00C3181C806C46247922
:1052F0009E70DC7001310432C6E7002BD2D0200052
:105300001FF0AAFE6368023543606B469B88AD00C0
:105310002B52B5E7FF030000C409002010B500219F
:105320000400FFF773FF0D4B0833DA6F002310788A
:10533000834200DB10BD99005118897A8C4201D05C
:105340000133F5E702339B00D3181F229A70012323
:10535000A021A340024AC9058B50EBE7C4090020F5
:105360000C05000073B516000D4A0B005468156853
:10537000012804D94C682500022800D08D6801A9B5
:10538000186803F0FFFF01009320019A00234000FA
:1053900006F084FA2B00310022000AF013FE76BDDD
:1053A000C409002010B504000C2020F0D4FA034BEF
:1053B0004460036001235B42836010BD10DB020088
:1053C00010B54A68014923F0C0FF10BD7D9F03005E
:1053D00001220020074B08495A600860A821DA60C2
:1053E000064AC9005A5006495A5004315A500549D4
:1053F0005A507047009000400C9C0040FCFF000099
:10540000440500004C050000034B04481B78002BAA
:1054100000D103487047C0462D09002010D6020075
:1054200008D60200F8B5A826324A334BF6001968B0
:1054300013680420CB18C9181160304A8C461278C2
:105440001B11170009112E4A2E4C2F4D002F47D04B
:10545000002B39DA9051C31AA920C00013508123C0
:105460009B00002936DA591A135151510123274C58
:10547000D3602378002B21D03F222548254B01689B
:105480009B6F01310A409D5C1C4B1B78002B01D0A7
:10549000803D6D001C23026062466B4308339B1AFB
:1054A000154A9B1013601F23194007D11A4B1A7815
:1054B000002A03D019481970FCF7A4F901232278B7
:1054C000042053402370F8BDA9270433FF00D051B6
:1054D0009351C4E7535181239B00C9181151C5E76B
:1054E000043390515351A9208123C0009B001350D5
:1054F000F3E7C046F802002008030020480200201D
:10550000009000404C050000440500002C090020DC
:10551000FC020020C409002049020020235102009F
:1055200030B585B001220400080001A90EF0B8F9D9
:10553000029A202A00D920220023019D934204D000
:10554000E85CE11808710133F8E7014805B030BDA7
:10555000D8F5020070B50400080015000DF0E6FF54
:105560000E491F2815D8002D05D10D490D4820F0F2
:1055700055FD11F01CF92418042D04D101202379C4
:105580005B00184370BD28000DF0D0FFFF2802D942
:1055900005490648EBE720710548F3E781640300FD
:1055A0009564030034FD0200BA640300ACFD020000
:1055B000D8F502000123A022834010B5134CD20578
:1055C00013510300C133124CFF339B009C50114B0D
:1055D0008900C918A223DB00CA580F4C00022240E0
:1055E000CA50F82252011040C022CC5892022243E5
:1055F00010430322C850CC58084822432043C850C7
:10560000C046C046C046CA5010BDC0460C0500008A
:105610000303000000600040FFE0ECFF031F0000F8
:10562000A0221E21114BD20070B59C58104D8C4306
:105630009C50A324E4001D510E4C0F4D0F4E5C51A5
:1056400004355E510E4D80005C51A5240D4DE400E3
:105650001D51084C0C4D00190C4C185104341D51AF
:105660000B4C185198580143995070BD00F00140FF
:1056700040910040006000401C0500004491004043
:1056800024050000489100404C9100402C0500008A
:105690003405000070B50D00040010F0BFFD134E7E
:1056A0002800310010F0DEFD3100200010F0DAFD9E
:1056B0000F4BA0221C600F4BD2051D6060790124A6
:1056C0002100814026000C4BD15069798E40002189
:1056D000D650FFF76FFF68792100FFF76BFF2000BE
:1056E000FFF79EFF054B1C7070BDC046CC22030027
:1056F00000030020040300200C05000048020020E5
:1057000010B504000A4910F0ADFD0A4BA0211C6041
:1057100001236079084A8340C9058B500021FFF7B7
:1057200049FF0020FFF77CFF0022044B1A7010BDD8
:10573000CC220300000300200C05000048020020DA
:10574000F8B50025FFF744FE214B2800DD67FCF784
:1057500027F8A0221E201F4B1F491D701F4BD2008F
:105760001D601F4B1F4C1D608B581F4F83438B5078
:10577000A223DB00E2581D4E3A40E250E2581C4999
:105780003243E2500122E5501A4B186843799A409F
:105790001300A022D205535010F04EFD164B1B787B
:1057A000AB4213D0154B1249E2581740E750E2586C
:1057B00016430122E650E550114B186843799A4090
:1057C0001300A022D205535010F036FDF8BDC0469C
:1057D000C40900202D09002000F00140F80200203B
:1057E0000803002000600040FFE0ECFF001F030002
:1057F0000C050000000300204802002014050000F2
:1058000004030020F0B53A4E8DB0F36F0500002B75
:1058100003D1FFF795FF0DB0F0BD002801D00EF0C9
:1058200015FF684610F0A8FF00281DD1F06F09F0A1
:105830008DFE040010F0B6FF002D01D00EF010FF19
:1058400020222C4B1D68B36F6D1101356D01154081
:105850005D19002C2CD121002800F46726F066F891
:105860000122254B1A70D6E7002D01D00EF0F8FE6C
:10587000019B2249186802F0BFFB00240500A042EA
:10588000DED1019F38000DF069FD1D4B98420BD110
:105890002900012000F05AFA2A000400F8601F21B4
:1058A000184803F0C1F8A060019B00243363C7E7E8
:1058B00020000DF053FD144B984207D000231349EC
:1058C0001348F36720F0AAFB3063A4E763682B60FA
:1058D000A3686B60E368AB602369EB6063692B616D
:1058E000A3696B61E369AB61236AEB61B8E7C0460A
:1058F000C4090020FC0200204902002074FC0200C0
:1059000000FB02004F64030058DC02006F640300D8
:1059100034FD020010B5FFF713FF014810BDC0466B
:10592000D8F50200F0B589B00493704B03901B7852
:105930000E001500002B01D0FFF702FF6C4B1A7808
:10594000002A07D16B4C4020E26701321A7020F028
:1059500002F8A06780270122674BBF00674CDF6712
:10596000674BE250FFF734FD0023664AF021A35055
:105970000432A3500832A350C22209039200A1505E
:10598000E351614F0594BE4200D09FE0B54200D084
:1059900096E05E4D07AC280010F058FC002805D0BA
:1059A00001235B492800237010F05CFC594D28004E
:1059B00010F04CFC002805D00123554928006370E5
:1059C00010F050FC544D280010F040FC002805D089
:1059D00001234F492800A37010F044FCA0270024A5
:1059E000FF0507ABE35C002B33D10134022CF8D167
:1059F000464801F0E1FDFFF783FE002601240398ED
:105A000009F07EFD3F22454B3A4D1E70444B8021EC
:105A10001C70444BE8671A60A86F121925F086FFC6
:105A20003000FFF7EFFE404B304F1C60059B5022CB
:105A30001C603E4930003C70FBF77EFE049BB34285
:105A400052D03B78002B4FD02B6B002B4CD120BF7A
:105A5000F7E7374BA200D65803227379651CC13390
:105A6000FF339B00DA5107ABEB5C002B24D0304BAB
:105A7000AA00D358019304230093012273799A401A
:105A8000A123DB00FA50019B0533180002931FF09D
:105A900028FB012810D173799840264BF8500298C2
:105AA0001FF01FFB002807D1009B013B0093002B38
:105AB000E3D10199300014E00135032DD3D194E7EF
:105AC0001D491E4820F0AAFA10F071FE300001F0C6
:105AD00073FD0400BD428ED0280001F06DFD010071
:105AE0002000FFF7D7FD88E709B0F0BD2D090020A1
:105AF0002E090020C409002004E100E000900040CD
:105B0000FC0F000004050000D8F5020030E102009F
:105B10009C22030078E1020088E102002C090020A9
:105B200049020020FC0200200C9C0040255400008B
:105B300010DC02000C050000CD64030034FD0200FF
:105B400010B5084B86B002AC00930194042304F016
:105B5000FDFD02982379E268A168FFF7E3FE0248A1
:105B600006B010BD1CDC0200D8F50200014B18780D
:105B7000C0B270472D09002010B524201FF0EBFEA5
:105B80000400044B202208C0802125F0CFFE200015
:105B900010BDC04658DC0200F8B5050008000E0034
:105BA00017000DF0DBFB324B984201D00020F8BD0E
:105BB000681F0F28FAD814F0E7FC080835F9F9F93E
:105BC000F9F9F9F9F9F9F9333358FFF7D5FF042357
:105BD0000400F25CE2540133242BFAD138000DF0BA
:105BE000BDFB234B9842E1D10121052D05D0123D8B
:105BF000691E8D4101216D4229430422FF20BB5CB7
:105C0000A55C803B4B435B19FF2B03D90500DB17D9
:105C10009D432B00A3540132242AF0D12000C6E773
:105C20003400DBE7FFF7A8FF04230400F25CE25432
:105C30000133242BFAD138000DF0DCFC0F211FF0CA
:105C400075FA2100FF25221D24311378803B434340
:105C5000DB138033FF2B03D92E00DB179E43330069
:105C6000137001329142F0D1D8E73400E3E7C04627
:105C700058DC020070B50E0010490400002523F026
:105C800099FA73689D420AD3012B03D10C49200075
:105C900023F090FA0B49200023F08CFA70BD002D00
:105CA00003D00949200023F085FAAB00F318012244
:105CB000996820000DF06AFB0135E2E7F6A70300C2
:105CC000EF6403002FA703008338030070B50D00B5
:105CD00001281ED0002803D0022807D0002004E0AD
:105CE0004B680E48002B00D10D4870BD00260D4CAE
:105CF0006B689E4203D3012064002043F5E7B300A4
:105D0000EB189968022009F099FA4010241801361E
:105D1000EEE74B685B001843E7E7C04610D6020089
:105D200008D6020094DC020010B5040010201FF019
:105D300012FE044B84600360034B43600023C36086
:105D400010BDC04640DE02007B51020070B5060067
:105D50000D000C48002E0FD0B41CA40020001FF032
:105D6000FAFD094A030002604660002D04D00022BB
:105D7000083C944201D1180070BDA8589918886059
:105D80000432F6E794DC02009CDC0200F0B504006B
:105D900085B00D00160007284CD003D8052824D064
:105DA000002144E00300193B042BF9D808000DF052
:105DB000D5FA30000DF0D2FA2C4B426A9A4205D047
:105DC00030002B491FF01AFC061E0CD033002900AE
:105DD00072680831009208336A6820000BF0DCFC1E
:105DE0002449002823D1244921E010000DF0B6FAFF
:105DF0001F4902F001F9011E19D06B687268002179
:105E00009818FFF7A3FF070029006B6808379A006E
:105E100008310400380025F06EFD310068687368B1
:105E2000800038189A00083125F065FD210008002F
:105E300005B0F0BD03A910000DF0B6FB00218842AB
:105E4000F5D0039888420FDD6B685843FFF77EFF5B
:105E5000040023002800083300930830039B6A687D
:105E6000042121F084FDE1E70449E0E7295D000019
:105E70009CDC020010D6020008D6020094DC02006E
:105E800030B5040085B0042A2DD103250D4020D162
:105E9000164B0A689A421CD101AA40680BF042FCDA
:105EA000002802D112480AF0D7F8019B0298290075
:105EB000C01AFFF74BFF050021006B6808319A00FC
:105EC000019B08309C00091925F015FD280005B03C
:105ED00030BD0A000023616820680DF0FFFB02302E
:105EE00080000059F3E70020F1E7C046B81E030028
:105EF00004630300F0B50C001100002285B01E0001
:105F000000920123200004F0EFFB184D002C1DD05F
:105F10003568AB0703D1164B2A689A4216D0102079
:105F20001FF019FD0400306809F0EAFA0025042684
:105F30000390039809F030FB071E0AD128002100C6
:105F4000FFF704FF050020001FF02CFD280005B01E
:105F5000F0BDAE4205D8F10020001FF012FD040094
:105F60007600AB001F510135E3E7C04694DC020028
:105F70009CDC0200F0B593B0060006A80F001400E8
:105F800010F0FAFB051E2BD13368310001263A00D0
:105F900003A80193FCF7BAFDA3082A003340019936
:105FA00003A80DF03BF80500032001F0D3FB280007
:105FB00021F042FA0120404201F0CCFB10F0F2FB4C
:105FC000344203D03100134801F0F8FB01250121D0
:105FD0000C4202D00F4801F0F1FB280013B0F0BDD5
:105FE0000120404201F0B6FB01210C4202D00948D9
:105FF00001F0E4FB07980DF0B1F9074901F0FCFF4F
:10600000051E04D1079905480DF0E4F9DFE7802566
:106010006D00DCE7C5650300F8FC02008C2203007C
:106020001FB520216846802421F0C8FA6400254865
:106030001FF092F9684621F0F7FA23481FF08CF917
:1060400001F0A4FB0128F2D002280BD11F481FF059
:1060500083F9684621F0DDFA012200201C4B1A70FA
:1060600004B010BD032803D1684621F0DDFAE7E74C
:10607000042804D0C1B2684621F02BFBE0E71548A4
:106080001FF06AF9019A002A08D110481FF064F93C
:10609000684621F0BEFA80204000E1E72820002376
:1060A0000299FF3005F0FAFB002803D10A481CF0E2
:1060B00061F8BFE701221100FFF75CFF2042B9D071
:1060C000CEE7C0469D650300107C0300B266030066
:1060D0004A0200203E600300B865030070B586B038
:1060E000202102A8802421F069FA640044481FF0AE
:1060F00033F944481FF030F902A821F095FA4249DB
:1061000002A81DF049FC01280AD140481FF024F9DB
:1061100002A821F07EFA00203D4B187006B070BD39
:10612000022803D139481FF017F9DFE7032801D10E
:106130003648DFE7042808D134481FF00DF902A8DB
:1061400021F067FA80204000E8E7052836D1314881
:106150001FF002F902A821F067FA01F017FB6B4665
:10616000C1B2DD1D29700329E2D0042917D12748C7
:106170001FF0F2F8012502A821F061FA060002A83A
:1061800021F064FA0200282000233100FF3005F0DE
:1061900085FB00282CD120481CF09CF8ACE702A815
:1061A00021F097FA2B780D2B03D11C481FF0D4F85F
:1061B000D3E70121280001F001FBCEE702A821F07E
:1061C00045FA002898D002A821F072FA0FF06CFB73
:1061D00000280BD00A2102A821F07BFA104902A85E
:1061E0001DF0DAFB0328A3D00428ECD10025C2E778
:1061F00006222900FFF7BEFE204200D17CE78DE792
:10620000F1640300366503005C650300B2660300B9
:106210004A02002061650300868503009165030042
:106220009865030010B5034809680DF0D3F80248DB
:1062300010BDC0468C220300D8F5020073B50600DD
:10624000194D0C0028001CF045F8310017481BF0D0
:1062500091FF17481CF03EF816481CF03BF8FF234E
:106260009B00E61821787F2901D0B44206D128008E
:106270001CF030F810481CF02DF873BDA37850299D
:106280000CD80E4A505C0E4A525C0193637800931E
:1062900003000C481BF06EFF0434E3E762780A4801
:1062A0001BF068FFF8E7C04680660300AD66030098
:1062B000B56603003E6603005C660300606203008F
:1062C0000F620300D6660300F9660300F0B51D00F7
:1062D0008BB007901B48160008911BF0FBFF2900AC
:1062E00019481BF047FF19481BF0F4FF18481BF032
:1062F000F1FF0024AC4204DB12481BF0EBFF0BB0B3
:10630000F0BD089B375DA0000799181803788278C4
:10631000095D049707689B063F037F0E0397C778C4
:106320009B0E09933B09029300883F07C004400E6F
:106330003F0F019012090097099B06481BF01AFFB6
:106340000134D7E780660300CD650300FA650300DA
:106350002C6603005E66030010B588B001AA69468A
:10636000040006F055F8009B022B2AD902AA32211C
:1063700004A80AF08DFA019B13495A6802A822F07A
:10638000E4FF20000CF0EAFF104BC2689A4210D1E3
:1063900023680F495A6802A822F0D7FFE368002B50
:1063A00007D05A68002A04D00022996802A80CF08D
:1063B000EDFF04A821F07CF901F04EFA04A821F0C9
:1063C00028F908B010BDC04647670300A9C1000006
:1063D0005067030070B5050090B0002804D11F4835
:1063E0001BF078FF10B070BD04A810F0C5F9041EB2
:1063F00019D12E68290001A80122FCF787FB230090
:106400002200310001A80CF009FE0400032001F075
:10641000A1F9200021F010F80120404201F09AF982
:1064200010F0C0F9DEE70120404201F093F9059930
:106430000B480CF0CFFF05980CF090FF09490400C1
:1064400001F0DAFD0028CDD10749200001F0D4FD8C
:106450000028C7D10598FFF77FFFC3E71A6703003D
:106460008C220300F8FC02007CFA020037B52A4BAC
:1064700001AA1A60FBF772FCE120C000FBF778FC70
:10648000264927480EF0B6F808F02CFE01F040F936
:10649000FBF722FD07F02AFA0023224C224D636706
:1064A0002B78012B0BD1F8239B021A784D2A1BD194
:1064B0005A78502A18D159881C481EF0B1FE2B7802
:1064C000002B25D1FFF7ACFD0028F8D018481EF0AE
:1064D00043FF08220021174825F028FA00239034B2
:1064E000236020F0A5FF37BD002307211A001248C2
:1064F00003F068FF002802D01EF09CFEDFE7482072
:1065000001220E49FF3009F0DDFC20F0C8FFD6E77C
:10651000FFF7E4FDD8E7C0460C0300200038002058
:1065200030130020C40900204A02002004E00300C8
:106530005C670300300A00205467030094DC02000B
:1065400007B50EF0E9F8054B01A81968091A890882
:106550000EF09AF80EF0F4F807BDC0460C030020C8
:10656000F0B58BB0079310AB10CB009001911B7866
:10657000062A12D8012A08D93F230B700B000133D9
:106580000193002301990B7001E0002AF9D1012049
:106590009042804140420BB0F0BD009900292ADAB8
:1065A000019B01995F1C2D230B70802109068C46ED
:1065B000009B63440093019BFF210993009BC90545
:1065C00018000840884224D12021079BF81C0B406A
:1065D0001900009B5C024E23002C13D14B40492232
:1065E0007B7046234A4059403A70B97000230370CB
:1065F000019BC01ACFE7019F002BDCD03900013787
:106600000B70D8E741240B4361403B707970BB703D
:10661000ECE7002C00DA06240199013A7D1A551B9B
:106620002022079911430291672942D1002C00D101
:10663000D5E1002B7BD0A84A934200D9D5E0A749E9
:10664000009814F0ADF9431E984100230026303025
:106650000393203305900493A14B039A0099D058DB
:1066600014F094F9002808D0049B039AF6189D4B67
:106670000098D15814F048FE0090049B5B100493DE
:10668000039B04330393182BE6D115330493009A2C
:10669000914B934260D39149009814F081F90028FE
:1066A00054D0002E01D12B230493FE239B0500938D
:1066B00052E0002BBFD1029B662B38D1631C9D4258
:1066C00000DCAC1E029B651C039300231E00049398
:1066D0000593E343DB171C40039B652B00D0F1E0DF
:1066E000651C00230693069B9D424EDD009815F025
:1066F000DFF87B1C0893030030333B70059A069B40
:10670000934205D1002C03D0BB1C08932E237B7031
:1067100015F0EEF8011C009814F016FF724914F001
:10672000F3FD069B009001330693089FDBE7631D92
:106730009D4200DCAC1F029B652B00D0ADE0002524
:1067400003933A3B049305952E00C2E700986649EF
:1067500014F0DAFD01360090029B662B03D0672B04
:1067600037D1042E35DC6B461B7D3B70029B672BBB
:1067700001D1731EE418631C9D4200DCAC1E002C8A
:1067800012D16623013703930494029B662B00D039
:10679000B0E0012E00DDEDE05449009814F000F95E
:1067A000002800D0ACE0E5E02E23250030227B70ED
:1067B000BB1C013E1F00002E74D0002D05D1049596
:1067C00001235B42059367334CE01A70013D0133AE
:1067D000EFE76B1F9C4270DB029A672A64D01300BC
:1067E000AC1F00250393059573E700230026039350
:1067F000203304933B4B039A0099D05814F0BCF813
:10680000002808D0049B039AF618354B0098D158FD
:1068100014F07AFD0090049B5B100493039B0433F7
:106820000393182BE6D13049009814F0B9F80028EA
:1068300005D000982E4914F067FD01360090029BA8
:10684000662B11D1AE4212DAA31901339D4203DC4B
:10685000AD1BAC1E00D56C1E002335190493013509
:1068600005966633039334E7029B652B09D16B1FB2
:106870009C4200DBAC1F2B230025049305953A3383
:10688000F0E7029B672B12D1231D9D4200DC6C1F99
:10689000A6420CDA731CE41ADEE70025029B04957D
:1068A000039350E704968BE71C00029B99E7029B39
:1068B000002503932B23049395E70025029B059560
:1068C000039309E7039B672B00D00AE7251E00D03E
:1068D00007E701252C0004E7FFFF7F3FF8FF7F3F1C
:1068E00010DE020028DE0200000020410000A0406F
:1068F000CDCCCC3D3B49009814F052F800282CD068
:1069000030217B1E1A782E2A60D0100030380928DA
:1069100053D901330193019B1B78302B14D1019A79
:1069200052782E2A09D10399662906D001994B7015
:10693000049B0A702D2B4BD1013E01373B00019A7D
:106940009A4247D331231370274B009A9A4204D8B6
:10695000039B663B5A425341E41A029B672B09D1C1
:10696000002C07DD3B00013F3A78302AFAD02E2A6E
:1069700000D01F00049B002B1AD02022079B0A2165
:1069800013401A00452313433B706B461B7C3000B9
:106990007B7013F0ABFE0A2113F08EFF3031B9701B
:1069A00030000A2113F088FF3C1D3031F9702700B8
:1069B00000233B70099BF81AEDE5392A02D0013219
:1069C0001A70A7E7019A19709342A4D0013B99E786
:1069D0000136B2E75A1E117819701300AFE701248F
:1069E00027E6C0460000A040FFFF7F3FF8B50D003E
:1069F00004001600FAF7F2FD2B00032723433B4265
:106A000019D1BE4217D9B2082900200013F060FD49
:106A10003100B94360183E406918002E02D03200A0
:106A200024F0B0FE80220549D2008B58002BFCD008
:106A3000FAF7C4FDF8BD29002000EEE700E00140B0
:106A4000F0B50D00002785B0110003901E0028004E
:106A50000F4B0222009703F047FEA81C80001EF097
:106A60007AFF039B040003606B1E3D0003934360A9
:106A700033688360039B9D4202D3200005B0F0BDC4
:106A80000135AF00F05908F03BFDE719B860F1E7B8
:106A9000FFFF000070B50600080020F009FE0500A9
:106AA0001EF0D8FF041E06D12A000849084805F048
:106AB00007FC0FF07CFE30001FF0BCF80121020043
:106AC0000300200009F07EFA70BDC0466A6703002B
:106AD0008CF9020010B5040020F0EAFD1EF0B2FBB4
:106AE00001280BD00649200020F0FCFD200020F0FA
:106AF000DFFD1EF0A7FB022800D0002010BDC0461D
:106B0000BB670300F0B59DB000AF0C68032859D9EE
:106B1000CB680025FB60042801D00D696D101C2393
:106B20002000F91802F02EFC7861002D5BD0A04CFB
:106B30006E216068FBF792F80600606800229621DB
:106B400004300EF04BF81823FA18D1180400300066
:106B500002F018FC3B6B013D0100C318002C05D16D
:106B6000994203D2013B1A782E2AF9D1013D31D244
:106B7000FE695C1A2500002E01D0751C65192B00DA
:106B80006A460E33DB08DB00D31A9D46220018004C
:106B90003B6124F0B0FE002E08D02E233A69601C21
:106BA000135510187969320024F0A5FE29003869C0
:106BB00006F00AFE012810D17E497F481FF02EFA08
:106BC0000FF0F5FD7D4B0025FB60A8E7013B1A782F
:106BD0002E2ACBD09942F9D3C8E706243B69C000DE
:106BE0000443FD617B61200001F040FF04F050FA96
:106BF000061E15D02E21786924F0E6FF00280BD060
:106C00006E4BFA689A4207D17B69C11A180006F0E8
:106C1000DBFD04F03DFA06003000BD461DB0F0BDBE
:106C2000182318200125FA18D2183818103B4021D3
:106C3000C01820F0E2FCBE603E61FB699D4205D9B0
:106C40005E4BFA689A42E7D1BE68E5E79D4204D000
:106C50007B695B5D2E2B00D097E02900786906F0F8
:106C6000B3FD18220823BA183860D01820F0EEFCC3
:106C7000002817D12A000823796918303818C0185D
:106C800020F07BFC18220823BA18D018FFF722FF47
:106C900078607B68002B14D13A684949464805F072
:106CA0000FFB8DE718220823BA18D0182F2109F0FE
:106CB000FBFD3B693969EA1A7B69182059180823DA
:106CC000DCE7386804F0E4F9041E48D1386804F0C1
:106CD000A5F9FB6904009D4208D13A4BFA689A4233
:106CE00004D15E226E2180681CF041FE7B68012B7E
:106CF00055D118220733BA18D01820F0A0FC18225A
:106D00000823BA187860D01820F0A0FC00220100F7
:106D1000786801F089FE12210200200008F0CCFB07
:106D200018220823BA18D0182F2109F0BDFD182207
:106D30000823BA18D018244920F0D4FC18220823BC
:106D4000BA18D01820F0B4FC1EF07CFA02281ED02D
:106D500018220823BA180C21D01820F003FD002EA9
:106D60000CD07A693B699446E91A6344180006F02E
:106D70002BFD22000100300008F09EFBBB68002BB9
:106D800000D1BC6026006B1C3B61013555E7182221
:106D90000823BA18D1182000FFF77CFED8E7182284
:106DA0000823BA18D1182000FFF774FED7E7C046B1
:106DB000C40900207F6703008CF90200D8F50200A7
:106DC0009E67030008D60200B367030010B50124D4
:106DD000037905499B005A580448224200D10448CF
:106DE000A243CA5010BDC0461003002010D60200B6
:106DF00008D6020010B504000FF0F2F90C498842E1
:106E00000AD020000FF02EFAA02204216379D205C7
:106E1000C133FF339B009950A223A022DB00D2058F
:106E2000D0586379D840012318401EF0B2FE10BD3F
:106E3000A422030070B50379064C05009B00185985
:106E400040081EF0A6FE01222B799B0019590A402A
:106E50001A5170BD1003002010B504000FF0C0F9E6
:106E6000084B984202D020000FF0C8F9A0226379A5
:106E7000D205C133FF339B0098580007800F1EF0E6
:106E800088FE10BDA422030013B50A4904000FF0C8
:106E9000E9F90521684661560FF0BAFE68460FF021
:106EA000DDFEA0230021044ADB00D1501EF071FE5C
:106EB00016BDC0469C2203000070004070B504005F
:106EC0000FF08EF9124DA84211D0124B98420ED0FD
:106ED00020000FF0B1F9290020000FF0C3F9A02223
:106EE0000C216379D205C133FF339B009950A02256
:106EF0000C216379D205C133FF339B0099502000E8
:106F000005F070FB044B002800D0044B180070BD46
:106F1000D4220300BC22030010D6020008D60200CF
:106F200070B5A222A025D200ED05AA581F23CA40A1
:106F30001100174C0340E056421EC90700D5421C01
:106F4000022A0BDC00218A421CDB124DEE5C300071
:106F50008E4201D00220E954E25470BD072A09DDB7
:106F60000C2A12DC0B490320CD5C002DF4D1023831
:106F7000C854F1E707490320C95C4D1EA9414942A5
:106F80000840E9E70A000800E6E703200C22E3E7EF
:106F90005F0200204B02002070B5050008000CF0D5
:106FA000C5FA0400431005D0124913481FF036F803
:106FB0000FF0FDFB28000FF013F9104988420AD0AA
:106FC00028000FF04FF9A02203216B79D205C133BD
:106FD000FF339B009950A02201236979D2058B4091
:106FE000002C04D0A121C9000548535070BD0549AB
:106FF000FAE7C0460C680300ACFD0200AC220300B7
:10700000D8F502000C05000070B5050008000CF072
:107010008DFA0B2303410400DB0705D40D490E480C
:107020001EF0FCFF0FF0C3FB28000FF0D9F80B4B4C
:10703000984202D028000FF0E1F8FF22A40092004D
:107040001440A0226B79D205C133FF339B00044862
:107050009C5070BDDE670300ACFD0200A42203005B
:10706000D8F50200032370B50B4004000800022B82
:1070700003D11C4B0B40062B28D10CF057FA1A4BAE
:1070800005009D4205D9194919481EF0C7FF0FF0A8
:107090008EFB20000FF0A4F8164988420AD0200089
:1070A0000FF0E0F8A02203216379D205C133FF334A
:1070B0009B00995060792900FEF7A8F8002D03D1B4
:1070C0000D4920000FF0CEF80C4870BD0CF092FA7C
:1070D00016F0F4F900220A4B14F0A0FC16F078F92F
:1070E000CDE7C046070080FFFF030000EB67030009
:1070F000ACFD0200EC2203009C220300D8F5020044
:107100000000E03F10B5034903481EF087FF0FF071
:107110004EFBC046CF670300ACFD020010B508006F
:107120000CF004FAFA239B005843FEF73BF80028C2
:1071300001D0FFF7E7FF014810BDC046D8F50200B7
:1071400010B508000CF0F2F9FEF72CF8002801D079
:10715000FFF7D8FF004810BDD8F502001F220379C1
:1071600001201340014AD35C584070474B02002075
:1071700010B5FFF7F3FF034B002800D1024B1800B6
:1071800010BDC04610D6020008D6020070B5CA4D28
:1071900028000FF025F8C94CA04205D028000FF0B8
:1071A0001FF8C74B98420BD103210020FFF7B8FE10
:1071B000022805D1C3490B689A1C012313430B60B5
:1071C000C14D28000FF00CF8A04205D028000FF0A8
:1071D00007F8BB4B98420BD102210120FFF7A0FE1C
:1071E000022805D1B7494B689A1C012313434B6011
:1071F000B64D28000EF0F4FFA04205D028000EF096
:10720000EFFFAF4B98420BD101210220FFF788FE20
:10721000022805D1AB498B689A1C012313438B606C
:10722000AB4D28000EF0DCFFA04205D028000EF088
:10723000D7FFA34B98420BD104210320FFF770FE28
:10724000022805D19F49CB689A1C01231343CB60C8
:10725000A04D28000EF0C4FFA04205D028000EF07B
:10726000BFFF974B98420BD105210420FFF758FE32
:10727000022805D193490B699A1C012313430B6122
:10728000954D28000EF0ACFFA0420BD028000EF068
:10729000A7FF924B984205D028000EF0A1FF884B23
:1072A00098420BD111210520FFF73AFE022805D1A3
:1072B00084494B699A1C012313434B61884D280074
:1072C0000EF08EFFA04205D028000EF089FF7C4B07
:1072D00098420BD10C210620FFF722FE022805D18F
:1072E00078498B699A1C012313438B617D4D2800DB
:1072F0000EF076FFA04205D028000EF071FF704B13
:1073000098420BD10B210720FFF70AFE022805D176
:107310006C49CB699A1C01231343CB61724D280041
:107320000EF05EFFA04205D028000EF059FF644B1E
:1073300098420BD112210820FFF7F2FD022805D157
:1073400060490B6A9A1C012313430B62674D2800A6
:107350000EF046FFA04205D028000EF041FF584B2A
:1073600098420BD10A210920FFF7DAFD022805D146
:1073700054494B6A9A1C012313434B625C4D28000D
:107380000EF02EFFA04205D028000EF029FF4C4B36
:1073900098420BD106210A20FFF7C2FD022805D131
:1073A00048498B6A9A1C012313438B62514D280074
:1073B0000EF016FFA0420BD028000EF011FF474B35
:1073C000984205D028000EF00BFF3D4B98420BD1A0
:1073D0001A210B20FFF7A4FD022805D13949CB6AF9
:1073E0009A1C01231343CB62434D28000EF0F8FE94
:1073F000A04205D028000EF0F3FE314B98420BD18D
:1074000014210C20FFF78CFD022805D12D490B6BB0
:107410009A1C012313438B60384D28000EF0E0FEC8
:10742000A04205D028000EF0DBFE254B98420BD180
:1074300017210D20FFF774FD022805D121494B6B60
:107440009A1C012313434B632D4D28000EF0C8FEF8
:10745000A04205D028000EF0C3FE194B98420BD174
:1074600016210E20FFF75CFD022805D115498B6B14
:107470009A1C012313438B63224D28000EF0B0FEAB
:10748000A04205D028000EF0ABFE0D4B98420BD168
:1074900015210F20FFF744FD022805D10949CB6BC8
:1074A0009A1C01231343CB63174D28000EF098FE5E
:1074B000A04231D02AE0C04630E102009C22030005
:1074C000A42203001003002078E1020088E10200FA
:1074D00090E1020098E10200A0E10200BC2203005A
:1074E000A8E10200B0E10200B8E10200C0E1020040
:1074F00038E1020040E1020048E1020050E10200F0
:1075000058E1020060E1020068E1020028000EF08C
:1075100067FE204B98420BD110210800FFF700FDB9
:10752000022805D11C490B6C9A1C012313430B64E0
:107530001A4D28000EF054FEA04205D028000EF08F
:107540004FFE144B98420BD100211320FFF7E8FCAB
:10755000022805D11049CB6C9A1C01231343CB643C
:107560000F4D28000EF03CFEA04205D028000EF082
:1075700037FE084B98420BD11E211420FFF7D0FC98
:10758000022805D104490B6D9A1C012313430B6596
:1075900070BDC046A42203001003002070E1020069
:1075A00080E10200A0230C220249DB055A5024315D
:1075B0005A5070474407000010B504000BF0CEFE8F
:1075C000084B98420BD0084B984208D0074B984282
:1075D00005D0074907481EF021FD0FF0E8F820000C
:1075E00010BDC0461CE20200B8E00200F4E0020058
:1075F000BF67030034FD020037B50400A06807F040
:10760000CBFF019000280ED06568074B9D4205D046
:1076100001AB00220121280007F078FE0CF0C4F82D
:107620000028EBD001983EBDD8F50200F0B5060069
:1076300000248BB0184B1948E15805F0B7FD03AF93
:10764000E05104341C2CF5D114230024734301931E
:107650000025795912481EF0B3FB0435300000F0C4
:1076600005F91C2DF5D1163DAB000D48F9581EF05B
:10767000A7FB300000F0FAF8013DF5D20134082CE8
:1076800003D104F0BFFB0BB0F0BD01231C42DFD1DE
:10769000019800F0EBF8DBE7C8E2020014000300F9
:1076A0002400002010B51920FFF7C0FF004810BDCE
:1076B000D8F5020010B50F4821F0B0FE002809D01F
:1076C0000D4821F008FF0D4B1B68984203D10C4B6D
:1076D0009A6E1A6310BD3F210A4A138801330B408A
:1076E000094909888B42F5D01188084C13806054F1
:1076F000F0E7C04634050020740500206403002034
:10770000C409002012090020140900202F090020BC
:107710000022094B10B51A80084B094909481A8004
:1077200021F081FE0122084B524208481A601EF0E7
:1077300068FC074B986610BD120900201409002050
:10774000B576000034050020640300207CFA0200B6
:10775000C409002010B50400431C03D0034B986EED
:1077600004F00EFE024B1C6010BDC046C409002090
:1077700064030020034B1888034B1B88C01A431E68
:10778000984170471409002012090020084A094B4B
:1077900010881988884201D130BFF9E7138806495B
:1077A000C85C3F21138801330B4013807047C046EB
:1077B00014090020120900202F09002070B50400D0
:1077C0004518AC4205D02178024821F079FE0134F9
:1077D000F7E770BD74050020F8B504004518AC4209
:1077E0000ED02378074E0A2B03D10D21300021F053
:1077F00067FE2178671C300021F062FE3C00EEE756
:10780000F8BDC0467405002070B504000825002CA2
:1078100008D02100082C00D929000348641AFFF77A
:10782000CDFFF4E770BDC0462A68030070B50500BF
:1078300004000826002C08D02100082C00D93100B3
:107840000448641AFFF7BAFFF4E72800FFF7DCFFEB
:1078500070BDC0462168030010B501000122024836
:107860001EF00BFB10BDC0462400002070B5041EA6
:1078700013D00A4D280010F029FD24180600A0425C
:1078800005D930BF280010F021FD8642F9D330BF62
:10789000280010F01BFD8442F9D870BDE0040020E0
:1078A000F7B5CC1CA400070020000E0001921EF0CA
:1078B00052F822000500054B4760866003600C3AD1
:1078C00001990C3024F017F82800FEBDFCE20200FC
:1078D000F8B504000D00A368002B0AD0344AE9680B
:1078E000914206D0EB58002B03D00422E3681A60C3
:1078F000F8BDA86B002822D063680022D9000623B7
:10790000043019430DF06AF9021E18D0237C002BB5
:1079100006D042680020E368216807F033FDE7E7FE
:107920002368181E07D02249EE688E4203D02149F1
:107930008D4200D01869E36852682900EDE723689A
:10794000002B12D16E6B002ED2D075680836002D38
:10795000CED000276B1E174A9F421AD3164BED1844
:10796000AD00AD599542B6D1C2E7227C002AE9D1DB
:107970000F4AE9689142E5D00E4A9542E2D0186973
:10798000E268616807F040FDE3681B68002BD9D00E
:10799000AEE7BB00F158914201D10137DAE7200090
:1079A000FFF796FFE3681B68002BF6D0A0E7C04600
:1079B000697C0000CC170300FFFFFF3FF0B514689F
:1079C00089B01700002C14D143685E6B002E10D0D4
:1079D000736803AD01938368083603936960AC60F4
:1079E000EA602C74019B9C4205D108492800FFF7EE
:1079F0006FFF09B0F0BDA300F1582800FFF768FF42
:107A00003B68002BF5D10134ECE7C046CC170300EE
:107A100010B54A68014921F098FC10BD7E69030049
:107A2000F0B58BB004000E00150000210822684656
:107A300023F07CFF1422002105A823F077FF2023E8
:107A400007936B46059408931C23002D02D0042D48
:107A500010D11A23216805A80693FFF739FF0221E8
:107A6000009F042F0ED12A00310020690BF0E6FEA2
:107A70000BB0F0BD1B23216805A80693FFF728FF74
:107A80000321EDE7381EF3D002AB002202940396E7
:107A9000049507F03BFC042DEAD00148E8E7C04616
:107AA000D8F50200F0B51F4B8BB08200D35803AF5E
:107AB0000C000822002106003800019323F036FF55
:107AC000019B05AD6B601423AB6000232800216887
:107AD0000594EF602B74FFF7FBFE0398042805D193
:107AE0002169300007F0AAFB0BB0F0BD00280AD0D6
:107AF00021001FF0A8FC022EF6D10BF043FD44003C
:107B000001202043F0E7022E01D00020ECE72623DD
:107B1000216828006B60FFF7DBFE3B68002BF4D187
:107B20006400EDE7C8E40200F0B51600724272414D
:107B30008BB01F320C00019200210822070003A81D
:107B400023F0F4FE019B05AD06930823079303ABD6
:107B500008930023216828002B740594FFF7B8FED2
:107B6000039B002B08D1002E06D11F33216828006B
:107B70006B60AE60FFF7ACFE039804281AD1206951
:107B80000BF0ECFB144BC2689A4211D1002E07D0C7
:107B9000236858681FF04FFB0100380021F00AFBF2
:107BA00080223243216938000BF0F0FB0BB0F0BDAE
:107BB0003200F7E7002805D021001FF044FC002226
:107BC0000100F0E7200020F0E7FF23000200034956
:107BD000380021F0BAFBE9E7A9C1000033680300CF
:107BE00070B504000D000B4921F0E4FA6968002229
:107BF00020000BF0CBFB0849200021F0DBFAA9683C
:107C0000002220000BF0C2FB0449200021F0D2FA30
:107C100070BDC0463C69030083380300107C03003C
:107C2000F7B50025436808300F0006002C000193CB
:107C3000019BAB4201D12000FEBDAB00F358084AC6
:107C4000934205D0074AD968914203D03B60013482
:107C50000135EDE73900586BFFF7E2FF2418F7E72D
:107C6000CC170300697C0000F0B58FB005000F0051
:107C7000406B05A901920293FFF7D2FF061DB600E3
:107C800030001DF068FE0400002120C021F0A9F89A
:107C900032002000103A1030002123F047FE012F5F
:107CA00005D1029B1B680393042B00D186E007AE2D
:107CB00008220021300023F039FE0922002309A800
:107CC0004260290003328260C66003740993FFF7A3
:107CD000FFFD079804282ED10598029BC668019ADB
:107CE0003900B047206120000BF038FB854265D198
:107CF00000230822290009A8089307930B930994ED
:107D00000A92FFF7E5FD079B002B57D001983843F7
:107D100036D107AA01001FF0A7FB0500294B9D42A1
:107D20004CD0280020F038FF27490200274804F0F3
:107D3000C7FA0EF03CFD0028D5D0019A3A4306D18F
:107D400006AB0121069507F0E1FA0400CBE7019BA1
:107D50005C00E4190134A40020001DF0FCFD221F8A
:107D60000390029920C023F0C6FD791C039B019A61
:107D7000306807F0CBFA040003981DF013FEB2E759
:107D8000019B5D00ED190235AD0028001DF0E3FDFB
:107D90002A000600079B029903600393089B083A98
:107DA0004360083023F0A7FD3200019938001FF02E
:107DB0005BFB050030001DF0F5FDAFE720000FB0C4
:107DC000F0BDC046D8F502008468030034FD02000F
:107DD00010B5C468002C06D142680449044804F078
:107DE0006FFA0EF0E4FCA04710BDC04645690300E1
:107DF00034FD0200F8B504000D0016001F001DF050
:107E0000F8FA002809D1200020F0C6FE0B49020034
:107E10000B4804F055FA0EF0CAFC042806D13B00CA
:107E200032002900206907F071FAF8BD2100F9F746
:107E3000B7FB3B0032002900F5E7C0466868030045
:107E400034FD0200F0B5154B89B016008200D558FC
:107E50000C000C2200210700684623F067FD182360
:107E600003A84560836000256B462168C3600394C6
:107E70000574FFF72DFD009B042B06D1320021690C
:107E8000380007F0C9FB09B0F0BD181EFBD06A46E8
:107E90002900012002961FF0E7FAF4E738E3020018
:107EA000F0B50D0085B001A907001600280002AA50
:107EB0001DF083F90023019902988B4225D13C20C3
:107EC0001DF05BFD244B04000360244B476083607E
:107ED000234B4563C360234B86630361224B03A995
:107EE0004361224B8361224BC361224B0362224BCD
:107EF0004362224BC3622800FFF792FE012812D989
:107F00001F4920481EF08AF809E09A008258D46878
:107F1000002C06D152681C491A4804F0D1F90EF021
:107F200046FC0133C9E7A36B0022181D4E210CF05B
:107F300055FE051E0DD0032243681A4009D11B6867
:107F40005B68F22B05D1031D012110481DF0ABFA2F
:107F50006860200005B0F0BD8CE40200297B0000C1
:107F6000697C0000F57D0000A57A0000457E0000D8
:107F70001D540200217A00007155020027550200AD
:107F80000E69030034FD0200E568030014E40200FA
:107F900037B50D001C0000231100009301220333AC
:107FA000280002F0A1FB012D07D0032D09D00949BB
:107FB00009481EF033F80EF0FAFB20680BF0CEF9FA
:107FC0003EBD206800F052FDA2686168FFF768FFBF
:107FD000F6E7C0466269030034FD020070B5050093
:107FE0000C200C001DF0B7FC024B45600360846060
:107FF00070BDC04650E40200F8B50F00B8421FD073
:10800000032505401ED1114B02689A421AD1406BDC
:10801000002816D0446808300600002C14D0631ED7
:108020009D4204D30A4BE418A400A059E6E7AB0034
:108030003900F058FFF7E0FF002802D10135EEE7E4
:108040000120F8BD0020FCE72000FAE78CE40200E4
:10805000FFFFFF3FF0B585B00500019108008B07D9
:1080600017D10B68154A93420BD10123029301AB40
:1080700003930024029E039FB44210D1104805B020
:10808000F0BD104A934204D103AA02A91DF095F84D
:10809000EFE70D490D481DF0C1FF0EF088FBA3006E
:1080A000F9580B4B994206D02800FFF7A5FF00288E
:1080B00001D10134E0E70748E1E7C0468CE4020063
:1080C00008D602009CDC0200AC68030034FD02000C
:1080D000CC17030010D6020010B5830703D1064B5E
:1080E00002689A4205D0054905481DF097FF0EF039
:1080F0005EFBFFF7AFFF10BD8CE402004568030094
:1081000034FD02000523020070B5094C094D2068BA
:10811000434309489B189B0018582B682260C018DD
:108120000F2319400901286008F048F970BDC046C6
:1081300068030020EC020020E4E40200A8390300F8
:1081400000B5080006292ED812F028FA040A1016E5
:108150001B2128009A18E223DB00D218107800BDFA
:10816000C4329200D05C8006800EF8E7C4329200E0
:10817000D05AC004400EF2E7C4329200D058000337
:10818000F8E7C43292009A1890780009E7E7C43201
:1081900092009A18D0780007000FE0E7C4329200EE
:1081A0009A18D078F1E7024A024B00201A60D6E70D
:1081B0008B69030010000020A83910B504000800E6
:1081C000062949D812F0EAF9040A141F2A343F009C
:1081D000E221A218C9005218137010BD3F210B40B4
:1081E0001800C4329200135D8B4303431355F4E728
:1081F0007F21C432920019401948135B8901034062
:108200000B431353E9E77F21C43292001940105900
:10821000144B490303400B431351DEE70F20C432D4
:108220009200A2181901937803400B439370D4E78E
:108230000F210B401800C4329200A218D3788B4350
:108240000343D370C9E70F20C4329200A218D1783B
:108250001B0101400B43F4E7034A044B1A60BCE7DF
:108260003FE0FFFFFF1FF0FFA9690300100000209F
:10827000F0B5D2B287B00F000593072113000B4071
:10828000013BDBB2042B02D92C4D2D4C25608A43D7
:1082900019020291002A29D12A4BC55C2D09ED4310
:1082A000EBB23D7801932C005B1BDBB204930826F4
:1082B000254B029A1B199B5C5A00D2B25BB2039207
:1082C000002B38DA1A210320013EF6B2FFF71AFF1D
:1082D000039B002EF0D10134049BE4B2E318DBB21F
:1082E000002BE4D1019BED1A3D701AE0D4431749ED
:1082F000E4B2CF5C0825144B029A1B199B5C5E000C
:108300005BB2F6B2002B0FDA05210220FFF7FAFE6E
:10831000013DEDB23300002DF1D10134E4B2002C67
:10832000E8D1059807B0F0BD39000120FFF7EAFE5B
:10833000002FE9D0ECE706210420C5E79669030089
:108340001000002019070000216F03007C75030056
:108350000022F0B505000F00FF200F248BB008AB02
:10836000654EDA710100C431890069188B781A09E9
:10837000B25C234012011343CA788B7013071B0FA2
:10838000F35CA243234013431A09B25C2340120159
:108390001343CB700138E5D2E223DB00EE5CB30877
:1083A000F31ADBB20593554B1B68002B0BD0E2226E
:1083B000C4218120D200890000013B00AA1869185D
:1083C0002818FDF783FF00244823029403930194A7
:1083D000009481222B1912019B181B78180004931A
:1083E0000723984320D008A92300049A07312800C6
:1083F000FFF73EFF0230C4B2023FFFB2002F78D039
:108400002B780393013EF6B2002E47D1E2222B19BE
:10841000D2009B181E78B308F31ADBB20593002331
:10842000029301930093D4E7354B009A9C469A5CE3
:108430002300C4339B00EB18997809090A4331499A
:108440008A5C019906926246DB78525C1907090F33
:108450000A432C491B098A5C2B490792029A8A5CC1
:1084600007991343069A52182649C95C01238918B3
:10847000FF2A00DC031CC918882309061B06C9183B
:10848000090F0020FFF73EFE039B013BDBB2039385
:10849000002BB7D10134E4B2013FAEE7059B013BAD
:1084A000DBB20593002B02D1049B002B18D12200D4
:1084B000C4329200535D00999B069B0ECB18DBB231
:1084C0000093535B0199DB045B0ECB18DBB2019385
:1084D0005359029A1B035B0ED318DBB2029378E761
:1084E00008A92300049A07312800FFF7C1FE040001
:1084F0008CE70BB0F0BDC046A56A0300F002002077
:10850000717403007D6C0300216E0300064B1B5C3D
:10851000002B05D0054B185C4843C011C0B2704712
:10852000034B185CFBE7C046CD6D0300466C0300AF
:10853000066B0300064B1B5C002B05D0054B185C3B
:108540004843C011C0B27047034B185CFBE7C046FC
:10855000CD6D030081750300566B0300F0B5037AFF
:108560008DB004007F2B00D145E1030007000025FA
:108570000933FF330837099301953E787F2E00D0E9
:1085800086E000230693019306998B00E31803937A
:108590001A7A481C1B7BC0B206907F2B00D11DE1CC
:1085A0009F49CE5C8D5C9F49AE4200D0F3E08D5C6C
:1085B000CB5C0493039B597A019B5918CBB201936E
:1085C000049BEB18DBB20793023B1B06DCD4A82606
:1085D000019B5D1BEBB20593A82E00D0E3E0039B4B
:1085E000A8215F7A5A7B7F085208BB180293019B2F
:1085F00020009A18D2B2DF1BFFF7A0FDFFB20500E2
:108600003A00A8212000FFF799FD2D1AEDB27F2234
:108610002B006DB293430893EB17E818584002996A
:1086200012F04AF92800CBB20299099312F05EF8D1
:108630000025C3B20A93059F029BDB19DBB20B93A3
:108640003A0031002000FFF779FD0A9B01370B9AB1
:108650001818FFB2C3B2974200D1B9E0099AAD1819
:10866000029AEDB2AA420DD8AD1A20216A465218DC
:108670001278EDB252B2002A00DAA7E0002B01D046
:108680000133DBB23A0031002000FFF795FDD7E758
:10869000012E7AD12B003100019A20001CF0BBFF83
:1086A000BA78614BA1789B185B7830000193FB7816
:1086B0000293FFF72BFF3F23E17803403000039341
:1086C000FFF738FF7F22594B9B5D1A40584B0492AD
:1086D0009A5D0F231A400592564A925D1A400692FF
:1086E000554A925D1A4007923F22544B9B5D089376
:1086F0007B78EB18DBB20A93039B134003937F2331
:10870000184083019C462A003F21C4329200135D29
:108710000F268B4303990B431355135B48490B40BA
:1087200061460B431353049B10595903454B0340B7
:108730000B430598190C3140000113510843A2184E
:1087400090701B0E0698B3430799034309011E401E
:108750000E4320206946D6708122091863190978D2
:1087600012019A181170E222D2009B180299019A04
:10877000013552181A700A9BEDB29D42C3D1099B74
:108780000437BB4200D0F8E6FBE6022E88D12B006E
:10879000019AFF2181E72C48AE4201D9C55C07E769
:1087A0008D5C835C05E7049B019A31009A18D2B274
:1087B0002000FFF7C3FC059A050031002000FFF7F9
:1087C000BDFC079B2D1AEDB2029320E7013B58E751
:1087D0000136F6B2AF2E00D0FEE6D5E602318900B2
:1087E0006118019B497859186368C9B2002B04D0FD
:1087F0002000FFF7ADFD0DB0F0BDE2228025D200D4
:10880000A0186D001A00C4329200125D067892061C
:10881000D20EB21A013302700130AB42F2D1E7E757
:10882000B66A03007D6D030071750300A66B03003B
:10883000B5690300056A0300556A0300217403004B
:108840003FE0FFFFFF1FF0FFF66B0300032230B590
:1088500002400121002A04D1084C03680D00A34204
:108860000AD00B0003401D1E06D1002A04D1036864
:1088700003481B1A5D425D41280030BD18D6020036
:108880004401030010B50400FFF7E0FF01230028B6
:108890000AD102332340022B05D105480440063C8F
:1088A000601E8441E0B203000120184010BDC046A4
:1088B000070080FF10B520F06FF90349020003485C
:1088C00003F0FEFC0DF073FFB875030034FD0200E9
:1088D00010B5040010201DF03EF8044B84600360C6
:1088E000034B43600023C36010BDC04640DE02005E
:1088F00031590200F7B504000E00019301208B18D6
:108900000A0000210093009B934212D827250029DA
:1089100000D0053D224F2A003900200020F015FD2F
:10892000009B9E4214D32A003900200020F00DFD48
:10893000F7BD1378272B08D0223B5D426B41DBB299
:108940000132002BDFD02725E4E700230100F7E701
:108950003278954205D12A001249200020F0F5FC1A
:108960001AE011495C2A14D01F2A09D97F2A15D090
:10897000019B002B02D053B2002B07DB3900ECE740
:108980000A490A2A05D00A490D2A02D0092A05D126
:108990000849200020F00EFC0136C1E70649DCE75B
:1089A00082790300817903008579030088790300C7
:1089B0008B7903008E79030091790300194B70B510
:1089C00006000D0098420ED14968A86804F0CAFE5E
:1089D000041E08D028001EF01CFEE0000023062420
:1089E0002B60204370BD10201CF0B5FF69680400A7
:1089F00081600660A86804F097FE6B686060591C8F
:108A00002B68994209D1AB68E3600023E268A16852
:108A100020005354AB602B60E4E7A8681CF0B1FF62
:108A2000E060F2E70818030070B504000D00002AAA
:108A300005D004F0C9FEC3000620184370BD04F041
:108A400091FE0028F7D12A00210002481CF03EFECA
:108A5000F4E7C0460818030010B50A0001000248F8
:108A60001CF034FE10BDC04640EE0200094B10B5AC
:108A70000340062B01D1C00810BD830708D1064B67
:108A800002689A4204D18168C06804F09DFEF3E751
:108A9000FFF710FF070080FF08180300064B10B512
:108AA0000340062B03D1C0081EF0CAFB10BD83682B
:108AB000C0680B60FAE7C046070080FFF0B50F0002
:108AC000002689B0110005001C0038000096032321
:108AD000320001F009FE0E20B7420FD0012F0FD156
:108AE00002AA102104A807F0D3FE216802A83200D0
:108AF0000AF04CFC04A92800FFF760FF09B0F0BDA4
:108B0000206883071BD1134B02689A4217D104A92E
:108B1000FFF7C4FF104B060020680340062B0CD162
:108B2000C0081EF07EFB04001020049F1CF013FF01
:108B300005608760C6604460E0E74468F4E704A924
:108B400001220AF0ADFE002205990498FFF76CFFA0
:108B5000D4E7C04640EE0200070080FFF0B58BB0BE
:108B6000049008680D00069207930AF0F7FB0600D0
:108B700068680AF0F3FB864202D06868FFF79AFE45
:108B800008A92868FFF78AFF040009A96868FFF7A9
:108B900085FF089A0590A3180393049B2700022BD6
:108BA00019D9AB681E498B4206D0012130000091D3
:108BB000210007F087FF0700049B032B0BD0EB6815
:108BC000174A934207D00122210000923000089AF0
:108BD00007F078FF0390039B059AD91B069B38008A
:108BE0000093099B1CF053FD002809D1079B013815
:108BF000002B0FD00B490C481DF010FA0DF0D7FDDB
:108C00000A4B9E4208D10100200020F0E1F9440007
:108C1000012020430BB0F0BD041B6400F8E7C04600
:108C2000D8F50200AA790300ACFD02000818030081
:108C3000F0B58DB0040003910AF090FB04A9060082
:108C40002000FFF72BFF0190039883071ED10368D4
:108C5000314A934217D106AA05A91CF0AEFA0024A6
:108C60002500059B9C4220D32900002508A81EF062
:108C7000BCFC0A9C059B9D4236D308A93000FFF737
:108C80009DFE0DB0F0BD254A934208D02348002236
:108C9000C36801210293029C03ABA047039006AA7C
:108CA00005A903981CF021F8D9E7069BA700D8591D
:108CB0000AF054FB864205D019491A481DF0AEF956
:108CC0000DF075FD002C01D0049BED18069BD859C2
:108CD000154B0340062B05D1C0081EF0A7FA2D182E
:108CE0000134BEE78068FAE7002D06D02000049A20
:108CF000019922F000FE049BE418069AAB009858F4
:108D000007A9FFF7CBFE079A0100200022F0F3FD30
:108D1000079B0135E418ADE79CDC020004D4020097
:108D2000BE79030034FD0200070080FFF0B50700A4
:108D300087B008680D000AF011FB04A90600286836
:108D4000FFF7ACFE05A904006868FFF7A7FE0390D3
:108D50002000022F07D901230093AB68049A210059
:108D6000300007F0AFFE059A041B049BA418064DC3
:108D70009C4205D8039922F0AFFD002800D1034D95
:108D8000280007B0F0BDC04608D6020010D6020089
:108D900073B50D00060069462868FFF77FFE01A93C
:108DA00004006868FFF77AFE0100022E02D9084825
:108DB00007F052F9019A0098064D824206D8801AAF
:108DC000201822F089FD002800D1034D280076BD2F
:108DD0009879030008D6020010D60200F0B58FB0D3
:108DE000079010680C0016000AF0B8FA0690012CE3
:108DF00031D070680AF0B2FA069B834202D07068E4
:108E0000FFF758FD0DA97068FFF748FE0D9B08900D
:108E100009930DA93068FFF741FE0D9B0B90049359
:108E2000079B012B1CD1049B5D1E01235B420A930F
:108E300000242700049B03940593059B002B13D16A
:108E4000039B002B23D1214B069A0E209A4200D07F
:108E50001F480FB0F0BD072309931E4B0893D8E7B6
:108E6000012300250A93E3E70B9B09995A19012373
:108E7000089800931CF00BFC002816D1039B002BD4
:108E800019D1079B002B09D12F00049B5C1E049B6A
:108E90000134E21B934212D13068DAE7079B2C00C1
:108EA000012B0AD001232F0003930A9BED18059B89
:108EB000013B0593C1E72C00F7E7039FE7E70B9B16
:108EC0000698D9191CF002FCC3E7C0460818030035
:108ED00030EE0200277A0300F0B589B004900868EC
:108EE0000D000AF03BFA070068680AF037FA87427B
:108EF00002D06868FFF7DEFC06A92868FFF7CEFD00
:108F0000060007A96868FFF7C9FD069A0590B3181F
:108F10000393049B3400022B19D9AB681D498B4283
:108F200006D0012138000091310007F0CBFD04008C
:108F3000049B032B0BD0EB68164A934207D0012207
:108F4000310000923800069A07F0BCFD0390079BA1
:108F50000025002B12D1039B2000191B20F047F89D
:108F6000013045000120284309B0F0BD05992000DB
:108F700022F0B2FC002808D101353400079A039B87
:108F8000A618B342F2D26D00ECE7200020F017F8EB
:108F90000600F2E7D8F50200F0B58BB00E0007002E
:108FA00003920AF0DBF9050030000AF0D7F9854298
:108FB00002D03000FFF77EFC05A93800FFF76EFDF8
:108FC00006A904003000FFF769FD069B0200002B94
:108FD00005D11A491A481DF021F80DF0E8FB19498E
:108FE0008D4227D10E2107910891099103990029FB
:108FF00022DD079703992000009105991CF047FB9B
:10900000002811D0071B3A00210028001CF05EFB4D
:10901000059B0699DA1B521A7918079061182800E7
:1090200008961CF053FB099007A90320FCF78EFE5D
:109030000BB0F0BD0449D6E70997DBE7037A0300DC
:10904000ACFD02000818030030EE020010B501006C
:1090500001481CF04CFC10BD0F90020010B501003F
:1090600001481CF044FC10BD21900200F7B5060039
:10907000080001A9FFF712FD019B0500002B01D19B
:109080001348FEBD134B04009E4207D10027019AEE
:10909000631B9A4211D8002F07D1F1E70E4B9E4275
:1090A000F4D0019A631B9A4201D80C48E9E7207872
:1090B000B04701340028F4D1E2E720780BF0EEFE4F
:1090C000002803D02078B047071ED9D00134DEE74E
:1090D00008D60200054F01001D4F010010D6020006
:1090E00010B501000148FFF7C1FF10BD854E01001A
:1090F00010B501000148FFF7B9FF10BD9D4E0100FA
:1091000010B501000148FFF7B1FF10BDB54E0100D9
:1091100010B501000148FFF7A9FF10BD054F010080
:1091200010B501000148FFF7A1FF10BD1D4F010060
:10913000F0B585B006000C0017000AF00FF969467B
:1091400005003000FFF7AAFC0600042F23D1A30777
:1091500016D1124B22689A4212D101AA210000981E
:1091600008F0E0FA002802D10D4806F075FF0199D9
:10917000029A2800521A71181CF0A8FA05B0F0BD26
:1091800000232200009928000AF0A8FA335C01208D
:109190005B001843F2E70020F0E7C046B81E03006A
:1091A0000463030070B51D008AB0002968D01868F8
:1091B000344C03002340062B05D083071FD1324BCC
:1091C00002689A421BD10239012953D806A9FFF738
:1091D00065FC060028680440062C0ED1C0081EF06D
:1091E00020F804001020069D1CF0B5FB274B85607D
:1091F0000360C66044600AB070BD4468F2E70129AC
:1092000038D80122104210D04410210006A81EF0C8
:10921000ECF9089B220000211800019322F086FB44
:1092200006A91A48FFF7CAFBE5E703A91FF0CAFC25
:10923000002805D0049A039914481CF047FADAE78D
:1092400028680AF08DFA1021002800D0411006A8E5
:109250001EF0B4F9286806F053F90400200006F067
:109260009BF90028DCD00AF061F9C1B206A81EF013
:1092700030FAF3E7064907481CF0D0FE0DF097FAE4
:109280000548B8E7070080FF0818030040EE020019
:10929000E475030034FD020030EE020073B50400F3
:1092A000080001A91600FFF7F9FB0500042E06D1FE
:1092B0000300019A0749200020F047F873BD0649D2
:1092C00020001FF077FF0123019A29002000FFF7FB
:1092D00011FBF3E7137A0300D9830300F7B502000B
:1092E0001C4B05000C001A401E00062A19D10B4029
:1092F000062B04D1441A60426041C0B210E0C0089D
:109300001DF08FFF07002640062E0CD1E0081DF04F
:1093100088FF002F09D0002807D0874205D0002001
:10932000FEBD4768EFE76068F3E769462800FFF78E
:10933000B5FB01A905002000FFF7B0FB009A019BD7
:1093400001009A42EBD1280022F0C6FA4442604163
:10935000D3E7C046070080FF084B07B50340062B44
:1093600008D0830704D10268054B92699A4201D064
:10937000FFF7A0FA01A9FFF791FB0EBD070080FFE0
:109380003D9900000A4B13B503400C00062B08D092
:10939000830704D10268074B92699A4201D0FFF714
:1093A00089FA01A9FFF77AFB019B236016BDC0462D
:1093B000070080FF3D990000F0B59BB00B900C00BA
:1093C000079210210EAA12A8099307F061FA079BD1
:1093D0009C4208D30B9A12AB13CB13C21B681360C9
:1093E0000B981BB0F0BD21787D2914D1631C059327
:1093F000079B621C934208D961787D2905D112A888
:109400001EF067F9059C0134E1E7B549B5481CF049
:1094100005FE0DF0CCF97B2904D012A81EF059F9F5
:109420000594EFE7079B651CAB4243D961787B2924
:1094300004D112A81EF04DF90595E3E72B007D2914
:1094400003D0212901D03A291FD100252E001A78F6
:10945000212A23D00022049200211A7805913A2A69
:1094600031D15A1C5B7805927D2B30D0130001223C
:1094700007998B421ED219787B291FD10132013303
:10948000F6E7079A01339A4214D01A787D2A03D05E
:10949000212A01D03A2AF4D11E00D8E707995A1C94
:1094A000914209D95A780492723A012A04D80233B7
:1094B0009942D1D88C49A9E78C49A7E77D29DED10B
:1094C000013A002ADBD1059A0593069205E0079B35
:1094D000059A9342EED900230693059B1B787D2BBA
:1094E00001D0834992E7002D45D0002328781693B8
:1094F0000BF0E0FC2C00002822D0099B1B6808938D
:10950000002B01DD7B4981E716AA310028001CF001
:10951000A6F8209A169B013A04009A4202D876498E
:10952000764874E7219A01339B009F580122099BDA
:1095300052421A60B4422ED2714806F08DFD0134B9
:10954000B44204D223782E2B01D05B2BF7D1611BC0
:1095500001222800FFF768FA002205000100229886
:109560000BF03CFB002804D1290066481CF04FFD9D
:109570004FE74768DEE7099B1B68002B01DA624969
:1095800044E7209A013A9342C9D2013321999A00C3
:109590005758099A1360069B002B16D1049B002B89
:1095A00058D010AA102116A807F072F9049A3900B1
:1095B000733A531E9A4110A8D2B209F0E7FE16A9D9
:1095C0005248FFF7FBF9070002E0049B002BE8D1AB
:1095D00001235B420D931093069B002B00D1B6E054
:1095E000F8F7D8FB229B059A0293219B06990193D9
:1095F000209B16A80093099BFFF7DEFE16A81EF01D
:1096000057F80026179B0400C3180A9303780493A5
:10961000B34213D03E4D1900280022F0D5FAB042D3
:1096200000D06FE16678002E17D03100280022F0BC
:10963000CBFA002800D067E1060004902378089355
:109640002B2B0CD02D2B48D00425202B08D0002507
:10965000089506E073230493A3E70496EEE702253A
:1096600001342378232B02D1133B1D43013423788B
:10967000302B07D1049B002B01D13D330493002EE6
:1096800000D130360DAA0A9920001BF0E8FF0378BC
:1096900006902C2B04D10C3B1D4303000133069391
:1096A000069B1B782E2B06D1069810AA01300A992A
:1096B0001BF0D5FF0690069B1C78002C07D02100DC
:1096C000144822F081FA002800D022E10400069B11
:1096D0001B78002B22D0104998E60025C0E7C04631
:1096E000E1760300ACFD0200227703000977030056
:1096F0003A7703005E770300A877030004FA0200BC
:10970000C177030040FA0200DE7703000818030067
:10971000287803002D7803003D78030016A81DF07B
:1097200078FF049B002B08D13800FFF7ABF83C23EF
:109730000493002801D002330493002E00D1203678
:10974000089B002B0CD0732C06D174495EE6069D55
:109750002C002E000895E7E7632C01D1704955E6EF
:10976000049B3D2B1FD05E2B1FD03C2B01D13B3BDC
:109770001D433800FFF76AF800282DD0632C50D025
:1097800026D8472C13D8452C26D2002C40D0252C87
:1097900022D038001FF000FA22000300614962481D
:1097A00002F08EFD35E64023E2E78023E0E7582C07
:1097B00053D0622CEDD1002303930D9B0222029320
:1097C00061230196009539000EA80CF08BFA19E67A
:1097D000672C17D8652C1BD33800FFF753F80028E7
:1097E0006CD0002C56D06E2C54D0472C3FD8452C32
:1097F00041D2252C50D038001FF0CEF922000300B2
:109800004A49CCE76F2C1AD0782C26D06E2CC0D1C8
:10981000002303930D9B01960293009561230A2276
:10982000D1E7380009F082FE0D9B16A908700122CD
:1098300001932B0000960EA80CF0F8F9E2E5EB0678
:1098400002D580239B001D43002303930D9B0196AB
:109850000293009561230822B5E7002223000392BA
:109860000D9A173B0292019600951022ABE7230058
:10987000653B022BBFD8380009F0BCFE109B2200CC
:1098800002930D9B011C01932B0000960EA81FF064
:1098900014FDB7E56724EEE73800802409F0AAFE3E
:1098A000234911F031FD109B640002930D9B2C4362
:1098B0000193011C009623006622E7E7049B3D2BE1
:1098C00001D11C49A2E5002C01D0732C13D116A99B
:1098D0003800FFF757FD109B0100169A002B00DAA5
:1098E0001092109B9A4200D916930D9B00960193FB
:1098F000169A2B009FE738001FF04EF92200030054
:109900000D494CE7013499E633000234049E049378
:1099100094E6069B01330693D9E6C04656780300C9
:1099200082780300B5780300ACFD0200E6780300FE
:109930000000C8421A7903004F790300F0B5A1B0C6
:1099400004000D000D920A2800D0E6E1073C0692C3
:10995000144038D11368BD4A93422ED10FAA10A9E2
:1099600006981BF02AFC0694109B11A908930F9BE4
:1099700028000993FFF792F800230A900C93AB0795
:1099800006D1B34A2B689B1A59425941CBB20C936A
:1099900014AA102118A806F07BFF119A00279446FC
:1099A0000A9B0A9C63440593059BA34212D8089B1B
:1099B000BB4200D1A7E1A749B1E0A74A934202D137
:1099C0000F941094D0E70DAB0F9301231093002355
:1099D0000693C9E72178252904D018A81DF079FE3F
:1099E0000134E1E7059B661CB34205D89B499C48BE
:1099F0001CF014FB0CF0DBFE6178252904D118A8BB
:109A00001DF067FE3400EBE7002528290ED1A01CCD
:109A100006003378292B1CD1311A0122FFF704F8F4
:109A200001000698F8F71AF9050001360023340002
:109A300040220026302104200B9320330793059BFE
:109A4000A34219D923782D2B0AD12C3B1E43013474
:109A5000F5E7059BB34201D88249C8E70136D8E74C
:109A60002B2B01D1293BF1E7202B01D10643EEE757
:109A7000232B49D0302B44D000231293059BA342C3
:109A800045D801235B421393059BA342AED92378AB
:109A90002E2B15D1059B601C8342A7D963782A2BF6
:109AA0004FD1089A3B00BA4238D9099A9B0098587E
:109AB00009F03CFD013713900234059BA34295D970
:109AC000002D07D1089A3B00BA4227D9099A9B007A
:109AD0009D5801372278672A5DD8652A00D3D1E0E6
:109AE000582A75D035D81300453B022B00D8C9E061
:109AF0000A9B5D49E41A00941300594802F0E0FB08
:109B000078E716430791A2E710230B939FE723788A
:109B10002A2B0FD1089A3B00BA4202D85349544825
:109B200066E7099A9B00985809F000FD01371290EA
:109B30000134A6E7200012AA05991BF090FD04004D
:109B40009FE7002313AA059913931BF088FD0400D7
:109B5000B3E7632A49D0642ACAD103222B001340F9
:109B6000022B0AD1434B2B40062B06D0FF23DB05EB
:109B7000E818904301F066F80500139B0A2203934E
:109B8000129B00960293079B01936123290014A85E
:109B90000CF0A8F824E7732A16D8722A00D381E0C3
:109BA000692ADAD06F2AA3D10B9B002B02D0842321
:109BB0009B001E43139B00960393129B0822029363
:109BC000079B01936123E1E7752AC6D0782A8FD1DC
:109BD0001300139A173B0392129A0292079A01926A
:109BE0000B9A164300961022D0E7224B2B40062BEF
:109BF00005D0AB0716D1204B2A689A4212D11CA976
:109C00002800FFF7BFFB1C9A0100012A01D01B4965
:109C100085E7129B019320230093330014A80CF0D6
:109C200005F8DDE62800FEF711FE00280BD028001D
:109C300009F07CFC129B1CA90870019320230122CF
:109C400000933300EAE70E4969E7C0469CDC020056
:109C500040EE0200AC760300CCCB0200FE750300A0
:109C6000ACFD020010760300777603002676030031
:109C700034FD0200070080FF081803004D76030042
:109C800066760300280009F0B5FC139B2278029346
:109C9000129B011C0193079B14A8009333001FF033
:109CA0000CFB9DE616AA10211CA806F0F1FD2378F6
:109CB0001A00723A50425041C2B2722B09D00C9B2A
:109CC000002B06D0AB0704D1544B2968994200D130
:109CD0000422290016A809F059FB139A1D9B002A9B
:109CE00000DA1393139A9A4200D91A00129B1E9914
:109CF0000193202314A8009333000BF097FF1CA8B6
:109D00001DF087FC6CE60C9B4448002B00D14448B6
:109D100018A9FEF753FE050019E0080009F01EFB24
:109D200016A906002800FEF7B9FE0700072C22D16D
:109D300018A90D9809F038FC0025A84207D01899F9
:109D4000A94207DC364B0E359E4200D0354D280027
:109D500021B0F0BD169B1CA859431DF046FC1E9B6C
:109D6000169A059300930121189B38001DF0FFFD02
:109D70001CA93000CDE70D9809F0F0FA86420FD10A
:109D80001CA90D98FEF78AFE1C9D05901D2C16D867
:109D9000192C3AD2052C21D0122C1FD00025D6E741
:109DA0001E4B00259E42D2D101221CA90D981EF007
:109DB00009FFA842CBD01C9B1D9D0593E6E71F2CF5
:109DC000ECD10123059A009316992B0038001BF063
:109DD0005EFC154D0028BAD1144DB8E7169B1CA89F
:109DE000E9181DF002FC1E9B169A39001800069314
:109DF00021F081FD169A1E9B944606936344180039
:109E00002A00059921F077FDB2E70095059B169A87
:109E1000390020001DF0DFFDDBE7C04640EE020008
:109E20000818030030EE020010D6020008D6020027
:109E300070B50C008AB0050004A920681600FEF772
:109E40002DFE00230593049B0100C218029605AB6A
:109E500006A801940095FFF7AFFA06A90248FEF79D
:109E6000ADFD0AB070BDC04608180300F0B505008E
:109E700087B008680C0009F071FA0090012D2AD90A
:109E80006668022D28D0A06809F050FB050000216B
:109E900008001AF013FF04A901902068FEF7FEFDE8
:109EA000049B0400C7183F4B9E423FD1A7422CD9C8
:109EB00020780AF0E7FF002811D1A74225D9002D0C
:109EC0000FD121003A1B00981BF000FC0100019803
:109ED000F9F7F2FC19E0334E01256D42D7E7013462
:109EE000E4E7260030780AF0CDFF002802D10136E1
:109EF000B742F7D12100321B00981BF0E7FB0100AD
:109F00000198F9F7D9FCB74202D8019807B0F0BD23
:109F1000340020780AF0B6FF002802D00134A742AE
:109F2000F7D1EB175B1BDB0FED1AC6E7300009F02A
:109F300015FA009B834202D03000FEF7BBFC05A956
:109F40003000FFF71FFA059B0390002B17D116492D
:109F500016481CF063F80CF02AFC3E002100321B6E
:109F600000981BF0B3FB01000198F9F7A5FCB7427C
:109F7000CBD9059BF418EB175B1BDB0FED1A260002
:109F8000059B0293002DE8D0029BF3189F42E4D377
:109F9000029A0399300021F09FFC0028DED00136A0
:109FA000F0E7C046D8F50200037A0300ACFD0200DA
:109FB000F0B50D008BB0022803D8FFF757FF0BB0A8
:109FC000F0BD086809F0CAF908A9049028686C680F
:109FD000FEF764FD0090A86809F0A8FA431C07008A
:109FE0000021180005931AF069FE354B05009C42CC
:109FF00002D1344806F030F809A92000FFF7C2F971
:10A00000099B0690002B05D12F4930481CF006F81B
:10A010000CF0CDFB089A3C009446009B63440293ED
:10A02000BB000393099B0193019A029B9E1A002C8B
:10A030000BD0009BB34208D8019A0699300021F05A
:10A040004BFC002822D0013EF1E7EB68BE009C19D2
:10A05000009A029B00999A1A04981BF037FB206023
:10A06000002F11D0059BDC1BEB68A70099193A0063
:10A07000180021F049FC6B6800211A1BEB68920064
:10A08000D81921F053FCAC60280098E7039AEB68DC
:10A09000944663440793029B04989A1B019B013FDB
:10A0A000D21AF1181BF012FB079B02961860E317F7
:10A0B0001B1BDB0FE41A039B043B0393B2E7C04670
:10A0C000D8F50200187A0300037A0300ACFD020001
:10A0D00080235B051869034B1B7843438020C00233
:10A0E000C01A70477009002080235B051869034B74
:10A0F0001B7843438020C002C01A704771090020BA
:10A1000070B5084DC4012B68002118191BF0ACF87C
:10A110002868054B00197F3000781B788342F0D205
:10A1200070BDC0466C0300206F09002010B5C379D4
:10A130000400002B08D0064A037981791068DB01FE
:10A14000C01801301BF090F80023237210BDC046E8
:10A150006C03002010B5034903481BF05FFF0CF0AF
:10A1600026FBC0462E7A0300ACFD020010B5124B50
:10A1700001001A684379DB01D31818007F30047896
:10A18000FF2C08D10879C00112185278FF2A0FD08D
:10A19000887990420CD08A799B180132D2B25878D3
:10A1A0007E2A01D08A7110BD00234C718B71FAE7B1
:10A1B00001204042F7E7C0466C030020F82270B54A
:10A1C000920213784D2B01D08022D202802680206B
:10A1D00076053469336964421440E41AC002316977
:10A1E000001B10F0F9F9284B284918703369E21860
:10A1F00052185D421540264B264A27499A1A521892
:10A200003169954230D38020C002401B10F0E4F940
:10A21000224B641B1870E411214BE4B21C70A12086
:10A22000012300251F4A20491360C0004D604B6880
:10A23000002BFCD01358DBB2A342F7D21B490133E9
:10A240000B7001235360FFF743FF03780500184CA0
:10A25000FD2B0BD180235B051869164BC009C01874
:10A26000C0012818206070BD6D18C9E7FFF73CFFDA
:10A270000378803DFD2B01D12560F4E7FFF734FF23
:10A28000FD211AF0F1FFF7E771090020FF87FFFFBA
:10A290009C0200200000002070C203007009002012
:10A2A0006F09002000D00040FCD00040720900205F
:10A2B0006C030020FFFFFF01F7B5254B254F1A78EF
:10A2C000254B14001B7839680133E001405CFF28FE
:10A2D00039D00134E4B29C4200D101249442F4D13B
:10A2E000802300265B051B69DB090093E3010193D2
:10A2F0003B68E2019D182A78280053425341F61822
:10A300001AF0C8FF0023002815D1134B01341B7825
:10A31000E4B201339C4200D101240D4B1B78A342CF
:10A32000E4D1072E11D91BF041FBC6E7DA01AA5C84
:10A33000002AEAD10133009A9342F7D13868019B91
:10A34000C0181AF09DFF2000FEBDFF24FBE7C046A9
:10A35000720900206C0300206F090020F7B5070088
:10A360000D0001240E4B1B7801930E4B1E68019BC0
:10A370009C4202D9FF242000FEBDE10171180B7838
:10A38000FE2B09D18B78AB4206D103312A0038006D
:10A3900021F0A2FA0028EED00134E4B2E7E7C0468B
:10A3A0006F0900206C03002010B5054A037910687E
:10A3B000DB01C018817800220330FEF735FB10BDA9
:10A3C0006C030020F0B585B002900D0016000393D9
:10A3D00078294BD8FFF7C2FF0400002E3ED0FF289B
:10A3E00001D0FFF78DFEFFF767FF0400FF2805D1BE
:10A3F0001F4920481BF012FE0CF0D9F91E4FC00176
:10A400003B680190FE2118181AF02EFF3B68019A54
:10A41000E9B2981802301AF027FF3868019B2A0029
:10A42000C01803300299FCF7E1FA0C201BF093FAF4
:10A43000039A0300002A17D0104A1A600E4A1C71B2
:10A4400012685C71E4011419A278DE7102329A710B
:10A4500001221A726A46127B5A7202E03300FF2808
:10A46000E3D1180005B0F0BD054AE6E70023F8E7A0
:10A470004B7A0300B4FB02006C03002070F602006C
:10A4800028F7020007B501A9FEF77CFF0199FFF745
:10A4900065FFFF2805D1054905481BF0BFFD0CF0FD
:10A4A00086F9FFF72DFE03480EBDC046617A030012
:10A4B000B4FB0200D8F50200F7B50192027A05005C
:10A4C0000091002A01D1FFF745FEC479002C06D186
:10A4D000214A17680279D201D25D002A04D10922EB
:10A4E00001201A604042FEBD69797E22C9017918B7
:10A4F00008007F30AB790078D21AFF2809D128797B
:10A50000C00138184078FF2819D0C01A824200D9FB
:10A5100002000198061B964200D91600002E19D0A1
:10A52000009A01331019C918320021F0E4F9AB790F
:10A530009B19DBB27E2B04D0AB71A419D4E70022A7
:10A54000E7E70023AB716B79DB01FB187F331B78E6
:10A550006B71F2E72000C6E76C030020F0B585B010
:10A560000393037A04000192002B01D1FFF7F2FD5F
:10A57000C379002B34D02D4A03791268DB019B5C30
:10A58000002B2DD0019B02910093009B002B2CD01F
:10A590007E22A379D71A009A974200D917006079D2
:10A5A000224E0133C001C01833683A0018180299CE
:10A5B000FCF71CFAA379DB19DBB27E2B33D1002325
:10A5C000A371FFF779FE0500FF2811D12079FFF76D
:10A5D00097FD002323721C23039A13601D3B03E0A5
:10A5E0000923039A13600A3B0193019805B0F0BD5B
:10A5F00060793368C001181829007F301AF034FEE2
:10A600003368ED01581961791AF02EFE62793368CA
:10A61000D2019B187F331B786371029BDB19029375
:10A62000009BDB1BB0E7A371F7E7C0466C0300207B
:10A63000002170B508001AF041FB012405000C4B05
:10A640001B78A34201D2280070BD0A4AE3011068BA
:10A65000C0180378FE2B08D1817800220330FEF762
:10A66000E3F901002800F9F727F90134E4B2E6E73D
:10A670006F0900206C03002073B501A9FEF782FE6C
:10A680000199FFF76BFEFF2805D10F490F481BF01A
:10A69000C5FC0CF08CF800257E260D4B1C68C30110
:10A6A000E31859789B780233DBB2C201A2187F32DB
:10A6B0001078FF2804D1C81A40191BF06AFA76BD39
:10A6C000F31AED180023F0E7617A0300B4FB0200EF
:10A6D0006C03002010B5024B024A1CF001FE10BDB5
:10A6E0002DA100006DA1000010B51C0002AB1B786D
:10A6F000002907D0002B05D10F4910481BF08EFC14
:10A700000CF055F8A24207D1824213D003000C4945
:10A710000A4801F0D5FDF3E7824205D9121A09492A
:10A72000064801F0CDFDEBE7844203D2030022008E
:10A730000549EDE710BDC0462235030034FD020097
:10A74000BA340300707A0300A27A0300F0B5002542
:10A75000170087B00C9C0D9E039004910593029501
:10A760000195059B9D4208D1019B039A934241D2DA
:10A77000244925481BF052FC26E0039B9D4211D240
:10A7800063689B05F4D4019B049A01330193AB00E9
:10A79000D058FF2263681340012B22D109F004F83E
:10A7A000307015E023680022D900062338001943D1
:10A7B0000AF014FA00280FD16368DB0506D5226879
:10A7C0001249114801F07CFD0BF0F1FFA3683360E2
:10A7D00001350C340436C4E7029B40680133029310
:10A7E000D7E7022B03D108F0A1FE3060F0E7032B7E
:10A7F000EED1FAE73B68029ADB0805499A42B8D3E2
:10A8000007B0F0BDE87A030034FD0200D17A0300FE
:10A81000097B030070B50D0008F0ECFE041C280055
:10A8200008F0E8FE211C10F08FFE051C1BF025F936
:10A83000011C281C10F068FD211C10F0E3F9032313
:10A84000020002209A43024B1043C01870BDC0465C
:10A850000000808010B51BF010F9032302000220D5
:10A860009A43024B1043C01810BDC04600008080C0
:10A87000F8B5070008680D0008F058FE0600012F23
:10A8800006D1002826DDF7F795FA1BF082F9F8BD0E
:10A89000686808F04BFE841B022F06D1864219DA45
:10A8A0002000F7F787FA8019EFE7A86808F03EFE66
:10A8B000051E0ADD2018013829000FF017FF0028B7
:10A8C00008DDF7F777FA6843EDE7002802D0201893
:10A8D0000130F1E702481BF094FB0BF068FFC04623
:10A8E000ACFD020010B5074C002802D00868A04259
:10A8F00003D1F7F77FFA200010BD08F043FEF7F709
:10A900009BFAF8E7D8F5020010B5040008F080FFC4
:10A9100008F00CFE002804DC07481BF072FB0BF06B
:10A9200046FFF7F747FA1BF034F904220100200034
:10A9300008F084FF10BDC04604FA020010B50248BA
:10A940001BF05FFB0BF033FFACFD0200F7B54F4B84
:10A950004F4E504F336000233B707B70BB70FB70D9
:10A960003B71A0238500DB05E022ED180323D20014
:10A97000AB50023B8340A0240093009A464BE40571
:10A98000E25012200FF0D0FCA123009ADB00E2502D
:10A9900028200138C046C046C046C046C046C04612
:10A9A000C046C046C046C046C046C046F1D1E022BF
:10A9B0000C23A221D200AB50384BC900625800983A
:10A9C000024202D1013B002BF8D1A222A024D200E6
:10A9D0001100324BE405A058009D284202D0013BF3
:10A9E000002BF8D1A12000223368C0001A500920A2
:10A9F000585080210224F830C902FF3019502848ED
:10AA00001A5028481C50C120A2248000E40019508C
:10AA1000A44610000721244CA0256646ED05AD593B
:10AA2000009E354201D1013CF6D2002A01D1012518
:10AA30001D600125DD601D000026FC350195AE641A
:10AA4000A0266546F6057659009D2E4216D1019C3A
:10AA5000A46C012C03D18C403D5C2C433C54002958
:10AA600011D10130C0B207310132282AD3D1FA20E6
:10AA7000273A5A6080000FF057FCF7BD661E002C85
:10AA8000E5D03400DCE70139C9B2EDE700900040C1
:10AA90001C0000202B0B00200C05000011270000DB
:10AAA000040500004405000010270000254B13B5E5
:10AAB0001A780400244B002A1CD0244A2449127816
:10AAC000002A12D1234A20001A6008F02FFD012825
:10AAD00012D0200008F02AFD022830D0200008F013
:10AAE00025FD1D4C102808D01C491D481BF096FA66
:10AAF0000BF05DFE1B4AE6E71B4C20000BF070FBE1
:10AB00001A4988420AD020000BF0ACFBA022042195
:10AB10006379D205C133FF339B0099506079FFF709
:10AB200015FF134CA0781BF034F8009020781BF030
:10AB300030F8694601900220FBF708F916BD0D4C6C
:10AB4000DBE7C046290B00201C0000202A0B002058
:10AB5000277B030000A0004068E10200637B030044
:10AB600034FD02000090004078E10200A4220300BE
:10AB70002B0B002088E1020010B510201AF0EBFE2C
:10AB80000400034B08C019F019F8200010BDC0469E
:10AB90004401030070B50C00052804D80FF0FEFC3A
:10ABA00006030E04151E0024200070BD081D19F0B8
:10ABB00036F90E4C0028F7D00D4CF5E7081D19F0BA
:10ABC00054FC012440000443EEE7FFF7D5FF211DAC
:10ABD0000500043019F056F92C00E5E7FFF7CCFF2B
:10ABE000211D0500043019F05DF9F5E710D60200CB
:10ABF00008D6020070B5050083070CD1104B02681F
:10AC00009A4208D1FFF7B8FF0400291D043019F05B
:10AC10002EF9200070BD280008F088FCC0231B0618
:10AC2000984205D180200021C0051AF0A3FFF1E76A
:10AC3000C2178318012053405B001843EAE7C0465F
:10AC40004401030070B544006408051C211C201C4D
:10AC500010F016FE002820D11149201C0FF096FE9E
:10AC6000002814D1281C1BF00FFA002808D0FFF789
:10AC700083FF0400291C043019F01FF8200005E0B0
:10AC8000281C10F015FE01244000204370BD05492A
:10AC9000054801F015FB0BF08AFD04490448F8E76C
:10ACA000FFFF7F7FD27B0300F0FB0200EB7B030002
:10ACB000ACFD020007B5C30701D540100EBD04303E
:10ACC00001A9F7F71FFD002801D00198F6E7034915
:10ACD00003481BF0A3F90BF06AFDC046A57B0300F7
:10ACE000F0FB02000123F0B58DB006000C000092CD
:10ACF0000B402ED04B10022202A903A818F09CFF93
:10AD000003AD009BDB072ED5009B02225B1002A93E
:10AD100003A818F091FF03AC092E01D0162E3ED1E6
:10AD2000200019F07CF8002867D1280019F0F3FB07
:10AD3000051C200019F0EFFB011C281C10F0F4F892
:10AD40000323020002209A438D4B1043C0180DB01C
:10AD5000F0BD0320084000D007E18A4B0A689A4200
:10AD6000F5D10D1DCDE70323009A1A4208D10099B1
:10AD7000844A09680191914202D1009B1C1DCBE7D6
:10AD8000009A1340022B04D17F4B1340062B00D0B6
:10AD9000EDE0009A2100300001F06EFDD7E7182E9B
:10ADA00000D9BAE0FFF7E8FE070030000FF0F6FB2D
:10ADB0006E74687A7A0D131A20DD4D8E946E746865
:10ADC0007A7A0D131A20DD4D8E0022002900381DDD
:10ADD00019F0FFF804E0381D2200290019F033F9BA
:10ADE0003800B4E7381D2200290019F079FAF7E796
:10ADF000200019F014F8002805D0644964481BF0BD
:10AE00000DF90BF0D4FC06A83E1D18F0D7FE230068
:10AE10002A0006A93000F7F709FB2B782278534067
:10AE2000DB070ED506A818F0FAFF002809D101218A
:10AE300009A8494218F0F6FE09AA3100300019F0BD
:10AE4000C8F806A818F0C6FECAE7200018F0E7FF09
:10AE50000028D2D109A83E1D18F0B0FE23002A0018
:10AE6000310009A8F7F7E2FA09A818F0B3FE2B7829
:10AE700022785340DB07B3D5220031003000A7E72A
:10AE8000381D2200290019F026F9A9E7381D2200F3
:10AE9000290019F0A2F9A3E7381D22002900F7F7CD
:10AEA00051FA9DE70098FFF705FF021E02DA3949C3
:10AEB0003948A4E7381D2900032E01D0102E02D1F5
:10AEC000F7F7D4F98CE719F024F889E7381D220048
:10AED000290019F088FA83E7200018F0A0FF002865
:10AEE0008BD1FFF749FE3E1D009023002A0004305D
:10AEF0003100F7F79BFA2B7822785340DB0704D513
:10AF000022003100300019F064F8009B09A90220EA
:10AF100009930A97FAF71AFF19E72100280018F099
:10AF200083FF193E03000020042E00D90FE73000F4
:10AF30000FF034FB0309160D12001848002B00DB3C
:10AF400005E7174803E71548002BFADCFFE613482E
:10AF5000002B00DDFBE6F4E71048002BF1DAF6E603
:10AF60000E48002B00D0F2E6EBE70020EFE62800C9
:10AF700019F0D1FA009A011C300006F001F9E6E65A
:10AF80000000808044010300070080FF7F7B0300F6
:10AF9000F4FD0200907B0300ACFD020008D6020025
:10AFA00010D6020010B54A6801491EF0CEF910BD56
:10AFB000047C030070B5150012680C008368002A39
:10AFC0000AD1CC000621181D214309F007FE0028F4
:10AFD00001D043682B6070BD1A79180092070BD519
:10AFE0000C4A9342F7D10C4E736C002B03D1012015
:10AFF00018F085FC7064706C06216A68E4002143D7
:10B00000002A03D118F0BDFC0023E3E718F0AFFCE1
:10B01000FAE7C046D0C50200C4090020F8B50625ED
:10B02000C3001D430700012229000C4809F0D6FD8A
:10B0300006004068002810D10C301AF08CFC084B38
:10B04000040003604760012018F059FC2A00A0604A
:10B050006E2118F08CFC20007460F8BDE809002017
:10B0600028F2020010B503210148F6F70BFE10BDCF
:10B07000E409002010B50C000621C00001430122A4
:10B08000024809F0ABFD446010BDC046E80900204D
:10B0900073B50625C3001D430600002229000F4892
:10B0A00009F09CFD041E17D1020029000C4809F08C
:10B0B00095FD041E11D06A460821406804F0A4F9E9
:10B0C000009B002B08D000216A4608001CF0CCF938
:10B0D00061683000FFF7CEFF606876BDE8090020A8
:10B0E00054F10200034B04481B78002B00D10348A5
:10B0F0007047C04600C0020010D6020008D6020009
:10B1000010B5DA201AF027FC00230370024B8C33B1
:10B110001860024810BDC046C4090020D8F50200DE
:10B12000F0B507000E001500094C87B02000019310
:10B130001AF0A6F802AB1F70019B102202A9200092
:10B14000039604950593FBF751FC07B0F0BDC0468C
:10B1500000C00200F0B5784B99B08C331A680192A8
:10B16000002A02D1002019B0F0BD00241C60019B10
:10B170001B78A342F6D00126019B704F0233109337
:10B18000019B109DD233119302933B002341334224
:10B1900011D01A2302991B1B280003931AF07FFD7C
:10B1A000BB235B00984206DC3300A34032009F4380
:10B1B000039B9A409743029B0134083B0835029356
:10B1C0000D2CE2D10A23089300230293029812F077
:10B1D00075F9089B12901391013B089314AA39004A
:10B1E0000198002B00D188E000261AF026FD109B64
:10B1F0000E93119B0D93524B0F931A239B1B0B9392
:10B200000E9B09960C930D9B0A934D4B04930C9B3C
:10B210004B4C07930B9B16AD05930A9B0693099B1A
:10B2200003933B00039A13410122134225D014AB30
:10B230000F9A1B882900D3182B8014AB5B88049AC3
:10B240000798D3186B8014AB9B8814AAE318AB80C3
:10B250001AF054FD011C02980FF098FB002862D1EF
:10B2600014AA290006981AF049FD8022029B1206B2
:10B2700099180FF08BFB002855D1039B01330393E2
:10B28000069B083B0693059B013B0593FA23DB00D5
:10B29000E418079BA4B208330793FA231B019C42CE
:10B2A000BFD1FA22D2009446099B033309930A9B2B
:10B2B000183B0A930B9B033B0B930C9B18330C938B
:10B2C000049B63449BB20493A342A0D10D9B093617
:10B2D000483B0D930E9B48330E930F9B63449BB2E8
:10B2E0000F931B2E89D112981399164A164B10F002
:10B2F00095FB12F035F9029068E71AF09EFC040005
:10B3000014AB04229B5E14AA0221525E14A90020F1
:10B31000095E1B01120109010120FFF701FF200056
:10B320001AF037FC1FE70122059B03999A4001237D
:10B330008B4013439F43A0E7C4090020FFDFFF07B2
:10B3400030F800009A9999999999B93FF0B5584CFD
:10B350008BB00390A37F002B05D1564956481AF0B5
:10B360005DFE0BF024FA0398FFF7CAFE0022534952
:10B3700020001AF082FD00F0ADFB00280BD05048F1
:10B3800001F0CCF8002804D14E4801F0C7F800289D
:10B39000F1D000F037FD20201BF008FF002307004C
:10B3A000190007AA995401330C2BFBD10224002366
:10B3B00025000293019306AB05AA04A9424819F09F
:10B3C0005CFD00232200290038001BF017FC049BC1
:10B3D0003E4A002593420CDB19000135C83108DBD9
:10B3E000C821033589008B4203DC013DC82B00DCFA
:10B3F000013D059B002493420CDB1A000134C83246
:10B4000008DBC82203349200934203DC013CC82BC2
:10B4100000DC013C0422029B134205D109232200D7
:10B42000290038001BF0EAFB0023294E0093009A04
:10B4300007ABD25C002A2AD0092372783178380011
:10B440001BF0DCFB009B0236013300930C2BEED18A
:10B45000174E390030001AF0B3FC6420FCF706FAEE
:10B46000029B01330293019B0B2BA4DD1949300091
:10B470001AF0A6FCFA208000FCF7F8F90398FFF711
:10B4800069FE040000F0BEFC20000BB0F0BD327875
:10B49000AA42D7D17278A242D4D10121009AD154C4
:10B4A000019B22000133019329000923C7E7C0460D
:10B4B000240000202A7C03002CFC0200567C0300A0
:10B4C000D0FE0200DCFE0200F4D90200E0FCFFFF27
:10B4D000127C03000C000300002310B518001A00B2
:10B4E0001900FFF71DFE014810BDC046D8F5020047
:10B4F00070B500210320FAF729FC084D04006868A4
:10B500001AF047FBA060A8681AF043FBE060E86807
:10B510001AF03FFB2061200070BDC04600C0020051
:10B5200070B548680C0008F001F80500A06807F045
:10B53000FDFF0600E06807F0F9FF32000300290074
:10B540000120FFF7EDFD014870BDC046D8F50200AF
:10B55000F8B50B4E3378002B10D10A4D2C78E4B29D
:10B56000002C0BD1012700682F7003685B68984797
:10B57000054A2C7013683770DB191360F8BDC0469C
:10B58000730900207409002070030020F0B53E4BC1
:10B5900087B01B780400002B01D1FFF7D7FE201DD8
:10B5A000FFF7D6FF394D28000DF0BCFE0021606882
:10B5B0001EF0D1FB344E049073680021606805933F
:10B5C0001EF0D6FBB36800210290606803931EF062
:10B5D000DCFBF368C01A10F08BF9041C28001FF084
:10B5E000C2FB061C28001FF0B5FB051C301C12F026
:10B5F00057FB071C301C12F0CFF90190281C12F0E9
:10B600004FFB061C281C12F0C7F9029B039A051C6D
:10B61000981A10F06DF9291C0FF076FE311C051CEC
:10B62000201C0FF071FE011C281C0FF0EBFA802388
:10B630001B06059AC518049B981A10F059F9019930
:10B640000FF062FE211C061C381C0FF05DFE011C71
:10B65000301C0FF0D7FA80231B06C018291C12F0EB
:10B660008FFC0B490FF050FE11F028FF094A0A4BDE
:10B6700010F0E4FC11F0ACFE002801DA6930FF3074
:10B680001AF087FA07B0F0BD00C00200BC06002027
:10B690000000B443EA2E4454FB21194010B50400C5
:10B6A0000430FFF755FF002160681EF06EFB034B6E
:10B6B000DB68C01A1AF06DFA10BDC04600C0020067
:10B6C00010B504000430FFF743FF002160681EF04E
:10B6D00042FB034B5B68C01A1AF05BFA10BDC04610
:10B6E00000C0020010B504000430FFF731FF002154
:10B6F00060681EF03DFB034B9B68C01A1AF049FAC4
:10B7000010BDC04600C0020070B500210500032036
:10B71000FAF71CFB0400281DFFF71AFF00216868D8
:10B720001EF019FB0C4E7368C01A1AF032FAA060B2
:10B73000002168681EF01CFBB368C01A1AF029FAD1
:10B74000E060002168681EF020FBF368C01A1AF060
:10B7500020FA2061200070BD00C00200F0B54C4B03
:10B7600089B08C331B680293002B4CD049480430BD
:10B77000FFF7EEFE484C002120001EF0ECFA0021FD
:10B780000311200003931EF0F3FA0021031120009F
:10B7900001931EF0FAFA03110493029B039A1B789B
:10B7A0005242002B31D1019B0321D31A9C464942BE
:10B7B0000800654609380124032664420319029FE4
:10B7C000DB00FB186A461F0092896A373A806A4696
:10B7D000928870337A806A46128A013EBA80049F4A
:10B7E00067437F191F800134002EE7D1019B03308E
:10B7F000ED188142DFD1039B09319C441829D7D130
:10B800000123029A137009B0F0BD019BD71A0322DD
:10B810005242110005970939012003264042049C39
:10B82000059B4443E3180693029C0B18DB00E318C6
:10B830001C00703407940025645FA446069C644590
:10B8400015DD6A24A4466D469C446446AD89258076
:10B850006C24A4466D469C446446AD886E332580B6
:10B860006C46248A1C806C46079B248B1C80013EFE
:10B870000130002ED3D10598019B0331C3180593E5
:10B880008A42C9D1039B0932FF18182AC1D1BAE7ED
:10B89000C4090020B4F30200F8060020F8B5050042
:10B8A00010200C0016001F001AF062F8011E09D0CB
:10B8B00044608460A4190760C460034B034A2800F5
:10B8C0001BF00EFDF8BDC046A95D0200935D0200AD
:10B8D00010B5034A034904481DF037FD034810BD65
:10B8E0003C7D0300F2BC03008C220300D8F502006B
:10B8F00010B5034A034904481DF027FD034810BD55
:10B90000647C0300F2BC03008C220300D8F5020023
:10B910000023FA21084A89001360084A1370084A74
:10B920001360084A1160084A1370084AD366136707
:10B930000122074B1A707047780300207509002018
:10B94000740300202000002076090020C409002094
:10B950007709002010B5084B084A1978002907D14B
:10B96000116B002902D0FFF7D3FF10BD30BFF4E701
:10B9700000221A70F9E7C04677090020C4090020A8
:10B98000837F0248002B00D10148704710D6020087
:10B9900008D60200A02010B50F49C0054B7F5A1CE5
:10B9A000002B09D14C8C0D4BA3430D4C03510D4B77
:10B9B0004A775200D05A0DE010335B00CB185C88F8
:10B9C000A123DB00C450092AF1D10120F5F7E8FEDC
:10B9D0000120404210BDC04624000020F01F00009E
:10B9E0000C050000F63303000023E021A02210B56F
:10B9F00083770C4B0902D205D1500B480AF01CFC8E
:10BA00000A480AF019FC0A480AF016FC09480AF02C
:10BA100013FC09480AF010FC08480AF00DFC08481D
:10BA200010BDC0460C05000090E1020098E1020044
:10BA3000A8E10200B0E10200C0E1020038E102002A
:10BA4000D8F5020073B5041E09D1194D2B78002BCF
:10BA50002BD0184918481AF0B3F92C7073BD174E43
:10BA6000F56E07F07BFC164B2100984214D0154B65
:10BA70002340062B05D0A30712D1134B22689A420C
:10BA80000ED101A92000FDF77DFC019B012B0CD1FB
:10BA900000781BF08BFB010028001AF091F9DDE71C
:10BAA0000A490B481AF0BAFA3063FFF731FFD5E7BD
:10BAB000760900205C05030024000020C409002052
:10BAC000DC050300070080FF08180300B67E0300B2
:10BAD00034FD0200034B1878013843425841C0B28C
:10BAE0007047C04675090020F7B5A123A024224A5B
:10BAF000E405DB00E250C37F012219000D318A40CA
:10BB000001331E49DBB262500191032B31D0C37760
:10BB100002000300002122333632198002339A4298
:10BB2000FBD1C47F164A63000133D31805220425D4
:10BB30009446012167465A1E12781E787A43114FA7
:10BB40000633BA180F00AF4092191279013552002E
:10BB50008218568C3E4356840D2DEBD10D34A02314
:10BB6000A122A140DB05D2009950828E01995A5042
:10BB7000F7BD0023CBE7C046F01F00000C05000016
:10BB8000807E03002400002070B5304D8CB0AB7F68
:10BB9000002B1FD02800FFF7A7FF2D4A2D4913685F
:10BBA0000968063313608B4207D300242A4B1460C4
:10BBB0001B78012B10D0022B43D000232A8C6B77EB
:10BBC000FF33FF331A4205D0E1222449D20001207D
:10BBD000F5F7B2FD0CB070BD214EF36E002B02D014
:10BBE000336F002B02D1FFF793FEE6E708F02EFD3E
:10BBF00068460AF0C1FD00280CD11A4B186803F002
:10BC0000A5FC04000AF0CEFD08F02AFD2000FFF795
:10BC100019FFD2E708F024FD019B13491868FCF7CF
:10BC2000EBF90028F2D1019807F098FB0F4B9842EE
:10BC300003D10F490F481DF088FB019B002433639B
:10BC4000E4E70D4928001AF0BBF8CCE724000020F7
:10BC500074030020200000207509002095B9000021
:10BC6000C40900207803002074FC020000FB0200DD
:10BC70004F6403008C2203005C050300F7B5002429
:10BC8000009308AB124D1B780600080017000193C3
:10BC9000EC662C6703F034FC6A460E4B1278186091
:10BCA0000D4BEE661F600D4B28671A700C4B1C7015
:10BCB00003F04CFCFFF7C6FE01220A4B1C600A4B46
:10BCC0001A70019BA34201D0FFF744FEF7BDC046A6
:10BCD000C4090020780300202000002076090020FD
:10BCE000770900207403002075090020F0B50024B6
:10BCF0002B4B8DB0DC661C672A4B07AC40C9013862
:10BD0000009301940523FEF721FD079863680590D1
:10BD10000293237B257A0393234B277C0340062B36
:10BD200005D083072ED1214B02689A422AD106A959
:10BD3000FDF728FB069B002B21D0012B0CD1002DF9
:10BD40000AD1002F08D100781BF030FA0590059930
:10BD500030001AF035F812E0059801F019FB059053
:10BD6000237C002B03D00598F9F71CFB0590039B5F
:10BD7000029A009305992B003000FFF77FFF0C48D3
:10BD80000DB0F0BD07F0EAFA0A4B9842E8D1002D59
:10BD900001D1002FDBD005A90120F9F7D7FFDEE79D
:10BDA000C409002094F40200070080FF0818030073
:10BDB000D8F50200DC05030030B5104B89B003ACA8
:10BDC00020C90138009301940523FEF7BFFC02A9A6
:10BDD0000398FDF7D7FA227C237B02990092039AFD
:10BDE00001F0C0FA237A0100009328000023626862
:10BDF000FFF744FF024809B030BDC046D0F402004E
:10BE0000D8F502000022074B10B51A70064B02321B
:10BE10001A70064B064A1B68063B1360FFF79AFD33
:10BE200010BDC046770900207509002020000020C1
:10BE30007403002010B5FFF7E5FF014810BDC046B0
:10BE4000D8F5020010B5042901D8042A05D90A49F9
:10BE50000A481AF0E3F80AF0AAFC092B01D90849AC
:10BE6000F6E70524614341188A18137101229A40AC
:10BE7000038C1343038410BDC47E0300ACFD020099
:10BE8000D97E0300F8B548680C000D6807F04EFB3A
:10BE90000600A06807F04AFB0700E06807F046FBD1
:10BEA0003A00030031002800FFF7CCFF0048F8BD3E
:10BEB000D8F5020010B5042901D8042A05D906498D
:10BEC00006481AF0ABF80AF072FC052359434018F3
:10BED0008018007910BDC046C47E0300ACFD02008E
:10BEE000F7B51B4F019038000AF098F9194E300051
:10BEF0000AF094F9184D28000AF090F917480AF052
:10BF00008DF917480AF08AF916480AF087F9164C95
:10BF1000380021000AF0A6F9300021000AF0A2F949
:10BF2000280021000AF09EF921000C480AF09AF935
:10BF300021000B480AF096F921000A480AF092F90C
:10BF400019F0C5FF0123019A08489377FEBDC0464A
:10BF500090E1020098E10200A8E10200B0E10200D5
:10BF6000C0E1020038E10200B4220300D8F502006B
:10BF700030B58DB0050068460AF0FEFB011E10D1F9
:10BF80002A1D01201BF070FA0122EB6804005B10EF
:10BF900001335B001343EB600AF004FC20000DB09A
:10BFA00030BD0198054A0368934205D0044A002435
:10BFB0009342F3D00AF0FBFB0024EFE774FC02008D
:10BFC00004FA020010B50400102019F0C4FC044B60
:10BFD000036023684360636883600123C36010BD0E
:10BFE0009CF50200054B002805D00023022802D151
:10BFF000012349000B4318007047C04608D60200D1
:10C0000010B502491DF0D6F810BDC0464A8603009F
:10C01000F7B5019111490400170000251DF0CAF879
:10C020007B689D4204D30E4920001DF0C3F8F7BD84
:10C03000002D03D00B4920001DF0BCF8019BAE0081
:10C040009A5909492000BE191DF07FF90122B168F3
:10C05000200007F09BF90135E2E7C046F6A7030090
:10C060002FA7030083380300F37E030030B50724B5
:10C070000278084DA24314000222224302707F225C
:10C08000039C41602240D400028883602A402243FE
:10C09000028030BD07FCFFFF10B50B0007240178BC
:10C0A0002340A14319437F23017004990A4C0B409C
:10C0B000D9000388426023400B430380039B04683C
:10C0C0005905064BC90A23400B430360029B83605A
:10C0D000059BC36010BDC04607FCFFFFFF03E0FFE8
:10C0E000C3790248002B00D10148704710D60200E6
:10C0F00008D6020010B5FEF719F8014810BDC04679
:10C10000D8F5020010B50868FEF710F8004810BD19
:10C11000D8F5020073B50D00022838D1012601A917
:10C120006868FDF72FF976423400019BC3188342FB
:10C1300011D101A92868FDF725F9734273416242C4
:10C140006241DBB2D2B20199FEF73CF9002822D15C
:10C150001149124817E00278722A01D0772A06D1D5
:10C16000611C0ED1723A544254410130DFE7622A19
:10C1700001D0742A05D1711C03D1743A564256413C
:10C18000F3E70749074819F049FF0AF010FB0126B9
:10C1900076423400CDE776BD617A0300B4FB02003D
:10C1A000F77E0300ACFD0200F7B50D001100002280
:10C1B0000600009228001F000B4BFEF795FA102096
:10C1C00019F0D6FB041E08D1084A094B094CDA6164
:10C1D000002326602000A360FEBD39002800F9F787
:10C1E000B5FDE060F4E7C046FFFF000094DC02000C
:10C1F000C4090020D409002010B5013810C9F9F78E
:10C20000A5FDE060004810BDD8F50200F8B57F2517
:10C2100053B204000E0017001540002B0ADB6B1E02
:10C22000012B07D80B6858681BF005F801002000A7
:10C230001CF0C0FF022D0ED10F4920001CF0BAFFE8
:10C24000F368002B02D05A68002A0CD10B49200059
:10C250001CF0B0FFF8BD002DF2D03A00F1682000CC
:10C26000F9F708FDF6E7012AF7D1002299682000C6
:10C2700007F08CF8EEE7C04642690300C66503008C
:10C28000C36803485A68002A00D098687047C046BF
:10C29000D8F50200136810B51400002B03D17D29D6
:10C2A00002D1C368136010BD044B02689A42FAD1F0
:10C2B000BA29F8D1FFF7E4FF2060F4E774FC02002C
:10C2C0000EB470B5050087B0102019F051FB041EA4
:10C2D0000BD11B4B1B4A1C4C1D619861DA6120007D
:10C2E00007B070BC08BC03B018470021056081602E
:10C2F0000120F9F72BFD0B9B0500E060002BEED031
:10C30000252118001FF060FC061E09D10B981FF0B4
:10C3100073FC320001000B98FCF786FBA860DEE797
:10C3200002A810211BF04AF90CAA0B9902A801924D
:10C3300004F00EFB02A90548E568FCF73FFBEDE7BA
:10C34000C409002094DC0200D4090020081803006E
:10C3500010B50300820708D1064A0168914204D152
:10C36000054AD9680120914203D004491800FBF71F
:10C3700043FE10BD8CE40200A9C1000084F8020055
:10C3800010B5040006F0EAFF044AC1682300914298
:10C3900000D0236900229A6010BDC046A9C10000E8
:10C3A000F7B50500160001930F0006F0D7FF174BF5
:10C3B000C2682C009A4200D02C69A568002D13D1C8
:10C3C0000C2019F0D5FAA06000280CD00323E580DA
:10C3D000A380E288A16893000332E280019ACB181F
:10C3E0001F605E609A60F7BDE388A18802338B42CC
:10C3F000EFDB033189000122280019F0CFFA002871
:10C40000F1D0A388A0600333A380E2E7A9C10000B4
:10C4100070B506000D00140006F0A0FF074BC168C0
:10C420003200994200D032699368002B02D12B6010
:10C43000236070BDD2882A60FAE7C046A9C1000017
:10C4400010B50400082019F086FA024B446003601E
:10C4500010BDC04630FE020010B50124037A054924
:10C460009B005A580448224200D10448A243CA50B3
:10C4700010BDC0467C03002010D6020008D6020082
:10C4800070B5037A064C05009B001859400819F056
:10C4900080FB01222B7A9B0019590A401A5170BD6A
:10C4A0007C03002070B5A222A025D200ED05AA5879
:10C4B0000723CA401100174C0340E056421EC9072B
:10C4C00000D5421C022A0BDC00218A421CDB124DE3
:10C4D000EE5C30008E4201D00220E954E25470BD7F
:10C4E000072A09DD0C2A12DC0B490320CD5C002D44
:10C4F000F4D10238C854F1E707490320C95C4D1E46
:10C50000A94149420840E9E70A000800E6E703209C
:10C510000C22E3E77B02002073020020072243681D
:10C5200001201B791340024AD35C58407047C04633
:10C530007302002010B5FFF7F1FF034B002800D174
:10C54000024B180010BDC04610D6020008D60200EB
:10C550001D4B70B559791879FFF7A4FF022805D152
:10C560001A490B689A1C012313430B60184B597925
:10C570001879FFF797FF022805D114494B689A1CD8
:10C58000012313434B60134C200009F029FE124D88
:10C59000A84203D161792079FFF784FF0F4C200076
:10C5A00009F01EFEA84203D161792079FFF77AFFD6
:10C5B0000B4C200009F014FEA84203D161792079C8
:10C5C000FFF770FF70BDC046A0E102007C030020B1
:10C5D00040E1020030E10200D422030078E10200D1
:10C5E00088E10200072203791340014AD05C7047BA
:10C5F000730200207FB54B680E005C102100684676
:10C600001AF0F3FF029D0021220028001FF08EF98E
:10C6100001213068014009D12B00220019F090FA65
:10C6200069460748FCF7CAF904B070BD4310200002
:10C63000042C00D904202A0000211CF02AFDEFE779
:10C6400040EE0200F0B50C00002585B0110020007E
:10C650001E00009502232A00FEF746F80120AC4296
:10C660002BD0844231D13068204226D103230340AD
:10C67000AB4203D11C4A016891421ED01B4A0240C2
:10C68000062A06D0002B0DD10268194B92699A42F6
:10C6900008D103A9FCF776FE00231A00039909F0DC
:10C6A00007FE0AE0032302001A40022A07D1FF22F4
:10C6B000D20580189843FEF7C5FA05B0F0BD06F024
:10C6C00035FF012340001843F7E703A93068FCF762
:10C6D00059FE04007068039F06F028FF2B0002003B
:10C6E00039002000DBE7C04644010300070080FF5B
:10C6F0003D990000F0B58DB00A9214AA1278050099
:10C700000B9215AA12780E000792DA0700D494E073
:10C71000180006F00BFF002305900693002803DAAB
:10C72000434205932D230693129B0027023B1E2BA9
:10C7300016D84F4B129A2020995C0DF04DFF079BA5
:10C74000C4B2BB4204D0601C03210DF045FF0700BA
:10C750001398002801D01FF04FFA0334E7193F184F
:10C760003368BB4204D2380019F0F5F8286037600E
:10C7700000222C68E619731E1A70059A002A2CD024
:10C78000099308930B9B0A3B0B93059812990EF0A3
:10C7900093F80E00059812990DF0A8FF330005904C
:10C7A0003033092E01DD0B9B9B19089A561E3370FE
:10C7B000079B002B30D0059B002B11D0B4420FD229
:10C7C000099B9B1B032B06D16B461B7F013E3370DD
:10C7D000B44205D209960896D7E73023023E33705B
:10C7E000139B002B06D018001FF006FA0023301A06
:10C7F000844219D3069B002B05D0B44203D26B466A
:10C800001B7E013E33702B68DF19BF1B0A9B013F63
:10C810001F6030000DB0F0BDB442E1D2059B002B8B
:10C82000D9D1DDE7C2540133139AD25C002AF9D181
:10C83000069B0600002BE2D1E5E79A0711D10D4ACD
:10C84000196891420DD1079A310003920B9A029216
:10C85000139A0192129A00920A9A19F048F9060066
:10C86000D7E700232A6813700A9A2E681360D0E76E
:10C87000047F0300440103001300144A10B50400B0
:10C88000934204D10122200002F0C6FE10BD104ADE
:10C89000934201D10322F6E70020072CF6D10D4A7E
:10C8A0001A40062A0ED09A07F0D11A680A4CA24202
:10C8B00008D00A4CA24205D0094CA24202D0094C31
:10C8C000A242E3D10A0007201900DDE708D60200E2
:10C8D00010D60200070080FF0818030040EE020097
:10C8E0009CDC020004D4020070B51500040019F0AD
:10C8F000F2FC2A000249200019F099FC70BDC046E4
:10C90000B562020070B543790D000024032B06D9EF
:10C91000836A074C9200E41AC369D358E4180321D0
:10C9200019F0C8FC447024120570847070BDC046B4
:10C93000FD7F0000F7B500230400617183608371FF
:10C94000E260036101330F0015004361032906D83B
:10C950000121836949429A00C0691EF0E7FF002364
:10C96000A36223622A8C6B8CD218002A00D1013278
:10C97000384E2000310019F05AFCAA8C31002000FA
:10C9800019F055FCE3682000197E19F08CFCE3686F
:10C990002000997E19F087FCE3682000197F19F0C8
:10C9A00082FCE3682000997F19F07DFC042F27D1D9
:10C9B000636A226A31009A1A200019F038FC3100AB
:10C9C0002A69200019F033FC3100EA68200019F0D0
:10C9D0002EFC00262B8D9E4217DBFF21200019F034
:10C9E0007AFC042F35D16A8BAB8B0237D3180093B6
:10C9F0000023009A93422CD02A8D0021019223E03B
:10CA00000221200019F041FCD9E7EA6AF300D318AB
:10CA10001A78032A03D19978200019F05CFC0136BA
:10CA2000D8E70126E86ACA008218507830420AD056
:10CA30005088834207D15268D200606B99003A4314
:10CA40000A500133D5E70131019A9142E9DB022214
:10CA5000F2E7F7BD8B62020013B543790400012BA6
:10CA600020D08268002A03D0164917481CF06DFCBC
:10CA70000021200019F017FC6379032B13D1226ADF
:10CA8000D01C9843A36A20626062E362C01818F069
:10CA900074FFE3682063588B9B8BC018800018F0EC
:10CAA0006CFF606313BD042BFCD1E068636AE26A2B
:10CAB000216B9A18037E00934069636BFFF7D6FAE7
:10CAC000F0E7C046257F03008C220300F7B5224B18
:10CAD0000600A8331B680191022B0DD844698C42D3
:10CAE0000AD2836A02690C1B9D1A23002B4304D1CE
:10CAF000B36A3361019B7361F7BD0095062C13D8AF
:10CB00001F2D01D91F2300932700032C00D90327D1
:10CB10000121300019F0B9FB009A7B011343037027
:10CB2000009BE41BED1AE0E70F2D01D90F230093C2
:10CB30000A4B27009C4200D91F000221300019F047
:10CB4000A4FB70223B0900991340F03A0A431343B7
:10CB500003704770E4E7C046C4090020FF070000E7
:10CB600070B50D000121040019F081FB0F2D14D0C8
:10CB7000102D17D010210E2D10D01721200019F0E4
:10CB8000AAFB0322A36A042103339343A362200078
:10CB900019F090FB044B036003E01121200019F011
:10CBA0009AFB70BD1221F9E74CDB0200F8B50500D5
:10CBB0000C00171E124E11D1110019F058FB8023E2
:10CBC0001B021C4203D03221280019F084FB2200F2
:10CBD000352132402800FFF795FEF8BD32000A40AB
:10CBE0004621FFF78FFE80231B021C4021004C1EB4
:10CBF000A141C9013943C9B2280019F06CFBECE727
:10CC0000FF7FFFFFA3230021024A5B000248D152AD
:10CC10007047C046C4090020D8F50200A3230121B3
:10CC2000024A5B000248D1527047C046C409002046
:10CC3000D8F50200A323044A5B00D35A0348002B13
:10CC400000D103487047C046C409002010D6020036
:10CC500008D6020010B5F9F773FC014810BDC046B4
:10CC6000D8F502000300203B5E2B00D93F200523AE
:10CC700020384343014A1068C018704774000020F0
:10CC800070B50500080068430130401008300C0002
:10CC900018F061FE0122044B857103600379447131
:10CCA0009343037170BDC046DC05030010B504005A
:10CCB000102018F050FE044B036063684360A368C3
:10CCC000C3600023836010BDB002030070B505008F
:10CCD000202018F040FE05210B4B040003600800E3
:10CCE000FFF7CEFF6B68EA68A060236162602A7C70
:10CCF0002000A276AA689B1863616B7CE37619F02A
:10CD000042FF200070BDC04624060300037910B521
:10CD1000DB0705D50349044819F080F909F047FD00
:10CD200010BDC046517F030034FD020070B50D00F8
:10CD30000400FFF7EBFF280006F0F8FB01000928CC
:10CD400005D90549054819F069F909F030FD2000B9
:10CD500019F07BFF024870BDD97E0300ACFD0200D4
:10CD6000D8F50200F0B50C000B6889B00700180078
:10CD70000493FFF7CBFF6568280006F0EFFA1F4B1E
:10CD80001F49984202D1072F05D11E491E4819F0AC
:10CD900045F909F00CFDA06806F0C8FB0690E068B4
:10CDA00006F0C4FB0790206906F0C0FB059060699F
:10CDB00006F0BCFB059B0600002B01DB002802DA15
:10CDC00012491348E3E7062F14D0A06906F0AEFB22
:10CDD0000700E06906F0AAFB059B0390009328007A
:10CDE00002970196079B069A049919F0DFFF0948FC
:10CDF00009B0F0BD00200700EEE7C046DC050300E7
:10CE00007E7F0300917F030034FD0200AB7F0300AF
:10CE1000ACFD0200D8F5020070B504000800160051
:10CE200006F084FB0500300006F080FB0600002DB4
:10CE300001DB002805DA0D490D4819F0EFF809F07B
:10CE4000B6FC200019F09DFF854204DA200019F09D
:10CE5000A6FF864201DB0749EEE7320029002000E9
:10CE600019F081FF43000120184370BDEF7F0300DC
:10CE7000ACFD020008800300F8B50D000C6820002E
:10CE8000FFF744FF686806F051FB0600A86806F04B
:10CE90004DFB0700002E01DB002805DA1049114880
:10CEA00019F0BCF809F083FCE86806F03FFB0500C8
:10CEB000092801D90C49F2E7200019F062FF8642E7
:10CEC00004DA200019F06BFF874201DB0749E6E72F
:10CED0002B003A003100200019F090FE0448F8BD04
:10CEE000EF7F0300ACFD0200D97E03000880030041
:10CEF000D8F50200F7B50E002649040001921CF097
:10CF000024FA019B002B03D1234920001CF01DFAB9
:10CF1000224920001CF019FA0025300019F03FFFCB
:10CF2000854221DA0027300019F02BFF87420CDA06
:10CF300039002A00300019F016FF194B19491A5C04
:10CF400020001CF002FA0137EDE7174920001CF021
:10CF5000FCF9019B002B05D1300019F020FF0138AE
:10CF6000854211DB0135D8E70C4920001CF0EDF9B2
:10CF7000019B002B03D10D4920001CF0E6F90C4960
:10CF800020001CF0E2F9F7BD0A4920001CF0DDF991
:10CF9000E8E7C046978003009E800300AC80030052
:10CFA000AE80030082790300A4800300B36603000F
:10CFB0002FA70300A6800300F0B50F001100002288
:10CFC0008BB01E00009203233800FDF78DFB032F6A
:10CFD00000D9D5E038000DF0E1FA020C9494052157
:10CFE0000800FFF74DFE040019F03DFE20000BB0D5
:10CFF000F0BD3068654B0340062B07D0830700D097
:10D00000C1E0634B02689A4200D0BCE007A9FCF77C
:10D01000B9F9079B03900593012B04D1039B187862
:10D020001AF0C4F8E3E700231E00039A0293039961
:10D030000598511A814218DA11780A2901D03A2943
:10D0400008D19E4200DA1E00029B013302930023A6
:10D050000132ECE701332029FAD03929F8DD4D49B6
:10D060004D4818F0DBFF09F0A2FB002B05D0029A17
:10D07000013202929E4200DA1E0002993000FFF750
:10D08000FFFD002507002C00039B0493039A049BDB
:10D090009B1A059A9A4223DD049B1B780A2B01D028
:10D0A0003A2B0FD1A64207DD210000232A003800C9
:10D0B00019F0A4FD0134F5E700240135049B013388
:10D0C0000493E3E7202B07D1002321002A00380036
:10D0D00019F094FD0134F1E7392BEFDC303BF4E734
:10D0E000029B3800AB4200DC81E7A64207DD21004D
:10D0F00000232A00380019F081FD0134F5E73800DB
:10D1000075E7306806F012FA0500706806F00EFA4E
:10D11000029001002800FFF7B3FD0390022F03D116
:10D1200019F0A1FD039862E7012207A9B06806F093
:10D13000B7FB002D1FDB029B002B1CDB6B43089A07
:10D14000934218D100242700029B9C42EAD03E0063
:10D15000EB190493049BF11B9E420ED0079B9A5D32
:10D16000131C092A00D90923DBB22200039819F005
:10D1700045FD0136EEE7094972E77F190134E3E71F
:10D18000074908486DE70849FBE7C046070080FFEC
:10D190000818030018800300ACFD02004280030061
:10D1A0005F80030034FD02007E800300F0B585B08F
:10D1B00001910500002101980DF0D4FB041E05D05B
:10D1C0002349244818F02AFF09F0F1FA280019F041
:10D1D000D8FD0600280019F0E2FD01003000FFF73D
:10D1E0004FFD0700280019F0CCFD84422CDA002600
:10D1F000280019F0C6FD864224DA320021002800FA
:10D2000019F0B1FD0EF074FB01990EF07DF810F0ED
:10D2100055F90022104B0EF001FC104B0022029039
:10D2200003910DF065FB0923002804D002980399AF
:10D2300010F0CEF8030032002100380019F0DEFCB7
:10D240000136D5E70134CDE7380005B0F0BDC04662
:10D25000C37F0300ACFD02000000E03F000022405D
:10D26000F0B587B007000391059219F098FD04000E
:10D27000380019F086FD0190039819F090FD844262
:10D280002DD121000198FFF7FBFC0025029006E05C
:10D29000049B1B1ADA43D217134019E00135019B96
:10D2A0009D4222DA0026A642F8DA32002900380030
:10D2B00019F059FD320004902900039819F053FD2C
:10D2C000059B002BE4D0049B1B18092B00DD0923D0
:10D2D00032002900029819F091FC0136E3E7044975
:10D2E000044818F09BFE09F062FA029807B0F0BDFE
:10D2F000B9800300ACFD0200F8B5040008000D0081
:10D30000160006F02BF8164FB84201D000200FE0AF
:10D31000053C042CFAD820000DF036F9141403F85B
:10D320000B00300006F066F9011C2800FFF73EFFF5
:10D33000F8BD300006F05EF9011CFE2080050DF0FE
:10D34000F3FDF1E7300006F009F8B842DED16242A1
:10D3500062413100D2B22800FFF782FFE8E7C04601
:10D36000DC050300F7B507000193142008AB0E009D
:10D3700015001C7818F0EFFA044B476003606B4609
:10D380001B798660C56003744474FEBD60060300AB
:10D3900070B505000C2018F0DEFA0521044B0400DE
:10D3A000456003600800FFF76BFCA060200070BDC3
:10D3B0006402030070B50C0005000B6805495A684B
:10D3C0001BF0C3FF2168280040312200FEF720FE39
:10D3D00070BDC0467D9F0300136870B5002B12D14D
:10D3E0000568EE6BB34200D170BD9C002C19246C13
:10D3F000A14201D00133F5E7591CF5D002339B005F
:10D400001B581360F0E70349034818F007FE09F0C2
:10D41000CEF9C046D780030048F80200F0B585B0C9
:10D420000C000325FBF722FB25400700002D03D14C
:10D430001E4B22689A4205D01D491E4818F0EEFD89
:10D4400009F0B5F903AA02A9200017F04EFC029ECC
:10D45000039B300010308000019318F07CFA040028
:10D460003C2229001EF062FA134B67602360134BC5
:10D47000E663A360124BE360124B6361124BA3613E
:10D48000124BE361124B2362124B6362124B6363D4
:10D49000AE4202D1200005B0F0BD019BAF00D859CB
:10D4A000FBF7E4FAE71938640135F1E704D4020028
:10D4B0000C81030034FD02008CE40200B5D30000AF
:10D4C000DDD40000CD5C00008D5D0000D9D30000EC
:10D4D000815E0000295D0000DC060300F0B51D0040
:10D4E00085B0C36B00AFFB607A608B18FA680600EA
:10D4F0000C009A4205D02B492B48FEF7E1FE09F0BB
:10D5000056F9FB688B424AD09A00130069460E33E5
:10D51000DB08DB00CB1A9D4618000021BB601EF023
:10D5200005FA0023A200934210D1F9687A688C466C
:10D5300062447A60ED187B689C420CD3B968F86845
:10D54000F8F704FCBD46066005B0F0BDE858B968C0
:10D55000C8500433E7E72868FBF788FA0021020087
:10D56000F36B3B603B68994204D110490E48FEF7CB
:10D57000A7FEC4E78B00F018006C824201D0013195
:10D58000F0E70131F1D0B968CB181968002901D052
:10D590000749EBE76A6802341A600835CBE7BD60DB
:10D5A000CCE7C046BA34030034FD0200EB80030030
:10D5B000F3340300F0B5114B87B003AD40C9013817
:10D5C000009301950323FDF7C1F868680C4C1E27F2
:10D5D000A04202D017F0A2FE0700A8680022A042D5
:10D5E00002D017F09BFE0200706803990771427128
:10D5F00009F012F9200007B0F0BDC0464C07030047
:10D60000D8F5020030B5124B8BB003AC20C90138FD
:10D61000009301940323FDF799F8616806A819F0B7
:10D62000E4FF039B089A5900237A00936868079BDC
:10D630000AF074FA021E05D006490748FEF740FEBC
:10D6400009F0B5F806A90548FBF7B8F90BB030BDED
:10D65000700703001A810300B4FB020040EE0200D1
:10D6600030B5114B89B002AC20C901380093019448
:10D670000323FDF76BF8012205A9606806F010F995
:10D68000029B059A5900237A00936868069B0AF06A
:10D690008FFA021E05D005490548FEF711FE09F074
:10D6A00086F8044809B030BD940703003D810300AB
:10D6B000B4FB0200D8F50200074BDB68002B01D158
:10D6C000180006E05A68824204D8801A04308000AC
:10D6D000C05870471B68F1E7C409002070B5114DB0
:10D6E0000400EB689868DB6883420FD30230C00007
:10D6F00018F031F9EB685A68D96803609B685218D2
:10D700005B00836000234260C360E860EA68D3681E
:10D710005068591C04339B000138D16040189C505C
:10D7200070BDC046C4090020074B4118884204D38D
:10D73000D8B2002800D1013070475A01D3180278BE
:10D7400001305340F2E7C04605150000034B044A80
:10D75000DA60002294331A607047C046C409002082
:10D76000E4070300F0B585B001900E00FFF7DCFF81
:10D77000144B0290DC68002C01D120001EE0270031
:10D7800010373D00E3689B00FB180393039B9D4209
:10D7900001D32468EFE72868029A03789A420FD1F0
:10D7A00043789E420CD10230320001991EF094F869
:10D7B000002805D1ED1B6068AD10281805B0F0BD3C
:10D7C0000435E3E7C4090020F0B585B0029001916B
:10D7D000FFF7C8FF002858D12F4C019B2700943732
:10D7E000DD1C3B68002B17D026002C4A98361268A7
:10D7F00031680392AA188A420ED9020069181800EB
:10D8000018F0CCF80390002841D1244B38681968EF
:10D8100018F0B7F8039B3B60230094331B68002B80
:10D8200017D12E00802D00D280263000270018F05E
:10D830009FF894373860002804D1280018F08BF83E
:10D840002E003860230098331E60230000229C3392
:10D850001A6023009C331A6894342468AD18019927
:10D860000298A4181D60FFF75FFF6B461B792070BC
:10D870006370019AA01C02991EF03DF80022019BE2
:10D880002000E3189A70FFF729FF05B0F0BD336858
:10D890005B193360C0E7C046C4090020600A00205D
:10D8A00010B50024074B1C70FEF752FEF9F76EFC12
:10D8B000FEF76AF9F6F7DEFBFDF750FF024B1C702E
:10D8C00010BDC0461E09002073090020064B10B58C
:10D8D0001A680823D16C0B43D36418F0BDFBF7F72B
:10D8E000A1F9F8F7C3FDFCE7B008002010B50C481B
:10D8F0000CF070F918F0EBFAFCF760FCF9F752FE47
:10D90000F7F738FC07481BF005FE0748F3F778FEE9
:10D91000F3F754FEF7F73CFCF4F76CFA10BDC04681
:10D92000E4050020EC040020A1D80000F0B50700B9
:10D93000443787B0040038000E00002519F074FE4B
:10D940002069431C1CD00A2804D1200019F081FC56
:10D950000125F5E707F096FA002803D0200019F01A
:10D9600078FCEDE72369232B08D1200019F071FC26
:10D9700023695A1CE4D00A2BF7D1E1E75C2B0ED0C7
:10D98000E369226AA363E263002E17D1636A002B66
:10D990001DDA220007214032117001331EE0200001
:10D9A00019F057FC23690A2BD8D0E369A363236AD3
:10D9B000E36304234034237007B0F0BD012BE5D1AD
:10D9C000012AE3D00622230040331A7007E0002B1F
:10D9D0001FD02200062140321170013B63622000FB
:10D9E00040300378082BE7D10023E56CB24EA46CDD
:10D9F0009A00915900228F18944200D170E28F5CF6
:10DA0000BC46AF5CBC4500D168E20133222BEFD1AC
:10DA1000D2E7002D34D0A36A002B31D1210005209C
:10DA200040310870551E6362226BA44B606BD318A3
:10DA30005B001B5A9D42BFD017D9E16A8A4207D3C7
:10DA40000831490017F09DFFE36A60630833E36221
:10DA5000236B5A1C2263626B5B009D52636A9CE7D6
:10DA6000013B2363636A013B6362236B934A9A1809
:10DA70005200125A9542F3D39ED002230B70AEE7A8
:10DA80002069431C1AD18D4A236B616B9B185B0084
:10DA90005A5A23004033002A97D005221A700023D7
:10DAA0006362864A236B9A185200525A002A00D1A8
:10DAB00082E7013B2363636A013BF1E727281FD01C
:10DAC00022281DD0752804D0102302009A43622A10
:10DAD00004D16369272B0ED0222B0CD0722800D0E2
:10DAE00015E26369622B00D017E2A369272B02D0ED
:10DAF000222B00D011E2752804D1200019F0A9FBD7
:10DB000000234DE0622842D1200019F0A2FB00233F
:10DB100002932369722B04D1200019F09AFB012390
:10DB2000029323000C2240331A70012305932369CA
:10DB30000393222B01D027230393200019F089FBA4
:10DB40000123039A0493236993420BD11300626962
:10DB5000934207D1200019F07CFB200019F079FBDB
:10DB600003230493002623690193013300D1C9E004
:10DB7000049B012B03D1019B0A2B00D1C2E0049B23
:10DB8000B34214D83100380019F0ECFD27E77228B1
:10DB9000B6D1200019F05DFB2369622BBCD00123B4
:10DBA000029323000B2240331A700023BEE7019B2F
:10DBB000039A934208D111003800013602F074FE36
:10DBC000200019F046FBCEE7019B5C2B00D096E0CD
:10DBD000200019F03EFB029B2569002B04D05C213C
:10DBE000380002F061FE5AE0622D00D1BEE130D86B
:10DBF0004E2D78D01BD8222D53D0272D51D0002662
:10DC00000A2DDDD0280030380728E8D80500032683
:10DC10006369303B072B42D8013E002E3FD02000E5
:10DC200019F017FB2369ED00303B5D19F0E75C2D1F
:10DC300037D0612D5AD0552DE4D1059B002B27D02C
:10DC40005C21380002F030FEE9B2380019F041FDE5
:10DC500013E0742D13D008D86E2D00D188E1722DF9
:10DC600014D0662DCED10C250AE0762D0CD0E4D34D
:10DC70000226782D10D06B1CC4D10026A0E7092500
:10DC8000059B002BE0D112E00B25F9E70D25F7E706
:10DC90000826752D00D1043E0025013E12D26B1CD2
:10DCA000EBD0074B9D4225D8059B002B20D12900A6
:10DCB000380002F0F9FDE0E790130300FFFFFF7F5B
:10DCC000FFFF1000200019F0C4FA23691800019327
:10DCD00007F0FCF8002800D113E101981BF0A9F926
:10DCE0002D012D18D9E7A54802F0B6F90725DBE785
:10DCF000FF2DA9D92300012240331A70BDE76B46DE
:10DD00001979A2E7049BB34200D83BE72300032222
:10DD100040331A7036E707F0CDF8002807D0260008
:10DD2000216940362E291CD10A23337029E023694A
:10DD30002E2B04D1606907F0BDF80028EFD12169CE
:10DD40002E2954D0002602228D4D2F78002F01D08D
:10DD5000B9426CD1200019F07CFA002F76D1012253
:10DD600031E60923337030290BD16269173313432D
:10DD7000623B162B03D8834DDD4001231D40012358
:10DD80001D40380002F090FD200019F062FA14E006
:10DD9000002D16D1652801D0452812D10A2365210E
:10DDA0003370380002F080FD200019F052FA21692A
:10DDB00002220B002B3B9343E3D02069431CE7D1A5
:10DDC0000DE607F06BF8002808D021692E29ABD0AA
:10DDD0000B00202293434A2BD3D1A5E7206907F0FB
:10DDE00069F80028F1D123692E2BEED0F7E5260043
:10DDF000380002F059FD200019F02BFA2369403653
:10DE00002E2B00D0B6E065692E2D00D0B2E029009F
:10DE1000380002F049FD2900380002F045FD2000DD
:10DE200019F017FA200019F014FA0D23A3E03B00B3
:10DE3000633B9343DBB2681C002B03D10500013622
:10DE4000013582E7452FFAD1013EF7E7330001356E
:10DE50002A78652A09D16A7821690136914212D15E
:10DE6000200019F0F6F9330001352A78452A20D12F
:10DE70006B7822699A420AD1200019F0EAF933003E
:10DE8000414AD25C04E01F0002353B00E0E701227A
:10DE9000230040331A70230040331B7804221900FA
:10DEA0009143422901D0442B10D1A36A0133A362CC
:10DEB00095E5632AE4D16A782169771C9142DFD124
:10DEC000200019F0C6F902353E00DEE7432902D0F2
:10DED000452B00D083E5A36A013BE8E701328AE5E0
:10DEE0003A78002A00D090E5212B08D1274BA8339F
:10DEF0001A680E23002A00D1023303705CE50E334A
:10DF0000FBE72300012240331A700500B8E66228BF
:10DF100003D16369722B00D1E7E506F0BFFF051E50
:10DF2000206904D15F2802D07F2800D8F3E62300BF
:10DF3000082240331A70C1B2380019F0CAFB200021
:10DF400019F087F92069431C00D148E506F0A6FFC7
:10DF5000002809D120695F2806D07F2804D806F060
:10DF6000A9FF002800D13AE5217CE5E7082587E6EE
:10DF70000A2585E64A23337031E5C046709D0300CB
:10DF80002E9D030001204000EF9D0300C4090020E6
:10DF9000036810B5186B00280ED0CB0702D50368B4
:10DFA000002B09D08B0702D54368002B04D04B0708
:10DFB00008D58368002B05D10349044818F02EF8D2
:10DFC00008F0F5FB10BDC0461A9E0300B4FB02002A
:10DFD000F0B5012189B00190FFF7DAFF802106003A
:10DFE000490004A819F0EAFA80240023069D640081
:10DFF000009303AB2200290001983768B847431CFF
:10E000001AD103990B290FD1009B1848002B09D076
:10E01000009B17480593337BDB0700D4154804A900
:10E02000FAF7CCFC09B0F0BD0123490019431248AE
:10E0300017F0EDFF08F0BBFB0028E9D0009B1B1890
:10E040000093844202D9241A2D18D2E7802104A813
:10E05000490019F002FB051E04D108490648FEF7E5
:10E060002FF9E7E780246400C3E7C046D8F5020033
:10E070000818030040EE0200B4FB0200479E0300B4
:10E08000F0B50E008BB0040001213068FFF780FF6F
:10E090000700012C04D13068FFF79AFF0BB0F0BDE8
:10E0A000706805F043FA030000900133F3D00125B6
:10E0B0003B7B2B4275D00100040006A819F07EFAC4
:10E0C000002303950193002C5FD0210006A819F0CE
:10E0D000DDFA011E05D142494248FEF7F1F808F089
:10E0E00066FB3D6805AB22003068A8470500431C6D
:10E0F00016D1210006A819F035FB05990B2908D186
:10E10000079B0093002B40D106A819F082FA3648ED
:10E11000C4E7012349001943344817F078FFDEE7CC
:10E1200084422CD8089B079C029302239C460198AA
:10E13000019A029B9B5C039A59B2002912DA1900DA
:10E140001F256246A943C0290CD01900103D0322A7
:10E15000A943E02906D004329343F03B1A00511E34
:10E160008A410432019BD3180193A34212D8009B29
:10E170000198013B0093A042DAD3009CA3E7211A47
:10E1800006A819F0EFFA002DCCD1194806A9FAF724
:10E1900015FC83E7E443009BE418019B0190E4181D
:10E1A00091E7009906A819F020FA05AB009A0899A2
:10E1B00030683C68A047431C0AD106A819F029FA28
:10E1C000059909480B2900D168E749002943A3E7CD
:10E1D0003B7B079006482B4200D1064806A9D6E7AC
:10E1E000399E030000FB0200D8F50200B4FB0200D8
:10E1F0000818030040EE02007FB50C000600012164
:10E200002068FFF7C5FE0222050001A9606805F03D
:10E2100047FB029A022E06D9A06805F087F9029AF8
:10E22000824200D902006B462D6801992068A847F8
:10E23000431C0BD1009908480B290AD0012349003F
:10E240001943064817F0E3FE08F0B1FA4300012035
:10E25000184304B070BDC046D8F50200B4FB0200FC
:10E26000F0B589B00191019B040001211868FFF706
:10E270008FFE0600012C1AD9019B5B685C10631CA1
:10E2800015D0210004A819F099F9631C03D0631E6E
:10E29000002C36D01C00012104A819F0F7F9071E44
:10E2A0000CD11E491E48FEF70BF808F080FA012435
:10E2B000102104A819F082F96442E6E701000198F0
:10E2C00003AB012200683568A847431C13D10399AA
:10E2D0000B2909D1059B0193012B0ED104A819F03C
:10E2E00098F9104809B0F0BD0123490019430E48C0
:10E2F00017F08DFED9E700280CD1012104A819F0F0
:10E3000031FA337B0948DB0700D4094804A9FAF73E
:10E3100055FBE7E73B780A2BB7D1F2E7399E0300BC
:10E3200000FB0200D8F50200B4FB0200081803004D
:10E3300040EE0200F7B50E00022104001700FFF7BF
:10E3400027FE01AB45683A0031002000A847431C76
:10E350000BD1019907480B290AD001234900194321
:10E36000054817F054FE08F022FA43000120184334
:10E37000FEBDC046D8F50200B4FB020003000F202A
:10E3800010B5084003280ED80CF008F90204090D56
:10E39000180010BD0648002BFBD10648F9E718000D
:10E3A00017F0F7FBF5E7180017F00EFCF1E7C04691
:10E3B00010D6020008D60200F0B5836999B05A1E43
:10E3C00006339B000492C218079102920F2101228A
:10E3D000C318043303930369019006A81A4009186F
:10E3E0000A70032293430A930CA808F0C5F9031E90
:10E3F00001D000F03FFD019A5568D468079A002AC1
:10E4000000D184E22A785E2A00D180E2079807933F
:10E4100001F03AFD04000AE0D24B63600434D24BB1
:10E420001A6B002A00D171E200221C6B1A6308F0FB
:10E43000B9F90D9400F01EFDCC4BEEE7CC4BECE7A8
:10E440007F216B785B06DB173A78DB01100052B254
:10E45000084003430137002AF6DB01225B00134327
:10E46000DBE700237F213A78DB01100052B208403D
:10E47000C3180137002AF6DBDB000622EFE7032290
:10E480000337974308CFC8E70023C6E700237F215F
:10E490003A78DB01100052B20840C3180137002A55
:10E4A000F6DB9B005B42029A9858002800D0EEE20F
:10E4B000B049B14817F0B2FDACE700237F213A78AC
:10E4C000DB01100052B20840C3180137002AF6DB06
:10E4D000029A9B005B42985817F0BAFDE5E70020CE
:10E4E0007F223B78C00119005BB211400818013748
:10E4F000002BF6DB251D00F045FE60605EE000208D
:10E500007F223B78C00119005BB211400818013727
:10E51000002BF6DB251D00F003FEEEE700217F2235
:10E520003B78C90118005BB2104041180137002B3D
:10E53000F6DB206818F0A7FF206070E700217F223B
:10E540003B78C90118005BB2104041180137002B1D
:10E55000F6DB220001CC00F087FF60E7251D00F00C
:10E5600029FECAE7251F04222168286805F066F9FC
:10E57000286023E000237F213A78DB01100052B2AB
:10E580000840C3180137002AF6DB9B005B42029A61
:10E5900021689950E3E000237F213A78DB011000E5
:10E5A00052B20840C3180137002AF6DB9B00029ADA
:10E5B0005B4221689858251F17F04CFD2C002EE770
:10E5C00000207F223B78C00119005BB2114008187F
:10E5D0000137002BF6DB2168251F00F0FFFDEDE77A
:10E5E00000207F223B78C00119005BB2114008185F
:10E5F0000137002BF6DB2168251F00F007FEDDE761
:10E6000000217F223B78C90118005BB210404118FD
:10E610000137002BF6DB231F1A68206800F04CFF3F
:10E62000083CFCE62200231F083A1268216818689B
:10E6300005F004F90C3CF2E600237F213A78DB0177
:10E64000100052B20840C3180137002AF6DB029AC4
:10E650009B00D31A1A68002A00D129E700221A6009
:10E66000DDE600257F223B78ED0119005BB2114009
:10E670004D190137002BF6DB029BAD005D1B2868AE
:10E6800017F0E6FC002800D112E70021286817F0F7
:10E69000E1FCC4E600207F223B78C00119005BB298
:10E6A000114008180137002BF6DB00F0A3FDB6E699
:10E6B00000207F223B78C00119005BB2114008188E
:10E6C0000137002BF6DB00F0ADFDA8E62368A4E6D9
:10E6D0002368A360231F1B68636008349FE6231F21
:10E6E000196822682160BAE7221F13682168236035
:10E6F0002300083B18681060196090E67B783A7830
:10E700001B0213431D4A9B18EF1888E67E783B785E
:10E71000206836021E4305F047F8EF1C251F2C0029
:10E72000002800D17BE6164BF618BF1977E67E78F5
:10E730003B78206836021E4305F036F8EF1C251F93
:10E740002C00002800D06AE6EDE77E783B783602A0
:10E7500020681E43EF1C05F027F80028E3D1043C95
:10E760005DE6C04608D60200C4090020D8F50200C4
:10E7700010D60200559E03003CFB02000380FFFF01
:10E780000080FFFF7E783B78360220681E43EF1C36
:10E7900005F00AF80028C6D0E1E726002768220025
:10E7A00038001721083600F05FFE380032001621CD
:10E7B00000F05AFE00213200080018F055FEAB7838
:10E7C0006A781B0213430A9A0F210C320A920A9AA2
:10E7D000EF1CFB181360022206ABC9180A9D0B78C8
:10E7E0001A43231D13436B6000230A9A0B70936036
:10E7F000A060340013E625002668AC4B083D9E421D
:10E8000008D16660A6602A000021032018F02CFEC3
:10E810002E60D3E6012131402CD07610231F012E2B
:10E8200011D126001A680C3E0592A04A00211A60F8
:10E83000032022606260320018F016FE059B3360F0
:10E8400003232B60ECE626002A68103E05921A6826
:10E8500000210692954A03202A601A602260320045
:10E8600018F002FE059B069A336023000C3B1A60E9
:10E870000523E6E72B682E602600103E2360320059
:10E88000032018F0F1FD04F08FFF00280DD00122C5
:10E89000864B06A933600A9B5B6813400E32521800
:10E8A00013700A9B0C3B0A93A3E723683360230091
:10E8B000043C22680C3B1A6080E67B783A781B02A5
:10E8C00013437B4A9B18EB186360EB780834236092
:10E8D0000F267F210220012506AA2368B6180B42C5
:10E8E00005D1221F1768002B00D0A3E698E60A9AEC
:10E8F000013B5268024270D0220008C205236360C7
:10E9000014000A9B1F680A9B0C3B0A933D00019B65
:10E910006F1C5D602B78180010385A2800D907E367
:10E920000BF046FE7AFD8AFD8CFD06038EFD060384
:10E930009FFDADFDB2FD0603B4FDCBFDDDFDEDFD9C
:10E94000FCFD0CFE1CFE20FE28FE39FE4EFE5EFE87
:10E950006EFE80FE8AFE9FFEB8FEC6FE060306031C
:10E9600006030603D4FED6FE1DFFDDFEE2FEECFE2E
:10E97000F4FE05FF13FF30FF0603060306033BFF0B
:10E9800069FF630063008000A300A700B700B70021
:10E99000CBFF06030603060306030603060306036E
:10E9A00006030603C800DA00EC00FE000D011601A4
:10E9B0002B013D014F016C0182013002570282029E
:10E9C0006F0206039701A201AD01BA01C601E2017F
:10E9D000FC011902DA02EF0200030A9A52682A4087
:10E9E00032700A9A0C3A0A9279E77B783A781B02DD
:10E9F00013430A9AEF1C0C320A920A9AFB1813600E
:10EA00002B780A9A403B584258410F21430006A8F0
:10EA10000918087803432343536000230A9A0B70B4
:10EA20009360FCE42068FDF793FC251F002804D0C8
:10EA300007F0B8FE2B680D931CE223681B4A2C00DC
:10EA4000934200D1EBE45B10DBB2012B00D03FE737
:10EA500002220A9B0399994200D8A3E107F0A2FE83
:10EA60000020019BDC6019B0F0BD206800F048FD7B
:10EA700062E57E783B7836021E43019BEF1CDC602A
:10EA8000206800F063FD002801D1043C4DE6606081
:10EA9000C4E401220A9B06A95B6813400E32521897
:10EAA00013700A9B0C3B0A93B9E4C046D8F50200E8
:10EAB0000380FFFF00207F223B78C00119005BB27A
:10EAC000114008180137002BF6DB8300E41A0434E8
:10EAD0002100F7F73BF92FE500207F223B78C001AA
:10EAE00019005BB2114008180137002BF6DB8300D8
:10EAF000E41A0434210016F0E1F81DE500237F211B
:10EB00003A78DB01100052B20840C3180137002ADE
:10EB1000F6DB9B005B4221681859F4F7CDFE1EE638
:10EB200000207F223B78C00119005BB21140081819
:10EB30000137002BF6DB251D14F0E1FEDDE4250096
:10EB4000231F083D1A682168286814F010FF35E576
:10EB500000237F213A78DB01100052B20840C3182D
:10EB60000137002AF6DB01339B00221F5B4212684B
:10EB70002168185914F0FBFE52E500207F223B78F3
:10EB8000C00119005BB2114008180137002BF6DBF9
:10EB90008300E41A0434210005F098F8CCE4002343
:10EBA0007F213A78DB01100052B20840C3180137C8
:10EBB000002AF6DB9B005B42216818591AF0D4F852
:10EBC000CDE500237F213A78DB01100052B20840E6
:10EBD000C3180137002AF6DB251F022B05D1DC4ABA
:10EBE0002168286804F0BAFEC2E42600083E2268C4
:10EBF0002968306804F0B2FE3060FAE500257F2114
:10EC00003B78ED011A005BB20A4055190137002B21
:10EC1000F6DB22002900206800F0E8FFCD4B5D19EB
:10EC2000AD006419FFF7FBFB00257F213B78ED0168
:10EC30001A005BB20A4055190137002BF6DB22009F
:10EC40002900206801F026F8FF222B0A1340154006
:10EC5000E5E70322FB1C93430022186811001F1DE7
:10EC6000251D17F098F948E40322FB1C9343251F48
:10EC70002268296818681F1D17F08DF978E40322AF
:10EC8000FB1C934319795F1D8A00A41A04342200E7
:10EC9000186817F09BF94FE40322FB1C9343187983
:10ECA0008021C243490092005F1DA4180143EEE792
:10ECB00000207F213B78C0011A005BB20A40101887
:10ECC0000137002BF6DBFF25FF220100C3096D0091
:10ECD00011402B405B189B00E41A000A0240231DE0
:10ECE000206800F013FB27E400217F223B78C90154
:10ECF00018005BB2104041180137002BF6DBFF22F1
:10ED0000CB0952001340CAB29B189B00E41A083C7E
:10ED10002200002000F03AFEFFF70EFC00237F20C7
:10ED20003A78DB01110052B20140CB180137002ABA
:10ED3000F6DBFF211800FF250840DA096D002A40A4
:10ED4000451C52199200A41A1B0A1940220018F0FF
:10ED50008BFBFFF7F1FB00217F223B78C9011800F4
:10ED60005BB2104041180137002BF6DBFF22CB09C4
:10ED700052001340CAB29B189B00E41A0C3C2200BC
:10ED80000120C7E70F2206ABD2181378002B00D161
:10ED90005EE601210A9B5B680B4013700A9B0C3BEB
:10EDA0000A9355E60A9B5B6813420ED003220A9B26
:10EDB00021685B6893431C0059609A600A9B083481
:10EDC0001F680A9B0C3B0A93A0E50A9B0C3B0A9325
:10EDD0003FE66B78022B03D1043C2068FFF718FB59
:10EDE000002BFAD10A9B039A934203D25A495B48FB
:10EDF000FFF760FB9868002801D0FFF709FB0C3B88
:10EE0000F1E7079E231F0593002E1CD0079E0021CB
:10EE1000320007910BAB201F006800F0C9FF0128EA
:10EE200015D12F000B9B236007F0BCFC019B06AAA9
:10EE30005F60DC600F239B181A780A9B0120134344
:10EE4000019A13610FE60BAB32002168E3E700285B
:10EE50002FD10B9B043C002B00D13D4B2360002E97
:10EE60004CD03F49300017F0E3F8002846D007F0B7
:10EE700099FC0D960D9B3B491868F9F7BDF80028E1
:10EE800000D1AEE0019B5A68002A00D1A9E01378B6
:10EE9000432B00D092E0937850781B02D11C03439F
:10EEA000019ACB185360D3680593043BD360FFF7F6
:10EEB0009BFA02280FD12B490B9817F0B9F80028BC
:10EEC00005D00B98FDF7DCF9043C2060C7E707F09C
:10EED00069FC0B9BAFE5059C00207F223B78C001BD
:10EEE00019005BB2114008180137002BF6DB251F13
:10EEF0002A68216800F0E6FFFFF73AFB059CFFF760
:10EF00008EFA00217F223B78C90118005BB21040C5
:10EF100041180137002BF6DB250001CD00F0E4FF9E
:10EF2000FFF7EBFA2068251F18F0B9FAFFF746FB48
:10EF3000AF2B05D80120803B5B000343FFF76DFA40
:10EF4000BF2B11D8B022D31A9B00FFF7ACFAC046F2
:10EF5000D8F50200FFFFFF3F9B9E03002CFC020040
:10EF600050F9020074FC0200CF2B04D8C022D31A3F
:10EF70009B00FFF70CFBD62B06D8D03B180021686E
:10EF800000F05CF9FFF7D8FAFA2B08D8251FD73B19
:10EF900018002268296800F03FFBFFF7E9FA4C49A6
:10EFA0004C4817F03BF8040007F0FCFB049B019A67
:10EFB00006339B00D3185C60022054E55E2B10D111
:10EFC000019B019ADC680D98231DD360FDF758F969
:10EFD000019B60605B68019A059301335360FFF702
:10EFE00003FA0D9B3C4A934231D03C4A93422ED0C7
:10EFF000019B0BA81B6805930B9314F018FA0400EF
:10F000000BA814F014FA05000BA814F010FA019BD9
:10F0100001005B680593019B1B680693069A059B9C
:10F020009E1A1F2301229C46361B0B9C2378002B23
:10F0300009D058B200282EDB6046013418405B0925
:10F040000B94864231D22B000D98FDF7A9F90F23BE
:10F05000012106AA9B181A78002A29D10A9A039935
:10F0600091422DD801221A700A9B0D991B680593B5
:10F07000059A019B05915A6003220A9B5B689343A2
:10F080000A9A9160164A5A600D9A9A6012680C3377
:10F090001A60019A0AE70F20E0271840FF001B01C1
:10F0A0001F40637802343B43CAE7361AD218BCE7E4
:10F0B0000A9A52680A401A700A9A0C3A0A92CAE7E7
:10F0C000049B019A06339B00D3180D9A5A6073E78C
:10F0D000819E030078FB0200A4F70200B4F702004F
:10F0E000D8F5020070B5FEF731FB0B4C002623006B
:10F0F000A8331E602663FBF7B5FF084D01212800E9
:10F10000F2F7C0FD28005E226E2114F030FC65602D
:10F110002560666470BDC046C4090020F80900205F
:10F1200070B50624134EC3001C437368002205000B
:10F130002100181D05F052FD021E18D1706C002828
:10F1400007D00430210005F049FD002801D04068B7
:10F1500070BD00222100084805F040FD021E06D1C6
:10F160002A0006490648FDF7ABF807F020FB506877
:10F17000EEE7C046C4090020D4C502009F9F0300EB
:10F180003CFB02000A4B10B5040018685B6898420B
:10F190000AD00621E30019430430002205F01EFDC9
:10F1A000002801D0406810BD2000FFF7B9FFFAE742
:10F1B000C4090020074B10B5586C002801D106483F
:10F1C00010BD04300022262105F008FD0028F6D0ED
:10F1D0004068F5E7C409002050C402000A00C100DD
:10F1E000062010B5024B0143186814F0C0FB10BD97
:10F1F000C4090020062110B5034BC0000143186864
:10F2000014F0BFFB10BDC046C40900200A00C100B5
:10F21000062010B5024B0143586814F0A8FB10BD3E
:10F22000C4090020062110B5034BC00001435868F3
:10F2300014F0A7FB10BDC046C409002070B505003E
:10F240000C00062806D1080004F0AEFA00280ED003
:10F25000274870BD012001421AD04B10042D08D060
:10F26000052D13D00800002DF3D1002BF0D021483C
:10F27000EFE7C0221206934204D18020C00516F0A9
:10F2800088FCE6E75B425B001843E2E7DB43FAE712
:10F29000022D12D1184B0B40062B08D08B070CD136
:10F2A0000A68164B92699A4207D1486802E0C8087A
:10F2B00017F0B7FF43000120E6E7200004F04EF806
:10F2C0004369002B0DD10E4BAD002000ED5819F015
:10F2D00063FC2A0003000B490B48FCF7F1FF07F021
:10F2E00066FA2100280098470028B2D1EBE7C04613
:10F2F00008D6020010D60200070080FF3D990000EA
:10F30000C8E402002BA0030034FD0200F7B504009E
:10F31000019116001F0004F021F80569002D09D1A4
:10F32000200019F039FC064902000648FCF7C8FF26
:10F3300007F03DFA3B00320001992000A847FEBDCE
:10F340006868030034FD0200F8B504000D001700E2
:10F350001E0000290BD0186804F000F8636898427A
:10F3600005D00649064816F059FE07F020FA33008A
:10F370003A002900A068FFF7C9FFF8BDBA9E030054
:10F3800034FD0200F8B506000F0014001D009307BD
:10F3900014D11368174A934202D163682B60F8BDF9
:10F3A000154A934207D1002802D003F0D7FF070087
:10F3B000636888C5F3E7114A934201D12C60EEE7F8
:10F3C0005B681A00F23A012A01D9F02BF6D1002E1F
:10F3D0000ED1200003F0C2FF094B984208D10C2047
:10F3E00016F0B9FA074B4760036084602860D6E7DF
:10F3F00050C5D4E714E40200D8E302008CE4020014
:10F4000090C902009C140300F8B5002313605360F8
:10F4100006000D00140003F0A1FF0700102D05D118
:10F42000836A002B02D00F4B48C4F8BDFB69002B48
:10F4300004D02200290030009847F6E7B86B002876
:10F44000F3D00621ED00294304301A0005F0C6FB75
:10F450000028EAD04268230039003000FFF792FF0D
:10F46000E3E7C0464CC5020070B5160004000D006D
:10F47000FFF7CAFF3368002B15D10B4EA3070BD142
:10F480000A4B22689A4207D12B0062680849300073
:10F49000FCF716FF07F08BF9200019F07DFB2B001D
:10F4A00002000449F3E770BD48F802008CE4020052
:10F4B000B89F0300DF9F030073B504000D00160022
:10F4C00003F04CFFC369002B09D00422019600927F
:10F4D00029006A4620009847009B002B0AD0200094
:10F4E00019F05AFB2B00020003490448FCF7E8FE20
:10F4F00007F05DF973BDC046DF9F030048F80200C6
:10F5000013B5040003F02AFF436A002B11D16A46A9
:10F510001A212000FFF778FF009B002B0ED120005E
:10F5200019F03AFB074902000748FCF7C9FE07F04B
:10F530003EF9200098470028E9D016BD6846FCF740
:10F5400041FDFAE74E9F030034FD020037B5040089
:10F5500003F004FF856A002D02D02000A8473EBDBD
:10F560006A4610212000FFF74FFF009B002B05D0BB
:10F570006A462900280017F077FFF0E7200019F00D
:10F580000BFB034902000348FCF79AFE07F00FF952
:10F59000809F030034FD020030B505008FB0F2F704
:10F5A000F9FB280003F0DAFE846A002C05D028005D
:10F5B000A047040020000FB030BD6A46102128008B
:10F5C000FFF722FF009B002B16D002A807F0D4F80B
:10F5D000002807D16A46010017F046FF040007F033
:10F5E000E1F8E7E7039B09491868F8F705FD0028EB
:10F5F000E0D1039807F0DBF8280019F0CDFA0449B0
:10F6000002000448FCF75CFEF4E7C04674FC02000C
:10F61000809F030034FD0200F0B585B003900F0019
:10F620001600202804D1914210D0B14805B0F0BD99
:10F63000039B1B2B01D01E2B0DD13100380003F092
:10F6400023FF039B002803D01B2BEED1A948EDE735
:10F650001B2BFBD1E9E7039B212B28D11000FCF7E2
:10F6600077FE002806D03100380016F0E1FC0028B3
:10F67000ECD1DAE70324344000D05EE19E4B3268DF
:10F680009A4200D059E173689C42CED2A300F3188D
:10F690009D682800FCF75CFE002800D14CE12900A1
:10F6A000380016F0C5FC0028D0D10134EBE7012367
:10F6B000194200D1FCE013404D100293002B00D101
:10F6C000EEE0039B54101D2B00D936E118000AF020
:10F6D00079FF1E0028002A002D0047004E0051002F
:10F6E00053005E0067007D008500BA001E00280000
:10F6F0002A002D0047004E00510053005E006700B5
:10F700007D008500D300D7003401DB00DF002543F6
:10F710000295029B5C00634000D5BDE001202043C0
:10F7200084E76540F4E72C400294F2E7002C04DA09
:10F730007249734816F072FCCFE01F2C08DC714B45
:10F7400023419D4204DCC0231B0623419D4205DA70
:10F75000E917280016F00EFA07004BE0A540D7E79E
:10F76000002CE5DB1F2C00DD1F242541D0E72B19E1
:10F770000293CEE72B1BFBE721002800F3F702F8EA
:10F780000028E5D1012065436D0028434EE7002C99
:10F7900000D1E5E02100280014F089FF0290B8E7CD
:10F7A000002C00D1DCE028000CF0A2F8051C2000A1
:10F7B0000CF09EF8011C281C0BF0B6FB032305007F
:10F7C00002209D43504B2843C0182FE7002C00D146
:10F7D000C6E02100280014F05AFFDFE72F00002CBC
:10F7E0002EDA28000CF084F8032302279843464BB6
:10F7F0000743FF18380003F0B1FD8369002B00D1E7
:10F800009BE03200390003989847002800D00DE7AC
:10F8100093E001231C4208D039000298F2F7B2FFAE
:10F82000002895D1029B7B430293012C00D170E705
:10F83000390038006410F2F7A5FF002888D17F4313
:10F84000002CE6D165E7002C00D189E000210220E0
:10F85000F6F77CFA21000600280014F028FF0127A3
:10F8600040003843B0602100280014F010FFB84079
:10F870000743F7603000D9E6A54200DAE6E6D4E6B1
:10F88000A54200DDE2E6D0E6A54200DCDEE6CCE6FD
:10F89000A54200DBDAE6C8E6029816F07AF9C5E67A
:10F8A00003231340022B03D1184B1340062B5AD1CC
:10F8B000039B1F2B9ED1300003F050FD8369040091
:10F8C000002B0CD1636A002B26D1300019F064F9AB
:10F8D0000F4902000F48FCF7F3FC06F068FF3A00FE
:10F8E000310003989847002800D09FE6EAE7C04619
:10F8F00008D6020010D602009CDC0200907B0300B8
:10F90000ACFD0200FFFFFF3F00008080070080FF8A
:10F910004E9F030034FD02003000FFF7F1FD0400AC
:10F920002000FFF739FE002800D17EE6390003F001
:10F93000ABFD0028F4D089E62E00039B38009A0026
:10F940000D4BD45819F028F90500300019F024F9AE
:10F950002B000090220009490948FCF7B1FCBCE7E4
:10F9600008490948E6E628000BF0C2FF3200011CF6
:10F97000039801F005FC48E738E30200299F0300E3
:10F9800034FD02007F7B0300F4FD0200F0B5136834
:10F990008DB00693002800D06CE00400131D039383
:10F9A000FF220B00090A1340114001934B000593FD
:10F9B000059A019B04919B18039A9B00D558D31874
:10F9C0005F68381E09D00020BB0706D1844B3A6817
:10F9D0009A4202D1380013F0C7FF049B1E18002D75
:10F9E0004DD1019B76000133F3189800009315F078
:10F9F000B2FF25000600002C01D001250460019B08
:10FA0000A8009A00301803991BF075FF019B5B1941
:10FA10000293029B9800049B3018DA00019B990026
:10FA2000039B59181BF067FF029A059B9446634499
:10FA30001C00002F0FD003253D4000D09CE0684BF8
:10FA40003A689A4200D097E0380013F0A3FF41686B
:10FA50008D4200D07FE0029B0299E21A52083300E7
:10FA60000698FFF753FC0400300015F09BFF2000C0
:10FA70000DB0F0BD130008330393546890E7AB0753
:10FA80002FD12B68574A934202D0574A934228D12C
:10FA900028000AAA09A903F0EBFD099B019A01338A
:10FAA0009B1876009B199800009315F054FF2500D1
:10FAB0000600002C01D001250460019BA8009A00DB
:10FAC000039930181BF017FF019B0A995819099BDD
:10FAD00080009A0030181BF00EFF019B099A9B18BA
:10FAE00095E7019B7600181D33189800009315F0D8
:10FAF00032FF02940600002C02D00123046002931E
:10FB0000029B03999800019B30189A001BF0F3FEAA
:10FB1000019A029B9446280063440293FFF7F0FC8D
:10FB2000029B07909C000798FFF736FD051E00D149
:10FB30006FE7009B029A934207D8D900300015F076
:10FB400020FF0600009B5B000093029B35510133B0
:10FB500002930434E7E78368EF00DA59002A09D0FA
:10FB6000042A07D0A300F2508268F318D219526811
:10FB700002345A6001356BE70AAAC5213800FFF745
:10FB800073FC00210AAA080017F06EFCFFF7B8FC0E
:10FB9000A50001900198FFF7FFFC071E00D15AE76E
:10FBA000009A631C9A420BD853000093042B01D295
:10FBB00004230093009B3000990015F0E2FE06003C
:10FBC00009AA0221380003F075FD099B02341B6865
:10FBD0007351099B5A6873195A600835DAE7C046B1
:10FBE000CCCB02009CDC020004D4020073B50C00F4
:10FBF000150083071ED10368204A934207D0204A8C
:10FC0000934217D101AA694615F06FF803E001AAE3
:10FC1000694615F0D2FA009B9C4228D817D3019B65
:10FC2000A4001C19043B043C9C4200D173BD226813
:10FC300004C5F8E7FFF764FC002306000093009B6F
:10FC40003000A34206D3FFF7A7FC0028EED0220025
:10FC50000C490EE0FFF7A0FC002808D0009A0A49E2
:10FC6000A31A5B189B00013258510092E7E7009AF3
:10FC700006490748FCF724FB06F099FD9CDC0200CE
:10FC800004D402006CA00300FFFFFF3F49A0030063
:10FC9000ACFD0200F7B514000A0AFF230E001500A0
:10FCA0001E401D4083073BD107683D4B9F4208D053
:10FCB0003C4B9F4234D1FF231143194224D1206091
:10FCC000F7BD01AA694615F078FA009B72199A42AD
:10FCD0005ED89A009446002001998200A84218D16B
:10FCE0009B1BB5004919181AA41814F0E7FF019BD3
:10FCF00020605D190023013601339E42E0D09A0056
:10FD000051426958A150F7E701AA694614F0EDFF86
:10FD1000DBE76746BF1A043FCF590130A750DCE745
:10FD2000FFF7EEFB002307000093009B9E4217D8CD
:10FD30000021080014F0C2FF06003800FFF72CFC79
:10FD4000011E1AD1B1688D4222D8AB00E3181E60A3
:10FD500088009C4215D1491B300014F0CBFFAFE75F
:10FD60003800FFF719FC002812D0009AB31A5B196B
:10FD70009B00013218510092D7E73000F3F79CFD49
:10FD8000DBE7F268C71AA218D259043B1A60E0E711
:10FD9000009A05490548FCF793FA06F008FDC046AD
:10FDA0009CDC020004D4020049A00300ACFD020068
:10FDB000F0B587B01D0006000C00019203F0CEFAEA
:10FDC0002E4B984207D12B00019A21003000F4F706
:10FDD00081FD07B0F0BD876A294B002F08D09C42F7
:10FDE00021D13000B84728600028F2D00120F0E788
:10FDF0009C4218D103AA10213000FFF705FB039B9A
:10FE0000002B0CD103AACD213000FFF72DFB059468
:10FE100003AA0021012017F027FB2860E6E703AAC8
:10FE200039003800F7E7002CECD1019B2000002BB3
:10FE3000CFD0180003F092FA1249F8F7DDF8002845
:10FE40000FD003AACC213000FFF7DEFA039B002B72
:10FE500007D003AA2100200017F006FB286020002D
:10FE6000B7E703AACE213000FFF7CEFA039B01AA21
:10FE7000002BCED1019B02202B60AAE79CD8020068
:10FE8000D8F5020050F9020010B50400FCF760FA42
:10FE9000002808D0002320001A001900FFF736FAC6
:10FEA0000400200010BD200016F0BCF80028F8D196
:10FEB0000249034816F0B2F8F2E7C04601A0030079
:10FEC00034FD02007FB5C30006201843054B0190A6
:10FED0000491052001A9029303930592F6F712FEFF
:10FEE00007B000BDD8F502001423F0B58DB000AF07
:10FEF000FA1805000C00FFF787FABB69002B06D043
:10FF000022002C492C48FCF7DBF906F050FC7869FC
:10FF100000284BD1280015F0E9F90028F0D014236F
:10FF20002800FA180D21FFF76FFA10237869F918E5
:10FF3000F9F728FAB860200017F078F96A463E69A8
:10FF4000B968731C7B60C318FB600E33DB08DB00F1
:10FF5000D31A9D46320068461BF0CDFC6D462E2319
:10FF6000AB557B682000EB18BB6017F064F9060006
:10FF7000200017F05BF931000200B8681BF0BBFCF1
:10FF8000F9686846FDF720FCC300062018430B4BB8
:10FF900010223B627B620A4BBA18BB620123FB62F0
:10FFA0000B33F861D1180520F6F7ACFDBD460DB056
:10FFB000F0BDC0466A9F03008CF90200D8F502002C
:10FFC00010D60200F0B5174C0F00616895B0039190
:10FFD0002168060008A804916260236006F0CCFB4B
:10FFE000051E06D0039B09986360049B236006F0FE
:10FFF000DEFB33683A00310005A80193F2F786FD75
:020000040001F9
:100000002B002A00019905A803F008F817F014FA4C
:10001000050006F0C7FB2800039B6360049B236078
:1000200015B0F0BDC409002010B5040004F022FB97
:10003000031E064804D0064915F0F0FF06F0B7FB92
:1000400022000449FCF73CF9F8E7C04600FB020037
:10005000D29E0300FB9E0300010010B5024815F07C
:10006000DDFF06F0A4FBC04678FB0200F0B5204B94
:100070008BB004AC20C90138009301940623FAF731
:1000800065FBE0681B4EB04225D105271A4BDF57B0
:100090002069B04223D1194B5B795BB2039360694D
:1000A000B04220D10522164B9A56012304355B42FB
:1000B000009303993B00280007F0B6F80023A268DC
:1000C0006168280007F036F82800049907F06AF8FC
:1000D00030000BB0F0BD15F021F90700D8E715F09E
:1000E0001DF90390DBE715F019F90200DDE7C046C2
:1000F00044150300D8F5020050E1020060E102005F
:1001000058E1020070B586B006000122080003A97C
:1001100003F0C6FB039D2C00049A631B01929A42D4
:1001200005D92178301D07F067F90134F4E701485B
:1001300006B070BDD8F50200F0B5140089B00122F8
:100140000600080002A903F0ABFB200000240222F5
:1001500005A9029F03F0A4FB059D039B01939C420C
:1001600006D2395D301D07F047F928550134F4E710
:10017000014809B0F0BDC046D8F50200F0B5050051
:1001800087B048680C000F6803F0D0F9010002A89E
:1001900017F02BFA0026032D03D1A06803F0C6F94F
:1001A00006000024039B01939C4209D2049B381D46
:1001B00031001D19019307F01FF901342870F1E790
:1001C00002A90248F8F7FAFB07B0F0BD40EE0200C2
:1001D00073B501A9F9F7D6F8019B06001849502B11
:1001E00016D88020400015F0B6FB164C0500231DE4
:1001F000D8670023019A93420FD15B222800EA546A
:1002000003F0B4FE2B0000280BD104340E49E06744
:100210000E4815F003FF06F0CAFAF15CE954013309
:10022000E9E75A1B0133591E09789B29F9D12900A6
:10023000074815F04BFA00230434E36776BDC04647
:10024000A3A00300C4090020B2A00300ACFD02007B
:1002500008180300F0B58BB00600080011001A0062
:1002600010AB1F78334B05AD019500930523FAF7CA
:100270006DFA9120000115F06EFB2F4B04A9D86791
:1002800002AB1B7B476043702B792C4F03702B7A9A
:10029000040083702B7BC3702B7C30003B60F9F72C
:1002A00071F80025264B03900C201D6015F053FBC0
:1002B000244B06000360F5F75FFCB060F5F75CFCCB
:1002C000214B224A1860224B11001D70214B706097
:1002D0001D70214B30001D602B00F5F723FB200023
:1002E000049A039914F000FC2000F3F751FA04007B
:1002F000A8420AD1F5F724FA0F4B1848DC67184BCF
:10030000196815F08BFE06F052FA0122154B1A708F
:10031000F5F72CFC0028FBD1134B0433D8673B685E
:10032000002B04D00C4B1148196811F023FF07482B
:100330000BB0F0BDF4150300C8090020F002002046
:10034000880300205416030084030020D8F502001F
:100350007A090020780900208C030020ACFD0200FF
:100360001000002079090020C409002094A0030097
:1003700000220D4910B50B78DBB2934210D10B4A25
:100380001478002C02D001240C701370084B1B78D9
:10039000002B07D0074A136820331360064B1A68F6
:1003A000100010BD8268FBE7780900207909002061
:1003B0007A0900208803002084030020D2235B00F8
:1003C0005843134AF0B51368000C984206D2114CFA
:1003D0002368013323601368203B13601F2305004B
:1003E00001270D4E9D431468A5420BD803401A1DEA
:1003F000202A00D92022094C2468934204D3084BB8
:100400001860F0BD3770EEE7E51829710133F4E7A5
:10041000880300208C0300207A0900208403002038
:1004200090030020F0B5802787B02C4D02907F42CA
:100430002C78002C1CD063B2002B10DA6E1C6D7867
:100440007C40E4B2002D13D0013CE4B2FF2C0DD06F
:1004500004AB981D01210570F7F7BEF9F4E704AB72
:10046000D81D012104702E00F7F7B6F9751CDFE7DF
:100470000627013F002F2ED00298F7F7F7F9012445
:10048000BC42F6DA0025052D22D0154E22002900A7
:100490003000FBF70FFD6B4601901B79002B15D048
:1004A000631E1A00290030000393FBF703FD031EAF
:1004B0000CD1220029003000FBF7C4FCFF22019B75
:1004C000290013403000621EFBF7BCFC0135DAE75F
:1004D0000134E4B2D4E707B0F0BDC046C9A00300C0
:1004E0002400002010B5C820FFF79CFF004810BD75
:1004F000D8F5020010B5043000F0D2FB004810BD62
:10050000D8F5020010B5043017F07AF9004810BD94
:10051000D8F50200F0B50500080087B01400E9889E
:1005200002000023286803F0D9F80600002C16D03A
:10053000042C17D103204643AB6803A99E1901235D
:10054000727852001A43039232789A401A43049206
:10055000B2789A4013430593F5F7F8FB04002000A6
:1005600007B0F0BD03AA0321200003F0A3F8039B0A
:10057000186802F0DBFF039B0400586802F0D6FF06
:10058000039B0700986802F0D1FFFF2C03D8FF2FD0
:1005900001D8FF2805D90849084815F03FFD06F0A5
:1005A00006F9C0B20435E2B20090FBB2B1B2280045
:1005B00017F039F9024CD2E780A10300ACFD02002C
:1005C000D8F5020073B51C00002300930233080025
:1005D00011001A00FAF788F8206814F09FFE050051
:1005E000606802F0A3FF041E05DC0949094815F004
:1005F00015FD06F0DCF80C2015F0ADF90600064BF1
:10060000E9B208C0A2B200F025FB300076BDC046BA
:1006100067A10300ACFD020044170300014B186002
:1006200001487047100B0020D8F50200F8B50125ED
:10063000264B07001D7002F079FF102805D02449D1
:10064000244815F0EBFC06F0B2F8A1220021224B61
:10065000D200A22699500922F6009A5180208022C9
:100660008000D2021A501D481D4C1950A9211F208C
:10067000C9005850C12189005A508023C022C2208D
:10068000DB005200A3508000225816491140C022BE
:1006900012040A432250C0225200A35038002360A3
:1006A00002F044FF0300A0220C21C133FF339B0062
:1006B000D20599504023C12223600B4B00021843FE
:1006C0000A4B920098519D500948F8BD2A0B002012
:1006D0008FA1030034FD020000A0004004050000CB
:1006E00000E100E0FFFF00FF0100020000600040A9
:1006F000D8F502000B4B0C481A68C16C013210B5DA
:100700001A600A4B012907D1C124A4001C596403B3
:1007100002D50024C464D960C82A02DD01225A60CF
:10072000DA6010BD9C030020FCA0004000A0004047
:10073000F7B5474B5A680193012A22D1C123454995
:100740009B00CB5813421CD0434C444D23683C2B98
:1007500009DD002342490B8042494A60CA60424A8F
:1007600023602B7013702B78002B0BD101223D4995
:100770002A702360CA600A603C4A13600023019A11
:100780005360F7BD3A4E226833783A4F01333370E5
:1007900000230D2A35D1337023603349314B0C3A95
:1007A0000A70DA603B78012B06D132783249013A7F
:1007B00093400A6813430B603378202BDED100236B
:1007C00001212E4A1370274A5160D1602A4A2360C2
:1007D0001068234C010C218029492B70088080B2BD
:1007E000136015F0D6F9274D2860208815F0D1F94F
:1007F000254B02001860254B2968186816F02BFE5F
:10080000BCE7012A04D117492360CA603B70C9E7DD
:10081000022A04D123600123124AD360F6E70B2A8F
:10082000C0D101210F4A23605160D160134A2B705F
:1008300013785B18DBB21370052BB3D9124B1A680F
:10084000104B1968114B186816F005FEAAE7C04650
:10085000FC600040006000409C0300207E090020F6
:100860001809002000A000407C0900209803002007
:100870007B0900207F090020940300207D090020CF
:1008800016090020140B0020180B0020100B00206C
:1008900070B50500140016F091FE024B25606360F0
:1008A00070BDC0467B75020010B50C007F2906D8CC
:1008B000012116F0EBFE002800D0047010BD224B81
:1008C000994210D8022116F0E1FE0028F6D040230C
:1008D000A2095B42134303703F23234080246442F8
:1008E0001C434470EAE7194B994214D8032116F0CF
:1008F000CDFE0028E2D02023220B5B4213433F2190
:1009000080220370A30952420B400C401343224340
:1009100043708270D2E7042116F0B8FE0028CDD0D3
:100920001023A20C5B4213433F2103708023220B50
:100930005B420A401A434270A2090A400C401A4323
:100940001C438270C470B9E7FF070000FFFF00007E
:1009500007B5034B00906846019305F0E1FA07BD27
:100960007B75020010B50400102014F0F4FF044B56
:1009700084600360034B43600023C36010BDC04626
:1009800040DE0200CD77020013B50400080001A983
:10099000F8F784F8002C03D0012C07D0002004E0E5
:1009A000019B0548002B00D1044816BD019918F0A1
:1009B0001EFB40002043F8E710D6020008D60200D4
:1009C000F0B585B00400080003A91500F8F766F833
:1009D0000600002D07D10300039A2F49200018F0CC
:1009E000B4FC05B0F0BD039B0200C3180021012038
:1009F0000193019B934206D82727002900D0053F89
:100A00003A0026491AE01378272B08D0223B5D4292
:100A10006B41DBB20132002BEBD02727F0E700233C
:100A20000100F7E7300018F0AFFA0500300018F0C9
:100A3000C6FA0600AF4205D13A001949200018F065
:100A400084FC14E017495C2D0ED02B00203B5E2B5C
:100A500001D82A00D5E714490A2D05D013490D2DD8
:100A600002D0092D0CD11249200018F0A3FB019BE4
:100A7000B342D7D83A000949200018F066FCB0E725
:100A8000FF2D02D82A000B49D8E70B4B2A000B494F
:100A90009D42D3D90A49D1E7137A03008279030032
:100AA0008179030085790300887903008B7903003D
:100AB0008E79030091790300FFFF0000E3A103009A
:100AC000EAA10300F7B51E0008AB0C0017001D7863
:100AD000F30715D576100196019BE219002B2BDA4E
:100AE00000213F260127501E84421BD9002900D037
:100AF0000193002D3BD11F491F48FBF7E1FB0DE09F
:100B000001A9300002F050FD0028E5D1300018F0B6
:100B100043F81A4902001A48FBF7D2FB05F047FEDA
:100B20001000E1E70278B243802A01D03900013396
:100B3000421E002BF4D1FEBD002B18D000213F2710
:100B4000012694420AD220000178B94380290CD0B2
:100B5000002BF0D0441C013B3100F2E7002900D00B
:100B600001931000002DE6D1C5E70130ECE720002D
:100B7000E1E7C046C9A1030004FA0200A1A10300F5
:100B800034FD0200F0B587B006000D00170002F03A
:100B9000E5FB02A904003000F7F780FF0600042FF0
:100BA0004FD1AB0736D1284B2A689A4232D105ABD8
:100BB00004AA03A9280018F03EF8059B234FBB4266
:100BC00004D0032B02D02248FFF746FA039B3500DE
:100BD000BB4207D00122310000922000029AFFF7A9
:100BE00071FF0500049BBB4211D00122310000922D
:100BF0002000029AFFF766FF06000E20B54204D8D7
:100C0000721B2900200014F061FD07B0F0BD029BAB
:100C1000F618F2E70023029A009331002B0020001F
:100C2000FFF750FF0278012153B2002B02DA402374
:100C30001A4203D10122F7F7F7FEE6E701315B081C
:100C4000F6E70020E1E7C046B81E0300D8F5020031
:100C500004630300F7B5032633000C00534305007B
:100C600018001700019310F07FFE2300A022C1336B
:100C7000FF33D2059B0068602C706F809E5001236B
:100C8000A340064953500022019BC318984200D14B
:100C9000F7BD0270427082700330F7E70C05000068
:100CA000F7B50400202010F05FFE7C4B06001860B2
:100CB000030005000327203301936088784310F078
:100CC00053FE019B01C5AB42F7D11022002394468D
:100CD000019362880199914234DB012322787049A3
:100CE0009340A022D205535032200138C046C0465E
:100CF000C046C046C046C046C046C046C046C046C4
:100D0000C046C046F1D1EFF3108672B66088032466
:100D10004443624800250768A1200194C000019C5B
:100D2000A54200D0BEE086F3108800255B4B1E680C
:100D30007059043510F022FE202DF7D1300010F04C
:100D40001DFEF7BD7F2162680425D21812780220AB
:100D50008A433168CA5440216268D21812780A4026
:100D60007168CA5420216268D21812780A40B168AA
:100D7000CA5461466268D21812780A40F168CA54AF
:100D800008216268D21812780A403169CA54626830
:100D90007169D21812782A40CA546268B169D218AF
:100DA00012780240CA5401216268F769D218127899
:100DB0000A40FA5467685A18FF187F787E318F43CB
:100DC00031688F546168CF1840217F780F40716877
:100DD0008F546168CF1820217F780F40B1688F54FD
:100DE0006168CF1861467F780F40F1688F54616861
:100DF000CF1808217F780F4031698F546168CF1870
:100E00007F7871692F408F546168CF187F78B169FE
:100E100007408F546168CF1801217F780F40F16936
:100E20008F5461681A18CF187F21BF788F433168BB
:100E30008F546168CF184021BF780F4071688F547C
:100E40006168CF182021BF780F40B1688F54616866
:100E5000CF186146BF780F40F1688F546168CF1892
:100E60000821BF780F4031698F546168CF18BF786F
:100E700071693D408D546168CD18AD78B1692840E5
:100E800088546168C8180121807803330140F069F3
:100E90008154019A013201921BE7C046A003002051
:100EA0000C0500003C68645D1350002C00D07BE012
:100EB000C0465350C046C046C046C046C046C04665
:100EC000C046C0467C68645D1350002C00D076E0BC
:100ED000C0465350C046C046C046C046C046C04645
:100EE000C046C046BC68645D1350002C00D071E061
:100EF000C0465350C046C046C046C046C046C04625
:100F0000C046C046FC68645D1350002C00D06CE005
:100F1000C0465350C046C046C046C046C046C04604
:100F2000C046C0463C69645D1350002C00D067E0A9
:100F3000C0465350C046C046C046C046C046C046E4
:100F4000C046C0467C69645D1350002C00D062E04E
:100F5000C0465350C046C046C046C046C046C046C4
:100F6000C046C046BC69645D1350002C00D05DE0F3
:100F7000C0465350C046C046C046C046C046C046A4
:100F8000C046C046FC69645D1350002C00D058E098
:100F9000C0465350C046C046C046C046C046C04684
:100FA000C046C0460135BAE6C046C046C046C04647
:100FB000C046C046C046C046C046535082E7C04601
:100FC000C046C046C046C046C046C046C046C046F1
:100FD000535087E7C046C046C046C046C046C046DC
:100FE000C046C046C04653508CE7C046C046C046C7
:100FF000C046C046C046C046C046C046535091E7B2
:10100000C046C046C046C046C046C046C046C046B0
:10101000C046535096E7C046C046C046C046C0468C
:10102000C046C046C046C04653509BE7C046C04677
:10103000C046C046C046C046C046C046C0465350E3
:10104000A0E7C046C046C046C046C046C046C046EF
:10105000C046C0465350A5E7FF2310B50324DB0567
:10106000CB18A3430200181CA24204D0042A0BD0C0
:101070000021002A01D0080010BD09F06DFC0749CD
:101080000028F8D00649F6E78022022112069B18B4
:10109000A3431943034BC918EDE7C04610D602001D
:1010A00008D6020000008080FF23DB0510B5040095
:1010B000C81803239843002386B001930733009395
:1010C0001022603302A9F5F74BFA02A9200018F0AC
:1010D00071F82E2102A81AF077FD00280FD16521A2
:1010E00002A81AF071FD002809D16E2102A81AF099
:1010F0006BFD002803D10349200018F05BF806B00F
:1011000010BDC0463B39030030B50C001100002271
:1011100085B01D00009201232000F9F7E5FA002CAC
:1011200023D02868124B0340062B06D0032420420C
:101130000ED1104B02689A420AD103A9F8F722F99E
:10114000002203990092130005F03AF905B030BD72
:1011500003002340022BF9D002F04CFA03000220D6
:10116000A3431843044BC018F0E70448EEE7C04619
:10117000070080FF081803000000808002008080C4
:10118000F0B5050087B01000019102F033FA041C9D
:101190000390681F182800D9B2E009F0FFF90D127A
:1011A0001F2435407176B1B1B1B1B10D121F243594
:1011B0004071949DA2A7AC000198211C09F022FD6A
:1011C00003E0211C01980AF0BFF901900323019864
:1011D0004C4A9843013B03439B1871E0211C019842
:1011E0000AF092F8F1E70021201C09F0B5FB002875
:1011F00005D04549454814F011FF05F0D8FA03A978
:1012000001A816F021FBE1E70021201C09F0A4FB56
:101210000028EED1211C019809F086FED5E70021B7
:10122000201C09F099FB0028E3D1211C01980CF047
:101230001FFF0021041C019009F08EFB002807D03D
:10124000039A0023002A01DA80231B060193BDE7DD
:101250000021201C039E012709F084FB002800D1F7
:10126000071C0021301C012509F07CFB002800D15F
:10127000051CFFB2EDB2AF42A8D0311C201C9DE787
:10128000211C01980CF0D8FF9FE70021201C09F0D9
:1012900063FB0028ADD103A901A816F0D5FA0322FB
:1012A0000220019B1749934303435B180493039B5C
:1012B000934303435B1804A90593F4F747FD030028
:1012C000180007B0F0BD0199201C09F05FFB104B1E
:1012D0000028F5D10F4BF3E70199201C09F042FBE0
:1012E000F5E70199201C09F037FBF0E70199201C74
:1012F00009F056FBEBE70199201C09F03DFBE6E7FE
:101300000023DDE7000080807F7B0300F4FD020006
:1013100010D6020008D6020010B502F06BF90CF0EE
:10132000CDF80022084B0BF0BDFA084A084B0AF032
:1013300085FE0CF015F90323020002209A43054BA9
:101340001043C01810BDC04600806640182D44549C
:10135000FB2109400000808010B502F04BF90CF031
:10136000ADF8094A094B0BF09DFA0022084B0AF030
:1013700065FE0CF0F5F80323020002209A43054BAA
:101380001043C01810BDC046182D4454FB2109401D
:10139000008066400000808010B502F02BF9011C2F
:1013A0000AF06EFA024B002800D1024B180010BD63
:1013B00010D6020008D6020010B502F01BF9440056
:1013C00064080849201C0AF05BFA002805D1054989
:1013D000201C09F0DBFA002801D0034810BD0348A7
:1013E000FCE7C046FFFF7F7F08D6020010D6020050
:1013F00010B502F0FFF8034B034002201843024BE4
:10140000C01810BDFCFFFF7F0000808010B502F007
:10141000F1F8440064080849201C0AF031FA002859
:1014200007D10549201C09F0A7FA002801D103487B
:1014300010BD0348FCE7C046FFFF7F7F10D60200C7
:1014400008D602001FB50023019302F0D3F801A9CA
:101450000CF080FB03220300022093430649034360
:101460005B180293019B934303435B1802A9039308
:10147000F4F76CFC05B000BD0000808070B50D0075
:1014800002F0B8F8041C280002F0B4F80AF010FAD0
:101490000100201C0CF03AFB0323020002209A43B7
:1014A000014B1043C01870BD000080801FB50023A1
:1014B000019302F09FF801A90CF0FEFA0323022425
:1014C0009843074B2043C0180290019814F061FB29
:1014D00002A903902000F4F739FC04B010BDC04607
:1014E0000000808070B50D0002F084F8041C280014
:1014F00002F080F8011C201C0CF0BAFD032302004E
:1015000002209A43014B1043C01870BD0000808038
:1015100070B50D0002F06EF8041C280002F06AF8A5
:10152000C00FC307600040081843032302249843F8
:10153000014B2043C01870BD0000808070B50D00C5
:1015400002F058F8041C280002F054F8011C201C7A
:101550000CF016FD0323020002209A43014B1043B6
:10156000C01870BD0000808010B502F043F80CF088
:10157000ABF80323020002209A43024B1043C01829
:1015800010BDC0460000808010B502F033F80CF0AA
:10159000A3FC0323020002209A43024B1043C0180D
:1015A00010BDC0460000808010B502F023F80CF09A
:1015B0003FFC0323020002209A43024B1043C01851
:1015C00010BDC0460000808010B502F013F80CF08A
:1015D000A5FB0323020002209A43024B1043C018CC
:1015E00010BDC0460000808010B502F003F80CF07A
:1015F00057FB0323020002209A43024B1043C018FA
:1016000010BDC0460000808010B501F0F3FF0CF063
:10161000C3F90323020002209A43024B1043C0186F
:1016200010BDC0460000808010B503490348FAF79A
:1016300047FE05F0BCF8C046F1A10300ACFD020076
:1016400070B5060008680D0001F0D4FF0021041CED
:1016500009F092F9002801D0FFF7E6FF201C0CF0FA
:101660006FFD041C012E06D1032302209C4320435E
:101670000C4BC01870BD686801F0BCFF0021051C50
:1016800009F07AF90028E7D1281C0CF059FD011C5B
:10169000201C09F049FC0323020002209A43104356
:1016A000E6E7C0460000808010B501F0A3FF0CF013
:1016B0006BFC0323020002209A43024B1043C01824
:1016C00010BDC0460000808070B50D0001F092FF93
:1016D000041C280001F08EFF011C201C0CF0ACFD46
:1016E0000323020002209A43014B1043C01870BD2F
:1016F0000000808010B501F07DFF0021041C09F07E
:1017000031F9002801D0FFF78FFF201C0CF028FFD3
:101710000323020002209A43014B1043C01810BD5E
:101720000000808030B585B003AB050014000800D0
:1017300002AA01A917F07FFA019A164900238A42EA
:1017400000D0531002984210884200D12A00002B8A
:1017500015DA5B19D843C0170340002A13DA52196F
:101760002360934200DA13006360039B8B420ED028
:10177000032B0CD000205B10A36005B030BD9D4250
:10178000EBD22B00E9E79542EAD22A00E8E70120F4
:10179000A060F2E7D8F50200F0B5060085B01700AA
:1017A0001B2805D10A9A974209D0002005B0F0BD48
:1017B00019281AD01C281AD00A9A0A9717001A005A
:1017C0000B0011000A9A0192BA4200D901971D003C
:1017D0000C0000230093009B019A934209D10A9BBD
:1017E000BB4220D0E1D30120E0E71A26EAE71D261C
:1017F000E8E70295039401CD02CC01F045FE0028F4
:1018000002D0009B0133E5E71B2ECED0039B3000B6
:101810001A68029B1968FDF7FFFE044BC01A434289
:101820005841C0B2C2E71A2EDDD1BEE710D6020081
:10183000F0B51E0085B0039018680D00170001F088
:101840008DFD7368019002930024022F0ED90123AD
:10185000B268290001F042FF0400032F06D02900DE
:101860000123F268019801F039FF0500A54205D86F
:101870000A490B4814F0D2FB04F099FF039AA30025
:101880000299D05801F000FE002801D10134EDE7A3
:1018900001206400204305B0F0BDC04603A2030050
:1018A000ACFD020010B54379012B03D1C06A13F0DF
:1018B00079FB10BD0B00C26A0249006B13F0AEFB4E
:1018C000F7E7C0469001030010B54379012B03D11F
:1018D000C06A13F087FB10BD0B00C26A0249006B9F
:1018E00013F09CFBF7E7C046A001030010B5437955
:1018F000012B03D1C06A13F075FB10BD0B00C26A47
:101900000249006B13F08AFBF7E7C0468001030031
:1019100010B5024B3F2216F02FF910BD6985020069
:1019200010B5024B912216F027F910BD852A01004F
:10193000F7B50F0011001A00C38AC579868A019392
:1019400000230400C3718382C382104B16F014F984
:10195000A368002B18D1E18A002908D0A38A002BA4
:1019600005D1206B14F0C0FF206B14F050FEA38A49
:10197000E28A3900200016F0AFF86B1E9D416B46DD
:101980009B88E571A682E382F7BDC04695260100DB
:10199000836870B504000D00002B09D111000548C3
:1019A00014F03CFBA060200029000C3016F04BF92D
:1019B00070BDC046B0FC0200F0B58DB06B46019220
:1019C0001B79040043710123E16203610B780D0070
:1019D000012B06D00021954A2000FFF7D9FF0DB05A
:1019E000F0BD019B012B07D9836B0A001E68030021
:1019F00001990833406BB047AB681800049312F0AC
:101A0000DEFF63790490032B0FD109900C2109A804
:101A100012F0EEFFA36B02009B680999606B984778
:101A2000A3686883002B00D0BCE0049812F0C7FFC5
:101A300004900378002B3AD00A3B0F2B32D809A927
:101A400016F01EF8099B772B2AD006D803220292A3
:101A5000312B08D0764A0499BEE7812B1DD0022293
:101A60000292992BF6D1049812F0A9FF5A21049002
:101A700004A812F0BDFF049D0390039B9D4218D162
:101A80006379012B04D9A36B02995B68606B98475B
:101A9000A368002B00D085E0A1E701230293E2E7D1
:101AA0000023FBE70100634A2000FFF771FF0223D8
:101AB000F4E704952B78432B04D1280012F07FFF24
:101AC0000500DAE7392B01D05B4AC4E705A92800F5
:101AD00012F07FFF03780600912BF5D112F06FFF13
:101AE000059B9842F0D105A9300012F072FF0378EF
:101AF00007000A3B0F2BE7D812F061FF059B060099
:101B00009842E1D00378A02BDED112F058FF059B5C
:101B10009842D9D106A9380015F0B2FF300012F072
:101B200053FF9C21079007A812F062FF010007985D
:101B300012F039FF069B06002E2B1BD1012804D181
:101B4000079803780A3B0F2B01D93C4A83E72669A3
:101B5000731C2361019B012B21D909A915F090FF6A
:101B6000A36B099ADB683100606B9847002816D197
:101B7000334A70E72F2B1BD1012803D10798037834
:101B8000032B01D02F4A66E7019B012B07D9A36BDA
:101B9000676B1E6912F0F3FE01003800B047A368BE
:101BA000002B8AD0200004990C3016F04CF816E770
:101BB000302B23D1012803D907980378032B01D0B8
:101BC000214A48E7019B012BE9D908A912F0C8FE78
:101BD0000127079007980378032B01D01B4A3AE7A7
:101BE00009A912F0BDFEA36B07905B69099A0899D9
:101BF000606B01379847BE42ECD1D0E7019B012BC7
